:0900000C32362E322E302E313234
:0100000B01F3
:1000000AE8312517E218070AF01515F31D21F6360F
:1000000A231215FB191CFE07070508070C09120F16
:1000000A0A51453702574A543911554A300B505C48
:1000000A603F1A353B1D373B202A2D292E322D2DD4
:1000000A3135302D503254255B4A4D33735E623799
:0500000A5C623A7A5827
:020000040800F2
:40800000F8ED0020397A0408417A040859860408457A0408477A0408497A040800000000000000000000000000000000158300084D7A040800000000CD83000831840008DB
:40804000537A0408537A0408537A0408537A0408537A0408537A0408F91D0108031E01080D1E0108171E0108211E0108537A0408537A0408537A0408E1D40008537A0408C6
:40808000537A0408537A04084BF900087F3014088930140893301408537A04082B1E0108537A0408537A0408537A0408537A0408537A0408537A0408537A0408537A040850
:4080C000537A0408D7BD0008E1BD0008537A0408537A0408537A0408537A0408EBD40008511E0108537A0408537A0408537A0408537A0408537A0408537A0408537A0408D3
:40810000537A0408537A0408537A0408537A0408537A0408537A0408851E01080944140827F900083FF9000833F90008914114089B411408537A0408537A04089D301408F7
:40814000A7301408B1301408537A0408537A0408537A0408537A0408537A0408537A0408537A0408537A0408537A0408537A0408537A0408537A0408537A0408000000000A
:40818000537A0408537A0408537A0408537A0408537A0408537A0408537A0408537A04080000000000000000537A040800F002F800F05AF80AA090E8000C82448344AAF19C
:4081C0000107DA4501D100F04FF8AFF2090EBAE80F0013F0010F18BFFB1A43F001031847885A0A00C85A0A0010F8013B0A4413F0030408BF10F8014B1D1108BF10F8015B29
:40820000641E05D010F8016B641E01F8016BF9D1002D15D010F8014B03F00C030C2BA1EB04040ABF10F8013BA4EB8314A4EB032405F1010314F8016B5B1E01F8016BF9D588
:40824000914238BF10F8013BD1D370470023002400250026103A28BF78C1FBD8520728BF30C148BF0B6070478EF1D9FF114637F10FFF0FB400F00CF80FBC38F14AFE7BF129
:4082800034FE03B437F11EFF03BC40F09DF8000004B08FF1D1FE044800218FF183FF8FF1DDFE7BF122FE00007C20001080F309887047EFF309807047684680F3098804482C
:4082C0000078C00714BF0220032080F31488704738CD1908DFF818C0EFF305831B0618BF6047EFF31483DB0708BF604700DF704705821908DFF818C0EFF305831B0618BF6B
:408300006047EFF31483DB0708BF604700DF7047A58E0408EFF30980816911F8021CE1BB90E80F1010B5E047BDE81040EFF3098C8CE80700214B93E80600914208BF704738
:4083400041B91EF0100F16D11D49086820F00100086010E01EF0100F06BF2CED108A0120002081F825002CE9F00FC1F828C00CB441F032F80CBC1A60D2F828C0BCE8F00FC5
:4083800092F8250000280EBF6FF0020E6FF0120EBCEC108A8CF30988704710B5094A1268914209D8084C54F8214090E80F10A047EFF3098C8CE80F0010BD00008C200010DA
:4083C00034EF00E0247A1908247A190810B590F1E7F8BDE81040154B93E80600914208BF7047EFF3098C1EF0100F06BF2CED108A0120002081F825002CE9F00FC1F828C000
:408400000CB440F0E9FF0CBC1A60D2F828C0BCE8F00F92F8250000280EBF6FF0020E6FF0120EBCEC108A8CF3098870478C20001010B590F15FF9CCE710B540F0B5FC90F1FE
:4084400059F9C6E740BA7047C0BA704770472DE9F04F2DED028B85B00020049003900290302040F0C3FA054682F196FF05462E46002002F0FBFABCEEC00A10EE107AAFF267
:4084800033023946304683F156F8002002F0CDFAB0EE408AAFF24B01304683F15FF832460021FE4848F1FAFA03A9FD4801F00DF800285BD002A9FA4801F00FF8002855D0E9
:4084C00000241C2040F092FA0746DDE9022121F0E7F80746B946B7EE000A484621F066F9642040F083FA804682F1B8FA8046C2464946504682F1A5FC204602F01FFA8346E4
:40850000AFF2B7025946504682F1EAFB204602F05FFABCEEC00A10EE10BAAFF2CF025946504682F1CAFB02F0CBFB012813DD01F04BFF834602F0C4FBBBFBF0FB02F0C0FBB4
:40854000401E0BFB00FBAFF2FB0259465046CDF804B082F121FD52462146D04847F116F852462146304683F1E3F800BF03A9CC4800F09BFF002855D002A9C94800F09DFF00
:4085800000284FD002241C2040F030FA0746DDE9022121F085F80746B946B7EE000A484621F004F9642040F021FA804682F156FA8046C2464946504682F143FC204602F008
:4085C000BDF98346AFF27B125946504682F188FB204602F0FDF9BCEEC00A10EE10BAAFF293125946504682F168FB02F069FB01280DDD01F0E9FE834602F062FBBBFBF0F0D9
:40860000AFF2B71201460190504682F1C5FC52462146A24846F1BAFF52462146304683F187F800BF049805B0BDEC028BBDE8F08F2DE9F84F01249B49984821F00DFA974846
:4086400046F1D5FF0020009000BF0221944800F0ECFD934800F0D9FE02F045FB0546AFF2132229468D4847F1AAFE02F059FB0546AFF227222946894847F1BAFE02F062FB95
:4086800008B1012000E000200546AFF23F222946824847F1C6FE01F07BFDC0EB00108500AFF2572229467D4847F11FFF01F07FFDC0EB00108500AFF26B222946774847F1D0
:4086C000E2FE01F084FDC0EB00108500AFF283222946724847F1F0FE01F0EAFD0546AFF2932229466D4847F1B5FE01F03CFE824650468DF13EFFC5B2AFF2AF232A46514696
:40870000664847F124FF01F04CFE0546AFF2C3222946624847F146FF01F069FE0546AFF2D32229465D4847F156FF01F099FE08B1012000E000200546AFF2EF222946574847
:4087400047F162FF01F079FE08B1012000E000200546AFF207322946504847F16EFF01F059FE08B1012000E000200546AFF2233229464A4847F176FF01F084FF0546AFF2DC
:4087800033322946454848F169F801F08EFF0546AFF247322946414848F179F802F087F90546AFF2573229463C4848F1C3F802F091F90546AFF26B322946384848F1B3F992
:4087C00002F09BF90546AFF27B322946334848F1DCF902F0A5F90546AFF28F3229462F4848F1E8F902F020FA0546AFF29F3229462A4848F1C3FA02F02AFA0546AFF2B3329E
:408800002946264848F1D3FA02F034FA0546AFF2C3322946214848F1E3FA02F051FA0546AFF2D73229461D4848F111FB01F0CCFE0546AFF2E7322946184848F1DBFB01F08C
:40884000D6FE0546AFF2FB322946144848F1EBFB01F0DFFE0546AFF20B4229460F4848F1FBFB01F0E9FE0546AFF21F4229460B4848F107FC01F0F3FE0546AFF22F42294654
:40888000064848F113FC01F0D8FD01284ED101F0FAFD0546AFF24B42294605E0381E00209C200010A9AD0008F04847F1F4FE01F0FDFD0546AFF26B422946EC4847F104FFFB
:4088C00001F007FE0546AFF27B422946E74847F114FF01F011FE0546AFF28F422946E34847F126FF01F024FE0546AFF29F422946DE4847F136FF01F02EFE0546AFF2B3425C
:408900002946DA4847F146FF01F038FE0546AFF2C3422946D54847F156FF01F042FE0546AFF2D7422946D14847F166FF01F072FD01281ED16946CE4800F0D7FDC8B12820DB
:4089400040F054F80546009983F182FC0546A846202040F04BF8064620F0DBFD064637464146384620F0B2FD3946C04846F175FD00BF01F075FD012859D100256946BC487B
:4089800000F0C3FD20B3182040F030F80646009920F01EFF0646B0469FEDB60A404620F08BFF2C2040F022F8074683F1E2FA07463D464146284683F1AAFAAFF26F52012150
:4089C000284683F173FB2946A84846F1A6FC00BF6946A74800F091FD40B3182040F006F80646009920F0F4FE0646B0469FEDA10A404620F061FFA8203FF0F8FF074683F1B6
:408A00004AF80746B9464146484683F107F82946484682F1FEFFAFF2CB520021484683F1F3F84946914846F1D9FC00BF00BF02F08AF80546AFF2EB5229468C4847F122F8C3
:408A400002F0A6F80546AFF2FB522946874846F1E7FF02F0C3F80546AFF20F622946834846F1A2FF02F081F80546AFF21F6229467E4846F1EEFF02F09EF80546AFF233627C
:408A800029467A4846F1A9FF02F0BBF80546AFF243622946754846F16EFFFFF7D8FC04402046BDE8F88F10B581F129F801F095FE04461FF095FE01F07DFE04461EF0ECFD8B
:408AC00001F065FE044679F1C5F901F099FE044679F168FF01F0F3FE04461FF0C7FE01F0A2FE044681F150FB01F0B0FE04461EF053FA01F0BEFE04461FF0FAFE01F0CCFE78
:408B0000044678F1FFF801F0EDFE044676F142FE01F002FF044675F1B5FFFFF789FD00231A465549514820F040FF0023022252494E48A03020F039FF002303224E494B48E1
:408B4000703020F032FF002304224B494748283020F02BFF0023052247494448CC3020F024FF002306224449444820F01EFF0023072241494148303020F017FF00230822BE
:408B80003D493E486C3020F010FF002309223A493A48A03020F009FF00230A2236493748D43020F002FF00230B223349344820F0FCFE3448006830B100230C222E493148F9
:408BC000006820F0F2FE2F48006830B100230C2229492C48006820F0E8FE244848F18FF9224848F1F9F908F0ECFF02F0DCFF10BD08B5FFF758FF01F035FB10B1012801D192
:408C000014E000BF002001F044FB00F00CFD6FF07F4000F039F8684600F0FCFC28B1002301221549009820F0C0FE1AE001F02DFB10B101280DD000BF00F0F5FC684600F068
:408C4000E9FC28B1002301220B49009820F0ADFE05E000220121054848F1DBF800BF00BF00BF00BF012001F001FB08BD381E00209C2000106F12833AA9AD0008381F0020A3
:408C800058200020B41F001070B505466FF07F40281A00D100BF0A2001F00EFB002410E09FED180A204601F075FE9FED160A204601F09DFE9FED130A204601F0C1FE601C50
:408CC000C4B2042CECDB9FED0F0A002001F0B8FE9FED0C0A002001F0D4FE002001F0FEFE012001F0A5FF012001F0B5FF012001F0C5FF002001F018FF002002F027F800BF9F
:408D000000BF70BD0000000070470020684904E00A68824200D9086849680029F8D170470020634902E00A68104449680029FAD1704710B5FFF7F4FF5E490860FFF7E5FF9B
:408D40005D4908605D48007840B100205B4908705948016857480068FFF7D6FF10BD10B5FFF7E7FF10BD01465148814204D35448814201D8012070470020FCE700B50246FA
:408D80001046FFF7F0FF00BD024600207047704770472DE9F84F16461F460BAC94E83006DDF828800020009020602860062089F8000000208AF8000000210F980160109858
:408DC0000160B6F56F4F64D1412F60D1B8F1420F03D0B8F1430F58D128E037493548FFF7D3FF10B3334A1068334A11684122354B1A7042225A70344A904200D91046324AD1
:408E0000914200D911462F4B9870020ADA70020C1A7159710A0A9A710A0CDA7108222A601A4622600122009200BF2EE0FFF778FF20490860FFF769FF1F4908601D48036820
:408E40000846D0F800B041201E490870432048701D48834200D903461B48834500D9834618498B70180AC870180C087181F805B04FEA1B2088714FEA1B40C871082028604D
:408E8000084620600120009000BF00BF00BF00BF00BF00BF0098BDE8F88F10B50B48FFF776FF04460A4AAFF217113EF0EFFF10BDE8BF0220080000100C0000101000001005
:408EC000E8FF022011000010FDFFFF000400001000800008B0EE402AF0EE602AB4EEE11AF1EE10FA01D2B0EE611AB5EEC01AF1EE10FA02D0C1EE810A01E0F7EE000A20EE7F
:408F0000823AF7EE003A73EEE03AB0EE430A03EEA20A70470246B4EEE00AF1EE10FA01D2B0EE600AB5EEC00AF1EE10FA02D080EE801A01E0B7EE001A01EE902AF8EEE11AAA
:408F400021EE212AF7EE001A71EEC12A01EE901AF8EEE11A02EEA12AFDEEC21A11EE900A7047704770B504462046FFF7FAFF05463FF034FD70BD0000084B036041600272E4
:408F80007047704770B504462046FFF7FAFF05463FF024FD70BD014600207047E0CD0A082DE9F04104460D4616461F463A4631462046FFF7E1FF04460C482060E560204639
:408FC000BDE8F08110B504462046FFF7DAFF0446204610BD70B504462046FFF7F3FF05463FF0FCFC70BD01460320704708D20A08004870476CED0010FFFFFFFFFFFFFFFFD1
:409000008EF19EB992F1CCBD10B5044600202070606838B1606818B1606802685168884700206060A06838B1A06818B1A0680268516888470020A060E06838B1E06818B195
:40904000E0680268516888470020E060206938B1206918B1206902685168884700202061606938B1606918B1606902685168884700206061A06938B1A06918B1A06902685F
:40908000516888470020A061E06938B1E06918B1E0690268516888470020E061206A38B1206A18B1206A02685168884700202062606A38B1606A18B1606A02685168884741
:4090C00000206062A06A38B1A06A18B1A06A0268516888470020A062E06A38B1E06A18B1E06A0268516888470020E062206B38B1206B18B1206B02685168884700202063DE
:40910000606B38B1606B18B1606B02685168884700206063A06B38B1A06B18B1A06B0268516888470020A063E06B38B1E06B18B1E06B0268516888470020E063206C38B102
:40914000206C18B1206C02685168884700202064606C38B1606C18B1606C02685168884700206064A06C38B1A06C18B1A06C0268516888470020A064E06C38B1E06C18B156
:40918000E06C0268516888470020E064206D38B1206D18B1206D02685168884700202065606D38B1606D18B1606D02685168884700206065A06D38B1A06D18B1A06D0268EA
:4091C000516888470020A065E06D38B1E06D18B1E06D0268516888470020E06510BD10B5044600206060A060E06020616061A061E06120626062A062E06220636063A06381
:40920000E06320646064A064E06420656065A065E0652046FFF7F8FE204610BD10B504462046FFF7F1FE204610BD2DE9F04704460F462046FFF7E8FE2770207800287DD0E3
:40924000012802D002287AD100E000BF0C203FF0CDFB05460022522185F17BF9054660600C203FF0C3FB05460022532185F171F90546A0600C203FF0B9FB054600225421D1
:4092800085F167F90546E0600C203FF0AFFB05460022552185F15DF9054620610C203FF0A5FB05460022512185F153F90546606108203FF09BFB06463D2185F17DF9064656
:4092C000A06208203FF092FB06463E2185F174F90646E06208203FF089FB0646132185F16BF90646206308203FF080FB0646142185F162F9064660631C203FF077FB804692
:4093000001223F2184F1C0FF8046A0630C203FF06DFB054600223B2185F11BF90546E0630C203FF063FB054600223C2185F111F905462064606C68B90C2001E061E061E0BB
:409340003FF054FB81460022242185F185F98146606400BFA06C50B90C203FF047FB814600221D213BF0E3FE8146A06400BFE06C50B90C203FF03AFB814600221E213BF05C
:40938000D6FE8146E06400BF206D50B90C203FF02DFB814600221C213BF0C9FE8146206500BF606D50B90C203FF020FB8146012217213BF0BCFE8146606500BFA06D50B91F
:4093C0000C203FF013FB8146012218213BF0AFFE8146A06500BF606D08B9A06D80B1E06D70B90C203FF002FB8146172185F134F88146E065E06D01688A6A0121904700BFD5
:4094000000E000BF00BFBDE8F08710B5044603F0EBFD10BD0146087870470246002053680B600B6803B1012070470246002093680B600B6803B10120704702460020D36880
:409440000B600B6803B1012070470246002013690B600B6803B1012070470246002053690B600B6803B1012070470246002093690B600B6803B10120704702460020D36934
:409480000B600B6803B10120704702460020136A0B600B6803B10120704702460020536A0B600B6803B10120704702460020936A0B600B6803B10120704702460020D36AF0
:4094C0000B600B6803B10120704702460020136B0B600B6803B10120704702460020536B0B600B6803B10120704702460020936B0B600B6803B10120704702460020D36BAC
:409500000B600B6803B10120704702460020136C0B600B6803B10120704702460020536C0B600B6803B10120704702460020936C0B600B6803B10120704702460020D36C67
:409540000B600B6803B10120704702460020136D0B600B6803B10120704702460020536D0B600B6803B10120704702460020936D0B600B6803B10120704710B50448FFF7C4
:409580002EFE0446034AAFF26B313EF07FFC10BD9C2000100080000810B50446F94800688047E060002020746074A074E07420756075206881682046884710BD10B5044646
:4095C000204620F0BFF90446EF4820602046FFF7E3FF204610BD10B50446204620F0B8F90446204610BD70B504462046FFF7F3FF05463FF0F3F970BD70B50546012406E04D
:40960000E24B00222146284620F052FA641C202CF6D370BD01460020DD4A12680A600A6802B10120704710B5D948006848B918203FF0DCF90446FFF7C1FF0446D448046024
:4096400000BF10BD10B5D248006870B1D048006830B1CF48006800684168CD48006888470020CB4908603BF031F910BD3EB5002000900190029068468CF17BFFC4B22146B3
:40968000684600F073FE002000F08FFEC14800F09FFE012000F0AFFE012000F0BFFE002000F0CFFE002000F0DFFE002000F0EFFE002000F0FFFE002000F00FFF002000F0DA
:4096C00029FFB54800F038FFB44800F048FFB44800F058FFB34800F068FF002000F0D6FF002000F0E6FF002000F0F6FF002001F006F8002001F016F8002001F026F80020FA
:4097000001F036F8002001F0DFFAFA2000F060FF4FF4FA6000F06FFF41F2707000F07DFF40F27E3000F08CFF40F6F85000F09BFF3EBD0146487D70470146087C704710B5D5
:40974000044600F0A2FD10BD2DE9F04107460C461546002600F099FDA04208D0204600F098FD2B4632460321384620F0A1F93046BDE8F08110B5044600F0F5FD10BD2DE91C
:40978000F04707460D4614469846002600F0EBFD8146142C01DA204600E014200246294648463EF0A6FB48B12146284600F0DEFD434632460421384620F07AF93046BDE851
:4097C000F08710B5044600F0ECFD10BD2DE9F04107460C461546002600F0E3FDA04208D0204600F0E2FD2B4632460521384620F05FF93046BDE8F08110B5044600F0E4FDB6
:4098000010BD2DE9F04107460C461546002600F0DBFDA04208D0204600F0DAFD2B4632460621384620F044F93046BDE8F08110B5044600F0DCFD10BD2DE9F04107460C4653
:409840001546002600F0D3FDA04208D0204600F0D2FD2B4632460721384620F029F93046BDE8F08110B5044601F02AFA10BD2DE9F04107460C46154600263846FFF7F2FFBE
:40988000A04208D0204601F01FFA2B4632460821384620F00DF93046BDE8F08110B5044600F0B8FD10BD2DE9F04107460C461546002600F076FEA04208D0204600F075FE7D
:4098C0002B4632461321384620F0F2F83046BDE8F0812DE9F04107460C461546002600F04DFEA04208D0204600F04CFE2B4632461221384620F0DCF83046BDE8F0812DE92B
:40990000F04107460C461546002600F024FEA04208D0204600F023FE2B4632461121384620F0C6F83046BDE8F0812DE9F04107460C461546002600F0FBFDA04208D0204631
:4099400000F0FAFD2B4632461021384620F0B0F83046BDE8F0812DE9F04107460C461546002600F0C9FDA04208D0204600F0D2FD2B4632460F21384620F09AF83046BDE8D4
:40998000F0810000AC030020B4D20A085B88040800000010E4D914013A9B220089C31400C5610A00EC7503002DE9F04107460C461546002600F08DFDA04208D0204600F022
:4099C0008CFD2B4632460E21384620F071F83046BDE8F0812DE9F04107460C461546002600F064FDA04208D0204600F063FD2B4632460D21384620F05BF83046BDE8F08197
:409A00002DE9F04107460C461546002600F03BFDA04208D0204600F03AFD2B4632460C21384620F045F83046BDE8F0812DE9F04107460C461546002600F0FFFCA04230D0AF
:409A4000204600F0FEFC2A4600213846FFF7D8FF2A4600213846FFF7BDFF2A4600213846FFF7A2FF2A4600213846FFF774FF2A46FC493846FFF759FF2A46FB493846FFF732
:409A80003EFF2A46F9493846FFF723FF2A46F8493846FFF708FF2B4632460A21384620F007F83046BDE8F0812DE9F04107460C461546002600F0AEFCA0420DD0204600F0B2
:409AC000ADFC2A4600213846FFF7B0FF2B463246092138461FF0ECFF3046BDE8F08110B5044600F0AAFC10BD10B5044600F0B8FC10BD2DE9F04107460C461546002600F0A9
:409B0000AFFCA04208D0204600F0AEFC2B4632460B2138461FF0CCFF3046BDE8F08110B5044600F0B0FC10BD10B5044600F0BEFC10BD10B5044600F0CCFC10BD10B5044626
:409B400000F0DAFC10BD10B5044600F0F1FC10BD10B5044600F0FFFC10BD10B5044600F00DFD10BD10B5044600F01BFD10BD10B5044600F029FD10BD2DE9F04107460C4640
:409B80001546002600F020FDA04208D0204600F01FFD2B463246142138461FF089FF3046BDE8F08110B5044600F021FD10BD2DE9F04107460C461546002600F018FDA042F4
:409BC00008D0204600F017FD2B463246152138461FF06EFF3046BDE8F08110B5044600F018FD10BD2DE9F04107460C461546002600F00FFDA04208D0204600F00EFD2B46AE
:409C00003246162138461FF053FF3046BDE8F08110B5044600F010FD10BD2DE9F04107460C461546002600F007FDA04208D0204600F006FD2B463246172138461FF038FFDE
:409C40003046BDE8F08110B5044600F008FD10BD2DE9F04107460C461546002600F0FFFCA04208D0204600F0FEFC2B463246182138461FF01DFF3046BDE8F08110B50446C5
:409C800000F000FD10BD2DE9F04107460C461546002600F0F7FCA04208D0204600F0F6FC2B463246192138461FF002FF3046BDE8F08110B5044600F0F8FC10BD2DE9F0415A
:409CC00007460C461546002600F0EFFCA04208D0204600F0EEFC2B4632461A2138461FF0E7FE3046BDE8F08110B5044600F0F0FC10BD2DE9F04107460C461546002600F03E
:409D0000E7FCA04208D0204600F0E6FC2B4632461B2138461FF0CCFE3046BDE8F08110B5044600F0E8FC10BD2DE9F04107460C461546002600F0DFFCA04208D0204600F054
:409D4000DEFC2B4632461C2138461FF0B1FE3046BDE8F08110B5044600F0E0FC10BD2DE9F04107460C461546002600F0D7FCA04208D0204600F0D6FC2B4632461D213846C2
:409D80001FF096FE3046BDE8F08110B5044600F0D8FC10BD2DE9F04107460C461546002600F0CFFCA04208D0204600F0CEFC2B4632461E2138461FF07BFE3046BDE8F0811E
:409DC00010B5044600F0D0FC10BD2DE9F04107460C461546002600F0C7FCA04208D0204600F0C6FC2B4632461F2138461FF060FE3046BDE8F08101214174704700B50246B4
:409E00001046FFF796FC08B10120907400BD0121C174704701210175704770B504460D46607DA84206D06575124B0022012120461FF03EFE70BD70B504460D46207CA8424C
:409E40000ED000212046FFF7E8FF25740A4800688047E060074B0022022120461FF028FE70BD00003A9B220089C31400C5610A00EC7503005B880408AC03002070B50446CF
:409E80002046FFF759FC09287ED2DFE800F0050C264E6C9EE9F6F500FFF7E8FB01212046FFF7C9FF22E12046FFF764FC0546142298A13EF01EF820B101212046FFF7ADFF7F
:409EC00003E000212046FFF7A8FFA07C012803D102212046FFF7AFFF08E12046FFF771FC78B12046FFF788FC58B12046FFF79FFC38B100F0E5FE20B101212046FFF78DFFC3
:409F000003E000212046FFF788FFA07C012804D103212046FFF78FFF06E0607C012803D101212046FFF787FFE0E001212046FFF774FFA07C01280ED12046FFF7D0FD012828
:409F400004D104212046FFF776FF0BE006212046FFF771FF06E0607C012803D102212046FFF769FFC2E02046FFF7D9FD90B12046FFF7DAFD70B12046FFF7DBFD50B120468E
:409F8000FFF7DCFD30B100E0ABE001212046FFF744FF03E000212046FFF73FFF2046FFF79EFD10B92046FFF729FFA07C012804D105212046FFF73FFF06E0607C012803D14A
:409FC00003212046FFF737FF90E02046FFF7BBFD58B32046FFF7BCFD38B32046FFF7BDFD18B32046FFF7BEFDF8B12046FFF7ABFD05462046FFF7ACFD854216D32046FFF71B
:40A00000A7FD05462046FFF7A8FD85420DD32046FFF7A3FD05462046FFF7A4FD854204D301212046FFF7F9FE03E000212046FFF7F4FE2046FFF753FD10B92046FFF7DEFE33
:40A04000A07C012804D106212046FFF7F4FE06E0607C012803D104212046FFF7ECFE45E001212046FFF7D9FEA07C012806D107212046FFF7E0FE12E032E011E0607C012835
:40A080000DD12046FFF72BFD012804D105212046FFF7D1FE03E003212046FFF7CCFE25E001212046FFF7B9FEA07C012810D108212046FFF7C0FEFEF7F6FC00220121164896
:40A0C00046F1A7FE154A01212046FFF73DFB06E0607C012803D106212046FFF7ACFE05E004E008212046FFF7A6FE00BF00BF00206074A074E074207570BD10B50446204680
:40A10000FFF7BCFE2046FFF717FB082801D1FFF799FA10BD00000000381E00205B880408F74890F8A001704710B5044600BFF44880F8A041012200F5D071F24836F160FBAD
:40A1400000BF10BDEE4901F5D47103C9704770B504460D4600BFEA4800F5D47030C00822E949E848083036F14BFB00BF70BDE748704710B5044600BFE148C0F8B0410422B9
:40A1800000F5D871DF48103036F13AFB00BF10BDDB484068704710B5044600BFD84844600422011DDA4836F12BFB00BF10BDD4480068704710B5044600BFD1480460042213
:40A1C00001464FF0D04036F11BFB00BF10BDCC488068704710B5044600BFC9488460042200F10801CA48001D36F10AFB00BF10BDC348D0F8BC01704770B506460D46FFF782
:40A20000F7FF0446012E0CD12C4300BFBC48C0F8BC41042200F5DE71BA481C3036F1F0FA0CE0AC4300BFB648C0F8BC41042200F5DE71B4481C3036F1E3FA00BF70BDB0483B
:40A24000D0F8DC01704710B5044600BFAC48C0F8DC41042200F5EE71AA48743036F1D0FA00BF10BDA64890F8C801704710B5044600BFA34880F8C841012200F5E471A148D8
:40A28000603036F1BDFA00BF10BD9D4890F8E001704710B5044600BF994880F8E041012200F5F0719748783036F1AAFA00BF10BD934890F8E101704710B5044600BF90485E
:40A2C00080F8E141012200F2E1118E48793036F197FA00BF10BD8A4890ED740A704710B52DED028BB0EE408A00BF854880ED748A042200F5E8718348683036F181FA00BF73
:40A30000BDEC028B10BD7E4890ED750A704710B52DED028BB0EE408A00BF794880ED758A042200F5EA7177486C3036F169FA00BFBDEC028B10BD724890ED760A704710B591
:40A340002DED028BB0EE408A00BF6D4880ED768A042200F5EC716B48703036F151FA00BFBDEC028B10BD68483A30704770B504460D46142164483A308CF167F9142D01DA17
:40A38000284600E01420024621465F483A303DF054FE14225C493A315A487A3036F130FA70BD5748D0F8F801704710B5044600BF5348C0F8F841042200F5FC71514890307A
:40A3C00036F11EFA00BF10BD4D48D0F8FC01704710B5044600BF4A48C0F8FC41042200F5FE714848943036F10BFA00BF10BD444890F80002704710B5044600BF404880F8FB
:40A400000042012200F500713E48983036F1F8F900BF10BD3A4890F80102704710B5044600BF374880F80142012200F201213548993036F1E5F900BF10BD314890F8020280
:40A44000704710B5044600BF2D4880F80242012200F202212B489A3036F1D2F900BF10BD274890F80302704710B5044600BF244880F80342012200F2032122489B3036F1F4
:40A48000BFF900BF10BD1E48B0F80402704710B5044600BF1A48A0F80442022200F5017118489C3036F1ACF900BF10BD1448B0F80602704710B5044600BF1148A0F80642A6
:40A4C000022200F206210F489E3036F199F900BF10BD0B48B0F80802704710B5044600BF0748A0F80842022200F502710548A03036F186F900BF10BD0148B0F80A0270476B
:40A5000000210010A0010068A8220010C0D401000400006810B5044600BFFC48A0F80A42022200F20A21FA4836F16AF900BF10BDF648D0F8F802704710B5044600BFF348B7
:40A54000C0F8F842042200F53E71F148EE3036F157F900BF10BDED48D0F8FC02704710B5044600BFE948C0F8FC42042200F53F71E748F23036F144F900BF10BDE348D0F81F
:40A580000003704710B5044600BFE048C0F80043042200F54071DE48F63036F131F900BF10BDDA48D0F80403704710B5044600BFD648C0F80443042200F54171D448FA3055
:40A5C00036F11EF900BF10BDD048D0F80803704710B5044600BFCD48C0F80843042200F54271CB48FE3036F10BF900BF10BDC748D0F80C03704710B5044600BFC348C0F815
:40A600000C43042200F54371C24836F1F9F800BF10BDBE48D0F81003704710B5044600BFBA48C0F81043042200F54471B948001D36F1E6F800BF10BDB448D0F814037047CA
:40A6400010B5044600BFB148C0F81443042200F54571B048083036F1D3F800BF10BDAB48D0F81803704710B5044600BFA748C0F81843042200F54671A6480C3036F1C0F84D
:40A6800000BF10BDA14890F80C02704710B5044600BF9E4880F80C42012200F503719C48801C36F1ADF800BF10BD984890F80D02704710B5044600BF944880F80D42012238
:40A6C00000F20D219248C01C36F19AF800BF10BD8E4890F80E02704710B5044600BF8B4880F80E42012200F20E218948001D36F187F800BF10BD854890F80F02704710B56B
:40A70000044600BF814880F80F42012200F20F217F48401D36F174F800BF10BD7B48B0F81002704710B5044600BF7848A0F81042022200F504717648801D36F161F800BF22
:40A7400010BD724890F81202704710B5044600BF6E4880F81242012200F212216C48083036F14EF800BF10BD684890F81302704710B5044600BF654880F81342012200F221
:40A7800013216348093036F13BF800BF10BD5F48D0F81402704710B5044600BF5B48C0F81442042200F5057159480A3036F128F800BF10BD5548D0F81802704710B504465C
:40A7C00000BF5248C0F81842042200F5067150480E3036F115F800BF10BD4C48D0F81C02704710B5044600BF4848C0F81C42042200F507714648123036F102F800BF10BD11
:40A800004248D0F82002704710B5044600BF3F48C0F82042042200F508713D48163035F1EFFF00BF10BD3948D0F82402704710B5044600BF3548C0F82442042200F509715B
:40A8400033481A3035F1DCFF00BF10BD2F48D0F82802704710B5044600BF2C48C0F82842042200F50A712A481E3035F1C9FF00BF10BD2648D0F82C02704710B5044600BF49
:40A880002248C0F82C42042200F50B712048223035F1B6FF00BF10BD1C48D0F83002704710B5044600BF1948C0F83042042200F50C711748263035F1A3FF00BF10BD1348E6
:40A8C000D0F83402704710B5044600BF0F48C0F83442042200F50D710D482A3035F190FF00BF10BD0948D0F83802704710B5044600BF0648C0F83842042200F50E71044889
:40A900002E3035F17DFF00BF10BD0000002100104202006844030068FC48D0F83C02704710B5044600BFF948C0F83C42042200F50F71F74835F164FF00BF10BD0146002063
:40A94000042902DAF34A52F82100704770B504460D46042C0EDA00BFEE4840F82450EC4A121D02EB8400EB4A02EB8401042235F147FF00BF70BDDFEDE80AB0EE600A042807
:40A9800007DAE449103101EB8001D1ED000AB0EE600A704710B52DED028B0446B0EE408A042C12DA00BFDB48103000EB840080ED008AD74A143202EB8400D64A103202EB6B
:40A9C0008401042235F11CFF00BFBDEC028B10BDDFEDD10AB0EE600A042807DACD49203101EB8001D1ED000AB0EE600A704710B52DED028B0446B0EE408A042C12DA00BF99
:40AA0000C448203000EB840080ED008AC04A243202EB8400BF4A203202EB8401042235F1EFFE00BFBDEC028B10BDDFEDBB0AB0EE600A20B9B549D1ED9C0AB0EE600A704728
:40AA400010B52DED028B0446B0EE408A5CB900BFAE4880ED9C8A042200F51C71AC48343035F1CEFE00BFBDEC028B10BDDFEDAA0AB0EE600A20B9A549D1ED9D0AB0EE600AEB
:40AA8000704710B52DED028B0446B0EE408A5CB900BF9E4880ED9D8A042200F51D719C48383035F1ADFE00BFBDEC028B10BD9748D0F87802704710B5044600BF9348C0F8B2
:40AAC0007842042200F51E7191483C3035F198FE00BF10BD8D4890F87C02704710B5044600BF8A4880F87C42012200F51F718848403035F185FE00BF10BD8448D0F88002CA
:40AB0000704710B5044600BF8048C0F88042042200F520717E48443035F172FE00BF10BD7A48D0F8F402704710B5044600BF7748C0F8F442042200F53D717548B83035F100
:40AB40005FFE00BF10BD7148D0F83803704710B5044600BF6D48C0F83843042200F54E716E4835F14DFE00BF10BD6848D0F83C03704710B5044600BF6448C0F83C430422F1
:40AB800000F54F716548001D35F13AFE00BF10BD5E48D0F84003704710B5044600BF5B48C0F84043042200F550715C48083035F127FE00BF10BD5548D0F84403704710B561
:40ABC000044600BF5148C0F84443042200F5517152480C3035F114FE00BF10BD4B48D0F84803704710B5044600BF4848C0F84843042200F552714948103035F101FE00BF6C
:40AC000010BD4248D0F84C03704710B5044600BF3E48C0F84C43042200F553713F48143035F1EEFD00BF10BD384890F88402704710B5044600BF354880F88442012200F527
:40AC400021713348483035F1DBFD00BF10BD2F4890F88502704710B5044600BF2B4880F88542012200F285212948493035F1C8FD00BF10BD254890F88602704710B50446A9
:40AC800000BF224880F88642012200F2862120484A3035F1B5FD00BF10BD1C48B0F8CC01704710B5044600BF1848A0F8CC41022200F5E6711648703835F1A2FD00BF10BDFF
:40ACC000124890F8F002704710B5044600BF0F4880F8F042012200F53C710D48B43035F18FFD00BF10BD0948D0F81C03704710B5044600BF0548C0F81C43042200F54771CA
:40AD00000348E03035F17CFD00BF10BD00210010740200684023001000000000107500681248D0F82003704710B5044600BF0F48C0F82043042200F548710D4835F160FD36
:40AD400000BF10BD094890F82403704710B5044600BF064880F82443012200F549710448001D35F14DFD00BF10BD0000002100105803006870472DE9F04104460D46174672
:40AD80009846069EA0B2324629462FF0D4FC32462946204635F15AFB33462A462146F94851F1B2FFBDE8F0812DE9F84305460C4616461F46DDF820800F2C3ED2DFE804F05D
:40ADC00008162425262728292A2B2C2D2E3D3C00E0B23B463246002100902846FFF7CBFFE2B24146284679F165F82FE0E0B23B463246002100902846FFF7BDFFE2B24146B9
:40AE0000284679F157F821E000BF00BF00BF00BF00BF00BF00BF00BF00BF00BFE0B23B463246002100902846FFF7A5FFE2B24146284679F13FF809E000BFE0B23B463246D3
:40AE4000002100902846FFF796FF00BF00BFBDE8F88338B504460020034602460E2100902046FFF7A1FF38BDC7480068704738B5044600200090694620461DF0B2F940B11F
:40AE800000980068C149C269009890471720FFF7E0FF38BDBE480068704710B50446FFF7F9FFA04207D0BA4804601620FFF7D1FF2046FFF7DCFF10BDB6480068704710B5CA
:40AEC0000446FFF7F9FFA04207D0B24804601520FFF7BFFF0020FFF7E0FF10BD10B50446FFF7C2FFA04207D0A74804601420FFF7B0FF0020FFF7E3FF10BD10B51420FFF7F9
:40AF0000A8FF10BD10B51520FFF7A3FF10BD10B51620FFF79EFF10BD9F480068704738B50446FFF7F9FFA04215D09B480460002000906946204678F196F8009820B19748A6
:40AF4000009977F1B8FC02E0944877F123FB1820FFF77FFF00BF38BD91480068704710B50446FFF7F9FFA04204D08D4804601920FFF76FFF10BD10B51920FFF76AFF10BD00
:40AF800088480068704710B50446FFF7F9FFA04204D0844804601A20FFF75BFF10BD10B51A20FFF756FF10BD7F480068704710B50446FFF7F9FFA04207D07B4804601B2053
:40AFC000FFF747FF0020FFF7CAFF10BD10B51B20FFF73FFF10BD75480068704710B50446FFF7F9FFA04204D0704804601C20FFF730FF10BD10B51C20FFF72BFF10BD6C48ED
:40B000000068704710B50446FFF7F9FFA04204D0674804601D20FFF71CFF10BD10B51D20FFF717FF10BD63480068704710B50446FFF7F9FFA04204D05E4804601E20FFF77A
:40B0400008FF10BD10B51E20FFF703FF10BD5A480068704710B50446FFF7F9FFA04204D0554804601F20FFF7F4FE10BD10B51F20FFF7EFFE10BD51480068704738B5044628
:40B080004F4874F151FAA0420DD0002000906946204674F1CBFD4A48009974F113FB2020FFF7D7FE00BF38BD46480068704738B5044643484C3878F137F9A0420ED00020CF
:40B0C00000906946204679F191FC3D484C38009978F129FC2120FFF7BCFE00BF38BD3A480078704710B5044637480078A04204D0354804702220FFF7ACFE10BD33487047A0
:40B1000010B504462CB12068304982692046904703E014212D488BF198FA2320FFF799FE10BD2B48704710B504462CB12068284982692046904703E0142125488BF185FA0B
:40B140002420FFF786FE10BD2248704710B504462CB120681F4982692046904703E014211C488BF172FA2520FFF773FE10BD1A48704710B504468CB32068174982692046A2
:40B18000904730E0BC0100100C000020C8240010140000201000002018000020001F00201C0000202000002024000020280000202C00002030000020340000203800002088
:40B1C000542000203C00002040000020782400108C240010A0240010B4240010FFE7142104488BF132FA2620FFF733FE10BD024870470000B4240010C82400100246012040
:40B2000053798B4200D05171704710B504460020207100212046FFF7F1FF0020083460762076A080A076E0762077E0602082606154F8080920B1A0683DF0D0FB0020A06023
:40B24000206920B120693DF0C9FB0020206110BD70B504460D4625602046FFF7D6FF204670BD10B50446A06820B1A0683DF0B6FB0020A060204610BD0246002011717047BF
:40B2800001460879704710B50346002093F82140012C00D10220012403F8214F59709A70213B10BD014691F82000704701464879704730B5044600252046FFF7F7FF20B964
:40B2C00001212046FFF79AFF0125284630BD30B5044600252046FFF7E9FF042804D103212046FFF78BFF0125284630BD2DE9F04104460D46002700262046FFF7D7FF042803
:40B300001FD1206920B120693DF068FB0020206128468BF12EF900F1010840463DF062FB064628468BF125F900F101084246294630463CF082FE266106212046FFF75EFF20
:40B3400001273846BDE8F0812DE9F04104460D46002700262046FFF7A9FF04281FD1206920B120693DF03AFB0020206128468BF100F900F1010840463DF034FB0646284661
:40B380008BF1F7F800F101084246294630463CF054FE266107212046FFF730FF01273846BDE8F08130B5044600252046FFF77EFF092804D10B212046FFF720FF01252846D9
:40B3C00030BD2DE9F04105460F464FF00008002400262846FFF76AFF042817D101E0601C84B2385D0028FAD120463DF0FBFA064666B12246394630468BF1DAF80C212846BB
:40B40000FFF7FCFEAE60AC814FF001084046BDE8F0812DE9F04105460F464FF00008002400262846FFF742FF09281ED1A868E0B901E0601C84B2385D0028FAD1601C84B24A
:40B4400020463DF0CFFA06467EB12246394630468BF1AEF82C21601E3154AE60AC810A212846FFF7CBFE4FF001084046BDE8F0812DE9F04104460F464FF000080025002637
:40B480002046FFF713FF09281CD1A068D0B90B203DF0A8FA05463B46F7A20B2128463CF0CBFBC6B20B2E0DDC65B1002E0ADD2C21701E2954A560A6810A212046FFF79EFE18
:40B4C0004FF001084046BDE8F08130B5044600252046FFF7EBFE09280ED1A06860B92046FFF7E0FE40B9E548A0600120A0810A212046FFF783FE0125284630BD2DE9F0412C
:40B5000005460F464FF00008002400262846FFF7CDFE09281DD1A868D8B901E0601C84B2385D0028FAD1601C84B220463DF05AFA064676B12246394630468BF139F80A218F
:40B54000601E3154AE60AC812846FFF757FE4FF001084046BDE8F0812DE9F04104460D4616461F464FF000082046FFF79FFE09280FD175B1002E0CDD5FB165612683E761F6
:40B580000020E169088008212046FFF737FE4FF001084046BDE8F0812DE9F04104460F4615464FF0000800262046FFF77FFE092813D1A06888B928463DF014FA064666B10A
:40B5C0002A46394630468AF1F3FFA660A5810A212046FFF713FE4FF001084046BDE8F0812DE9F0430546894614461E46079FB846012C03D129464046FFF73EFE3246214605
:40B600004046FFF740FEBDE8F0832DE9F05F06468B4614461F46DDE90B8ADDF828905546012C0BD131462846FFF726FEE869A0F800804246494668698AF1BAFF3A46214600
:40B640002846FFF720FEBDE8F09F10B586B004468BA0006805908BA207CA02AB07C3206820B900212046FFF7C9FDDEE020684EF133FF20B900212046FFF7C0FDD5E094F883
:40B6800021000128F1D1002084F8210084F820002046FFF70BFE0F2816D2DFE800F0C1C00816BF24323380C3559BA9C2C40094F82200012804D103212046FFF79FFD03E0F6
:40B6C0000D212046FFF79AFDAEE094F82200012804D104212046FFF791FD03E005212046FFF78CFDA0E094F82200012804D103212046FFF783FD03E00D212046FFF77EFDDE
:40B7000092E000BF94F8220001280ED109212046FFF774FD206920B120693DF05FF900202061002084F824000DE094F82400052805DA94F82400401C84F8240003E00D21FC
:40B740002046FFF75BFD6FE094F8220001280FD1A06828B1A0683DF041F90020A060A08109212046FFF74AFD002084F8240015E094F82400052805DA94F82400401C84F8B8
:40B7800024000BE0A06828B1A0683DF027F90020A060A0810D212046FFF730FD44E094F82200012807D109212046FFF727FD002084F824000DE094F82400052805DA94F8DA
:40B7C0002400401C84F8240003E00D212046FFF715FD29E094F82200012804D104212046FFF70CFD03E00D212046FFF707FD1BE094F82200012804D104212046FFF7FEFCD8
:40B8000003E00D212046FFF7F9FCA06828B1A0683DF0E4F80020A060A08105E000BF00BF00BF00BF00BF00BF00BF94F8200000287AD12046FFF73AFD0F280AD2DFE800F0D9
:40B84000090A0F2DCA3E4F6492CB7AA6B7CC080000BFC2E002212046FFF7D0FCBDE0AFF27F23224605A920684EF1FAFE80B1012084F8200010E00000257500004600002077
:40B880005C0000002E5C4D434D43303135315C000D212046FFF7B2FC9FE0AFF2BB23224602A920684EF1DCFE18B1012084F8200003E00D212046FFF7A1FC8EE0AFF2DF23D4
:40B8C000224602A920684FF1DEF818B1012084F8200003E00D212046FFF790FC7DE0206968B1AFF20330009023460622216920684EF118FF18B1012084F8200003E00D2125
:40B900002046FFF77BFC68E0206970B1AFF22F30009023460322216920684EF103FF20B1012084F8200004E058E00D212046FFF765FC52E0A068A0B1A08990B1AFF25F3017
:40B94000CDE90040A389211DA26820684EF1B8FF18B1012084F8200003E00D212046FFF74DFC3AE0AFF25D30CDE90040238B211D626920684EF1EAFF18B1012084F8200078
:40B9800003E00D212046FFF739FC26E0AFF2AF332246211D20684EF104FF18B1012084F8200003E00D212046FFF728FC15E0AFF2CF30009023460022A16820684FF1C4F898
:40B9C00018B1012084F8200003E00D212046FFF715FC02E000BF00BF00BF00BF06B010BD10B5044620684EF177FD10BDF8B50746002405E0804800EBC4000471601CC4B2EA
:40BA0000152CF7DB7D488CF191FB7D4908607D488CF18CFB7A4948607B488CF187FB7849886035F124F979480068804705460AE04A2005F071FE18B10A203DF0F9F802E02F
:40BA400038F1CAFB054628461EF07DF8B0F5FA6FEED337F173FC35F17FF910B90020FEF705FC40F105F96A483DF042F969490860002169488CF196FB5F49086507E06420F6
:40BA80003DF0D6F8654800686430644908605A4890F855000B2805DA6048006842F210718842ECD301220021B52005F003FF37F11FF9FDF79DF8002159488CF173FB4E49D1
:40BAC0008861002157488CF16DFB4B490861002155488CF167FB48498860002153488CF161FB45490867002151488CF15BFB4249886500214F488CF155FB3F490866002172
:40BB00004D488CF14FFB3C49886400214B488CF149FB39490863002149488CF143FB36498862002147488CF13DFB3349C1F89800002145488CF136FB2F49086200214348E4
:40BB40008CF130FB2C498867002141488CF12AFB2949C1F8800000213E488CF123FB2649C1F890006846FDF755FD28B100213A488CF118FB20498866002138488CF112FB46
:40BB80001D49C1F8A000002088638CF123FB06468CF12CFBF8BD10B500211F488CF102FB1549086510BD10B51348006C28B900212B488CF1F7FA1049086410BD10B50E4800
:40BBC000D0F8880030B9002126488CF1EBFA0A49C1F8880010BD10B50748006A50B1064890F82500032805D10349086A4FF400413DF096F810BD0000F0080020BCBD1908C3
:40BC000098090020C0BD1908C4BD1908AC030020C8BD190848000010B4BE19084C000010F4BD1908E4BD1908D4BD190804BE1908A4BE1908C4BE190894BE190864BE190842
:40BC400074BE190884BE190854BE190824BE190814BE190844BE1908E4BE1908F4BE1908D4BE190834BE190810B5002807DA0A07140E6C4A00F00F031B1FD45403E00A0757
:40BC8000130E694A135410BD10B56848006820B967488CF14BFA65490860664885F1D7F8002164488160FE21C160002181614161C16101624FF4804101615F485D494860D9
:40BCC000084685F134F80B212120FFF7CDFF0B212220FFF7C9FF212000F099F8222000F096F810BD10B505F07CFD52480068006840F400404F49096808604E4800680068C2
:40BD000020F400404B49096808604A480068406948490968496988434649096848614548006880694349096889698843414909688861FFF7A9FF10BD2DE9F84304460D46A2
:40BD400016461F464FF001084FF47A71374800688CF110FA88B933462A4621463548009785F1FAF98046B8F1020F01D1FFF7BAFF2E4800683CF0B0FF01E04FF003084046A5
:40BD8000BDE8F8832DE9FE4304460D4616461F46DDF828904FF001084FF47A71234800688CF1E8F990B901232A46214621488DE8C00287F180F88046B8F1020F01D1FFF75E
:40BDC00091FF1A4800683CF087FF01E04FF003084046BDE8FE8310B5164888F1C8F910BD10B5144888F1CAFA10BD12480068006820F480600F490968086070470D48006848
:40BE0000006840F480600B4909680860704700F01F02012191404209920002F1E022C2F80011704718ED00E000E400E09C01002060D70408681D0020801A0600000000005C
:40BE40000000000000000000000000003037373031373134353500000000000030373730313731343335000000000000526176656E20496E647573747269657320496E633A
:40BE80000000000000000000000000004A756E2D32382D32303138000000000032362E322E302E313200000000000000556E766572666572746820477261696E204361729F
:40BEC00074204D6F64756C6500000000303737303137313533380000000000000000000000000000000000000000000000000000000000000000000000000000FFFFFFFF45
:40BF0000FFFFFFFFFFFFFFFFFFFFFFFFFFFFFFFFFFFFFFFFFFFFFFFFFFFFFFFFFFFFFFFFFFFFFFFFFFFFFFFFFFFFFFFFFFFFFFFFFFFFFFFFFFFFFFFFFFFFFFFFFFFFFFFF41
:40BF4000FFFFFFFFFFFFFFFFFFFFFFFFFFFFFFFFFFFFFFFFFFFFFFFFFFFFFFFFFFFFFFFFFFFFFFFFFFFFFFFFFFFFFFFFFFFFFFFFFFFFFFFFFFFFFFFFFFFFFFFFFFFFFFFF01
:40BF8000FFFFFFFFFFFFFFFFFFFFFFFFFFFFFFFFFFFFFFFFFFFFFFFFFFFFFFFFFFFFFFFFFFFFFFFFFFFFFFFFFFFFFFFFFFFFFFFFFFFFFFFFFFFFFFFFFFFFFFFFFFFFFFFFC1
:40BFC000FFFFFFFFFFFFFFFFFFFFFFFFFFFFFFFFFFFFFFFFFFFFFFFFFFFFFFFF00001408BFDC190800C00008FFF90A0804880008FBBF000800800008FF870008D02B9FE6C7
:40C0000039F019B970477047F0EE401A02EE101AB8EE422ADFEDFE2A82EE223AB0EE430A90ED142AD0ED062A9FEDFA3A62EE832A00EE222A80ED142A90ED122AD0ED132A8B
:40C0400002EE802AD0ED112A72EE222A90ED152A02EE802AD0ED102A32EE222A80ED102A90ED112AD0ED132A02EE802A80ED112A90ED122AD0ED132A02EE802A80ED122A38
:40C0800090ED132AD0ED162A32EE222A80ED132A90ED102AD0ED172A32EE222AD0ED102A82EE823AF0EE430A90ED102AD0ED172A32EE222AD0ED122A82EE823AB0EE431A03
:40C0C00090ED102AD0ED102A00EEE22A80ED102A90ED112AD0ED112A00EEE22A80ED112A90ED122AD0ED102A01EE622A80ED122A90ED132AD0ED112A01EE622A80ED132AF4
:40C1000090ED142AD0ED0E2A9FEDC23A12EE832AD0ED142A40EE822AC0ED142A90ED142AD0ED0E2A9FEDBB3A12EE832A61EE812A62EE222A90ED072A9FEDB73A03EE622A3E
:40C1400080ED072A90ED142AD0ED1A2A9FEDB13A02EEC32AF6EE002A62EE222A90ED1A2A9FEDAD3A03EE222A80ED1A2A7047AB4800687047AA480068704770B52DED028B9F
:40C18000A84800681DF0DFFC05469FEDA70A10EE104A38F121F8A3490860FFF7E8FF962807DAB2EE048AA14890ED020A80ED070A1FE09E4890ED060AB0EEC00ADFED9C0AE3
:40C1C000B4EEE00AF1EE10FA11D2FFF7D3FF00EE100AB8EEC00AB0EEC00ADFED960AB4EEE00AF1EE10FA02D2B7EE008A01E09FED8E8A91480068D0ED000A8F4890F904006A
:40C2000000EE100AB8EEC00A20EE800A8A4880ED020A90ED020AD0ED040A20EE200AD0ED030A864890ED061A00EE810A8248D0ED050A7E4890ED061A00EE810A7E48D0ED74
:40C24000070A30EE600A10EE104A20468BF136FD08B979488461784890ED0F0A006A90ED001A754890F9240000EE900AF8EEE00A11EE200A704880ED0A0AD0ED0A0AB0EE67
:40C28000600A3CF09BFBDFED640A20EE200A6A48D0ED0C0A20EE200AD0ED0B0A674890ED0E1A00EE810A6448D0ED0D0A5F4890ED0E1A00EE810AFFF75AFF00EE900AF8EE82
:40C2C000E00A5A4890ED061A60EE810A9FED5C1AC0EE811A30EE210A10EE104A20468BF1EDFC08B954488463B0EE480A29465248FFF78AFE51480068D0ED000A4F4890F9E2
:40C30000040000EE100AB8EEC00A20EE800A4B4880ED020A90ED020AD0ED030A20EE200AD0ED040A444890ED061A00EE810A4348D0ED050A3D4890ED061A00EE810A3E486D
:40C34000D0ED070A30EE600A10EE104A20468BF1B5FC08B939488461384890ED0F0A006A90ED001A354890F9240000EE900AF8EEE00A11EE200A314880ED0A0AD0ED0A0AC8
:40C38000B0EE600A3CF01AFBDFED230A20EE200A2A48D0ED0B0A20EE200AD0ED0C0A264890ED0E1A00EE810A2448D0ED0D0A1F4890ED0E1A00EE810A10EE104A20468BF129
:40C3C0007DFC08B91D488463B0EE480A29461B48FFF71AFE15480068D0ED000A134890F9040000EE100AB8EEC00A20EE800A0F4880ED020A90ED020AD0ED050A20EE200A06
:40C40000D0ED030A0D4890ED061A00EE810A19E000007A4439FA8E3CE12E65422C000010300000103C0000100000000018070020E12EE54100009643AC0600204006002010
:40C4400000481946FE48D0ED040AFE4890ED061A00EE810AFA48D0ED070A30EE600A10EE104A20468BF12AFC08B9F5488461F448D0ED0F0A006A90ED001AF14890F92400D4
:40C4800000EE100AB8EEC00A51EE000AEC48C0ED0A0AD0ED0A0AB0EE600A3CF08FFA5FED220A20EE200AE648D0ED0D0A20EE200AD0ED0B0AE44890ED0E1A00EE810AE0480A
:40C4C000D0ED0C0ADF4890ED0E1A00EE810A10EE104A20468BF1F2FB08B9D9488463BDEC028B70BD70B5044637F176FE0546D748016828461DF037FBD5490968611A4FF4F9
:40C500007A725143B1FBF0F0D2490860D048046037F162FECD4908600521CF4800688BF129FE90BBCD48016828461DF01CFBB0F57A7F01D9C9480560C848016828461DF065
:40C5400012FB60434FF47A71B0FBF1F0C44AD2E90032C01842F10001C14A03C200BFC048D0E90021BF48C0E90221082200F10801BD4834F145F900BFB84805600920FEF738
:40C5800068FCB54800683CF0A7FB70BD70B504460025B6488078A04204D0B44884700720FEF757FC284670BD70B504460025AF48007BA04204D0AD4804730820FEF749FCF3
:40C5C000284670BDA948807870472DE9F04F8BB0A7488468A7488768A748D0F80890A748D0F80880A24840680A90A24840680990A14840680890A148406807909C48007B22
:40C6000006909C48007B05909B48007B04909B4890F80CB080780390FE20029007200190002000900398082828D2DFE800F00E041824252727264FF6FF20804504D84746BF
:40C6400007980990CDF814B018E04FF6FF20804504D8444607980A90CDF818B00EE04FF6FF20804506D8C14607980890CDF810B00120009002E000BF00BF00BF00BF4FF620
:40C68000FF20814525D8009810B9B9F5807F06D8009801281DD140F21510814519D94D46009880B900EE105AB8EE400ADFED740A20EE200ABCEEC00A10EE105AB5F57B4F70
:40C6C00001D34FF6FF25089E04980290022001904CE04FF6FF20844208D8874206D925460A9E06980290002001903FE04FF6FF20874208D8844206D93D46099E059802907A
:40C700000120019032E04FF6FF20874205D9844203D900250720019028E000EE104AB8EE400ADFED580A20EE200ABCEEC00A10EE10AA34B925460A9E0698029000200190F8
:40C7400014E0A4EB0A00B8420AD204EB0A00B84206D93D46099E059802900120019005E025460A9E0698029000200190FFF72AFF0199884203D13D484068B0420AD00298B6
:40C78000FFF712FF0198FFF701FF384846602846FFF7A8FE0BB0BDE8F08F10B504463A480078844204D0384804700520FEF751FB10BD0146002200200AE0344B53F820307D
:40C7C00023B9324B43F82010012203E0431CD8B20828F2DB1046704730B503460024002017E02A4D55F820508DB1284D55F820502D7B9D420BD1254D55F820502D888D4259
:40C8000005D1224D55F820501560012403E0451CE8B20828E5DB204630BD2DE9FC470546002600270020019000BF05F10C000CF0AFF90446286881692846884728E000002B
:40C8400018070020AC06002040060020440000102C000010300000103800001040000010200000102824001008750068F0050020100600200006002020060020300600205B
:40C880008AE38A3FCDCCCC3E34000010D00500201FFA80F828686946C268284690474FF6486084420AD0401C844207D04FF6E860844203D04FF22200844225D1284645F1B8
:40C8C00081FB814601AA2146FFF786FFE0B928686946C26828469047012815D1B8F1080F12DB10203CF082F80190284645F16AFB0199087301990C80F9480078401CF84964
:40C9000008700198FFF755FF0198002867D0A4F570402238002847D0A0F6266020B101281CD0A02858D12CE037F156FCED494860009800780099497840EA0120E94988609C
:40C94000284645F13FFBE74908730098C079C0F381073846FFF721FF01263FE037F13CFCE1494860009800780099497840EA0120DD498860284645F125FBDB4908730126C9
:40C980002CE037F129FCD9494860009880780099C97840EA0120D5498860284645F112FBD2490873012619E037F116FCD0494860009800780099497840EA0120CC49886085
:40C9C000284645F1FFFACA4908730098C079C0F382008870012601E0002600BF00BF012E07D1C448006A20B1C249086A01213CF097F9BDE8FC879FEDC00AC04880ED030AB9
:40CA0000B7EE000A80ED040A9FEDBB0A80ED050A9FEDB90A80ED0B0AB7EE000A80ED0C0A9FEDB50A80ED0D0A9FEDB30A80ED140A9FEDB30A80ED150A9FEDB20A80ED160AAF
:40CA4000B1EE000A80ED170AB7EE000A80ED100A9FEDA90A80ED110A9FEDA70A80ED120A9FEDA50A80ED130AB7EE000AA64880ED030A9FEDA10A80ED040A9FED9F0A80ED8C
:40CA8000050AB7EE000A80ED0B0A9FED9B0A80ED0C0A9FED990A80ED0D0A9FED970A80ED140A9FED970A80ED150A9FED960A80ED160AB1EE040A80ED170AB7EE000A80ED4E
:40CAC000100A9FED8D0A80ED110A9FED8B0A80ED120A9FED890A80ED130A9FED870A8B4880ED030A9FED840A80ED040AB7EE000A80ED050A9FED800A80ED0B0A9FED7E0A48
:40CB000080ED0C0AB7EE000A80ED0D0A70470EB501247F488BF10AFB7E49086037F15CFB05460321734880F82510FFF764FF0022AFF219314FF2220048F1AEFB0022AFF265
:40CB400025314FF6486048F1A7FB0022AFF235314FF6496048F1A0FB0022AFF241314FF6E86048F199FB00BF4FF0FF3100208BF10DFB8DE80700009840281CD0009808281B
:40CB800019D1019800F4804080B10021594880F825100020574908625E4800688BF1DEFA8BF118FB06468BF121FB04E0019800F0010000B101244B48007BFF280DD04949B7
:40CBC000486840F2DC511CF097FF30B1FF20454908734FF6FF70886001244348007BFF280DD04149486840F2DC511CF085FF30B1FF203D4908734FF6FF70886001243B4842
:40CC0000007BFF280DD03949486840F2DC511CF073FF30B1FF20354908734FF6FF70886001243348007BFF280FD03149486840F2DC511CF061FF40B1FF202D4908734FF675
:40CC4000FF708860072088700124012C06D1FFF7BCFC002437F1C0FA05460BE04FF4FA6128461CF049FF28B10020FFF73BFC37F1B3FA0546FFF781FA76E77047704770B524
:40CC800005460026062D29D2DFE805F00348709AC4EE00241FE0E0B2FFF7F0FF1B48006AD0ED000A194890F9240000EE100AB8EEC00A20EE800AF6EE000AB4EEE00AF1EE6D
:40CCC00010FA06DBE1B20022134843F1C3FB012603E0601CC4B2042CDDDB00BFEEE000003600001010060020000600202006002030060020F008002000000000AC060020AE
:40CD000017B7D13895BFD6334006002018070020B0CF040838000010381E0020002421E0211DC8B2FFF7AAFFA448006AD0ED000AA24890F9240000EE100AB8EEC00A20EE1B
:40CD4000800AF6EE000AB4EEE00AF1EE10FA07DB201DC1B200229A4843F17CFB012603E0601CC4B2042CDBDB00BFA7E0002423E004F10801C8B2FFF781FF9048006AD0ED49
:40CD8000000A8E4890F9240000EE100AB8EEC00A20EE800AF6EE000AB4EEE00AF1EE10FA08DB04F10800C1B20022854843F152FB012603E0601CC4B2042CD9DB00BF7DE0B4
:40CDC000002423E004F10C01C8B2FFF757FF7B48006AD0ED000A794890F9240000EE100AB8EEC00A20EE800AF6EE000AB4EEE00AF1EE10FA08DB04F10C00C1B2002270483E
:40CE000043F128FB012603E0601CC4B2042CD9DB00BF53E0002423E004F11001C8B2FFF72DFF6648006AD0ED000A644890F9240000EE100AB8EEC00A20EE800AF6EE000ACA
:40CE4000B4EEE00AF1EE10FA08DB04F11000C1B200225B4843F1FEFA012603E0601CC4B2042CD9DB00BF29E0002423E004F11401C8B2FFF703FF5148006AD0ED000A4F4845
:40CE800090F9240000EE100AB8EEC00A20EE800AF6EE000AB4EEE00AF1EE10FA08DB04F11400C1B20022464843F1D4FA012603E0601CC4B2042CD9DB00BF00BF00BF3046AE
:40CEC00070BD10B53E4843F1C1FA0446C01704EB9070801010BD70B500210C460D460121384800688BF146F928B9374830C8354800683BF0F1FE2046294670BD70B50446E6
:40CF00000D46072601212F4800688BF133F9B0B92D4830C000BF0838D0E900202B49C1E90220082208312A4833F16AFC00BF0026244800683BF0D0FE0920FDF78AFF3046B5
:40CF400070BD244890ED1A0A7047224890ED190A7047214890ED1A0A70471F4890ED190A70471E48007B70471D480068704770B5044600251A480068A04204D0184804608C
:40CF80000620FDF766FF284670BD1FEDA50A70470A4890ED190A704712480078704770B5044600250F480078A04204D00D4804700420FDF74EFF284670BD00001807002092
:40CFC000381E00203800001020000010282400100875006840060020AC060020F0050020280000103500001010B581F106FA04462CB104F0E6FD0020F749087002E0012028
:40D00000F5490870204610BD2DE9F0472DED028B04460027204681F113FA00F0FF08B8F1560F79DA20688168204688471B2874D2DFE800F00E1420262C327338FD43494F36
:40D04000555B736174B2C3D4FCFBFAF9F8F7F6000021404637F17AFE07464CE1B8F1510F07DBB8F1550F04DC0121404637F16EFE074640E10321404637F168FE07463AE1BD
:40D080000421404637F162FE074634E10121404637F15CFE07462EE10221404637F156FE074628E140463FF1C4FCB0F1FF3F01D0012000E0002007461DE10A21404637F16F
:40D0C00045FE074617E10921404637F13FFE074611E10B21404637F139FE07460BE10621404637F133FE074605E10721404637F12DFE0746FFE00C21404637F127FE074657
:40D1000025462068416A20468847064628683146826A28469047EEE0EEE0EBE040463FF1BAF981461021404637F110FE0746AB4800EB890090ED000AB5EEC00AF1EE10FA83
:40D140000DD02068416B20468847A44800EB8900D0ED000AB4EE600AF1EE10FA01D1012000E00020074025462068416B20468847B0EE408A2C462868816B28468847264640
:40D180002068C16A20468847B0EE408A34463068016B30468847AEE00D21404637F1D6FD074625462068416A20468847064628683146826A284690479DE00E21404637F121
:40D1C000C5FD074625462068416A20468847064628683146826A284690478CE040463FF15AF981461121404637F1B0FD07467B4800EB890090ED000AB5EEC00AF1EE10FA9F
:40D200000DD02068416B20468847744800EB8900D0ED000AB4EE600AF1EE10FA0AD107E067E065E063E061E05FE05DE01DE05AE0012000E00020074025462068416B2046CA
:40D240008847B0EE408A2C462868816B2846884726462068C16A20468847B0EE408A34463068016B3046884745E040463FF1D0FA81461221404637F169FD0746574800EB43
:40D28000890090ED000AB5EEC00AF1EE10FA0DD02068416B20468847504800EB8900D0ED000AB4EE600AF1EE10FA01D1012000E00020074025462068416B20468847B0EE4E
:40D2C000408A2C462868816B2846884726462068C16A20468847B0EE408A34463068016B3046884707E000BF00BF00BF00BF00BF00BF00BF00BF00BF3846BDEC028BBDE8C3
:40D30000F08770B50446204681F19AF8C5B20021284637F11BFD70BD002008E09FED300A2E4901EB800181ED000A411CC8B20F28F4D3704710B50446E0B23FF147FB10BD94
:40D3400010B50446E0B23FF1C4FF10BD10B50446E0B23FF16EFB10BD10B50446E0B240F1F6FA10BD70B504460D46E0B229463EF17BFD70BD10B52DED028B0446B0EE408A01
:40D38000E0B2B0EE480A3EF14BFEBDEC028B10BD10B52DED028B0446B0EE408AE0B2B0EE480A3EF1DCFFBDEC028B10BD70B504460D46E0B229463FF179F970BD10B52DED52
:40D3C000028B0446B0EE408AE0B2B0EE480A3FF180F9BDEC028B10BD50000010E01100200000000010B52DED028B0446B0EE408AE0B2B0EE480A3FF1D7F9BDEC028B10BDAC
:40D4000001480078704700005000001010B5002807DA0A07140E7B4A00F00F031B1FD45403E00A07130E784A135410BD774A0168116001791171704710B5754875490860E9
:40D440004FF4E13048604FF44071724881610C21416100210161C1608160C16187F139FE6D486E4908604FF00060486040216B4881600021C1604FF4806101610021416160
:40D480008161C1614FF40031016200214162032181624FF40001C1628910016382F16EFE00BF5E485B49086308465C49886300BF00210E20FFF7AAFF0E2000F097F80D21A9
:40D4C0002720FFF7A3FF272000F090F801225449504888F15FF810B101205249087010BD10B54E4883F1A1F810BD10B5494888F1BAFC10BD10B501224949464888F14AF85A
:40D50000044614B1012047490870204610BD10B5044645480078012826D1002007E0434909880144424A515C1154411C88B2414909883E4A1288891A8142F0DC3D48008832
:40D540003A490988401A3B49088000203749088038480088C0F1800200213548803089F16CF80020304908702D480178314802880088401C2F4B18802D488154184600887A
:40D58000802802DB00201946088000F040FB1B2805D02949886F03213BF0C2FB05E02649D1F8800002213BF0BBFB01221C49194887F1F0FF10B101201A49087010BD7047F5
:40D5C00010B504461D4800F02BF9022804DB1A49886F02213BF0A4FB10BD70B504460D462A4621460B4888F16EF870BD00F01F02012191404209920002F1E022C2F80011ED
:40D600007047000018ED00E000E400E0BC120020004800401C120020586002405C12002047000020480000205A010020560100201C16002054010020F0080020CC120020A0
:40D6400070B50446F648006820B9F6488AF16EFDF349086002F03EFE054688F115FF012060720020F04908700620F04908800020EF490870EF490870EF490870EF49087063
:40D68000EF490880EF4908800120EF4908700020EE490880EE490870EE490870EE490860401EEE4908604FF47A70ED4908800020EC490870EC48046000200DE00021EB4A8D
:40D6C0001154EB4A1154EB4A11540022E94B00F140015A54411CC8B24028EFDB1121E64888F1B3FF02F0F6FD05462B46E3A21121E1483AF0A1FA2C21E34888F1A6FF2C219E
:40D70000E24888F1A2FF206881682046884770BD10B5044620461CF015F90446DC4820602046FFF78DFFD0480460204610BD10B50446D7482060BA48006818B1B848006875
:40D740008AF10CFD20461CF003F90446204610BD70B504462046FFF7EAFF05463BF03EF970BD70B50546012407E0CA4B0022214628461CF09DF9601C84B2072CF5DB70BDA0
:40D780002DE9F04780460C464FF0010904F0E6F828B921464046FFF720FF814627E004F0DDF8012823D12646701CC7B2781CC0B2B94901EB0021781C01EB1025B7490D709A
:40D7C000280A4870280C8870280EC870084607710120487132464146B048801D88F1E8FEB01DC1B2AD48FFF7F8FE814600BF4846BDE8F08770B5054600249648007868B9B6
:40D8000093480078012809D1A54801789848FFF7B7FF18B901208F4908700124204670BD0146487A704770B505460C462846FFF7F7FFA04213D06C7200231A460421284611
:40D840001CF036F9012C08D100221146954843F1E0FA00207849087000E000BF00BF70BD70B58AB004460D46164601202B4622460146CDE9006002A80BF0DAFC02A848F112
:40D8800036FB02A80BF08CFD0AB070BD70B58AB004460D46164601202B4622460146CDE9006002A80BF0C4FC02A848F120FB02A80BF076FD0AB070BD30B50246002391B17F
:40D8C0008AB16348007870B9002004E0145C684D2C54441CE0B28842F8DB7148017001205B4C20700123184630BD10B502460B460020002100BF04E0545C0444E0B24C1C44
:40D90000E1B29942F8DB10BD2DE9F043A1B081460D4616461C464FF00008002E3CD0082C3ADC802101A83AF061FB04F10C0777208DF8040088208DF8050099208DF806002E
:40D94000F8B28DF80700FF208DF80800280E8DF80900280C8DF80A00280A8DF80B00E8B28DF80C00224631460DF10D0088F120FEFF21F81E01AA1154401C1154781EC1B2C0
:40D9800001A8FFF7B2FF791E01AA5054F9B201A8FFF792FF804600BF404621B0BDE8F0832548007870472DE9F041A0B005460C464FF0FF38802168463AF018FB0026002743
:40D9C000002D71D0002C6FD0206800286CD020683F2869D221782846FFF787FF216868542068401C20607E2238467F1C0DF8002000BF60E0A85D7E2805D0A85D7D2802D033
:40DA0000A85D7C2851D17C2238467F1C0DF80020A85DC043C2B238467F1C0DF8002049E05001002034D10408620100206601002063010020610100206401002065010020BF
:40DA400054010020560100205A0100205801002068010020690100206C01002070010020740100207601002078010020EE1600209C1600201C1600202E1700205548502016
:40DA8000534E2575000000003F1700206B17002044D31908078804082000FF00D415002060010020381E002015E0AA5D38467F1C0DF80020761C2068B0429BD87D2238464B
:40DAC0007F1C0DF80020276069462846226888F16FFD4FF00008404620B0BDE8F0812DE9F043A1B081460D4616461C46DDF8A080002744B3802101A83AF078FAFE48007877
:40DB00008DF804008DF805508DF80660424621460DF1070088F14CFD08F103000090694601A8FFF740FF002805DB0098C1B201A8FFF7C2FE0746012F04D1EF480078401CF9
:40DB4000ED49087000BF384621B0BDE8F0832DE9F041A2B004460026206821A9C2682046904700284FD000BF00BFE06820F0004000BF0546802101A83AF038FAFFF710FFFD
:40DB800001282FD1280E8DF80400280C8DF80500280A8DF80600E8B28DF80700206881692046884707463A4602A8219988F100FD2068816920468847001DC7B2062141F0F9
:40DBC000200000BF00BF00BF00BF00BF00BF804601AB00224146C94800970068FFF77FFF06460FE0FFF7DCFE60B92068816920468847C7B23B462946C048219A0068FFF797
:40DC000083FE064600BF304622B0BDE8F081BC480078704770B504460025B948007884420BD0B7480470B548006830B100232A460121B24800681BF03BFF284670BD70B544
:40DC400004460D460226122D14DC9CB1002004E0215CAC4A1154411CC8B2A842F8DB0020A849487400231A460621A44800681BF01FFF0026304670BD10B5024600230020E6
:40DC8000087010609F481060002008E09D4C245C1CB1012311240C7003E0441CE0B21228F4DB184610BD98480088704770B504460025FF2C01DD022508E0934804800023BC
:40DCC0002A4602218D4800681BF0F2FE284670BD8E480078704710B504468C48047000231A460321854800681BF0E2FE10BD0020704787490870704786490860704785483D
:40DD000000687047844870478449086070478348006870478249086070478148006870478049088070477F48008870477E49087070477D480078704710B504462046FFF736
:40DD40006FFD032805D1794843F15FF808B1012010BD0020FCE72DE9F04781460C4615461E462F784FF0000804F47000B0F5700F04D24FF47F4000EA142801E0C4F30F28D4
:40DD80004FF6C170804507D1202F05D1684B0022182168481BF08CFE324629462046FFF75FFDBDE8F0872DE9FE4F05460C464FF0FF300290002600274FF0000B4FF000083F
:40DDC000002001900090002D3CD0002C3AD04FF07D094FF0800A5246494620463AF07FF88046B8F1000F2DD0A8EB040000F1010B01270FE0E05D7C2807D17F1CE05DC043FD
:40DE0000C2B23046761C2A5403E0E25D3046761C2A547F1CABF10100B842EBD80020A855701E285C0190701EC1B22846FFF75DFD00900021701E2954DDE90010884201D19E
:40DE4000002002900298BDE8FE8F2DE9F04190B005460E469046402168463AF0C7F8002400276EB331466846FFF79DFF002827DB9DF801409DF80270204600F0800119B95D
:40DE800000BF04F0200040B128680DF103033A462146D0F818C02846E04700BF012020EAD41068B100BF012020EA941040B128680DF103033A462146D0F81CC02846E047D4
:40DEC00010B0BDE8F0812DE9F0470546002619E119481A490988445C19480088402802DB002017490880174815490988445413480088401C114927E06501002078010020C4
:40DF000062010020DC1600206601002063010020640100205C0100202E1700206C010020700100207401002076010020381E002007880408CC1200201C16002056010020B8
:40DF400058010020EE160020088008460088802801DB00200880FD4800680B282AD8FC48FA490968405CA04207D0F848006804281DD9F6480068092819D2F648F3490968D4
:40DF80004454F2480068401CF0490860084600680B280FD34021F04888F157FBEB480068421EEC49EC4888F103FB012602E00020E6490860FFF72BFE1B2801D1012E12D11A
:40DFC0000A2C0AD11720FFF725FE4021E24888F13CFB0020E149088094E0E0480088401CDE4908808EE0FFF7DBFC01281BD1DA4800787E2803D00020D849088004E0D74855
:40E000000088401CD54908807D2C7BD10120D4490870D2480278D0492846FFF716FF0020CE4908806EE0CC480078772803D00020CA49088066E0CB480068C8B9C7480088E6
:40E04000032815D1C448007877280ED1C248407888280AD1C0488078992806D1BE48BF490988405CBF49086002E00020BB490880BC480068401EB949098888423DD1B6483C
:40E0800040790006B449897940EA0140B249C97940EA0120B049097A40EA01074FF00008AD48C0780C3800F0FF09AE480068401EA94911F800A001F10908AA480078401E2F
:40E0C000C1B2A548FFF711FC504509D14B46424639462846FFF73FFE0120A149087002E09D4890F813A040219B4888F1AEFA00209A4908809B49086004E098480088401CAC
:40E1000096490880984800889849098888427FF4DFAEBDE8F087002008E09549095C01B906E00021924A1154411CC8B28028F4DB00208D4908808D4908807047002004E086
:40E1400000218C4A1154411CC8B24028F8DB0020894908708949087089490870704701468648007870472DE9FC5F05460F4614464FF001080020019005B901AD1FB1002177
:40E18000781E295401E000202870FFF740FD1D287ED2DFE800F00F1D2A5363D9D88C9CD7D6D5D4D3D2D1D0CFCECDCCCBCAC9C8C7C6C5C4000021892002F01BF9714842F185
:40E1C00024FE10B10120FFF725FD4FF00008B4E30121892002F00DF96B48006880476B4908600220FFF716FDA7E341F28831674800681BF081FC28B1FFF77CF9644833F110
:40E200008FFD1AE063A1284689F125FD20B963A1284689F120FD80B103F0A0FB012802D1FFF759FD02E00020FFF755FD0320FFF7F1FCFFF770FF4FF000087EE3594888F1EA
:40E2400098F9C6B231465748FFF79AFA18B90420FFF7E0FC01E04FF000086EE3402C07D10020FFF7D7FCFFF756FF4FF000081DE04DA1284689F1EFFC0646B6B105F17F0010
:40E28000864212D2B07D0A280FD1B146112100E04DE309F10400FFF7D2FC0720FFF7BAFCFFF739FF4FF0000800BF00BF45E33F4888F15FF9C6B231463C48FFF761FA18B99D
:40E2C0000820FFF7A7FC01E04FF0000835E3402C07D10020FFF79EFCFFF71DFF4FF000081CE033A1284689F1B6FC0646AEB105F17F00864211D296F82B000A280DD1B146DB
:40E300002C2249462C4888F153F90920FFF782FCFFF701FF4FF0000800BF00BF0DE305E3EAE2CFE2C3E299E288E264E222E28BE168E150E11EE106E1D9E0C1E0B0E055E05B
:40E340007BE06AE03AE000E2A2E100007C01002038D1040897170020EE160020580100205A0100208001002054010020560100201C1600209C160020600100206801002026
:40E3800069010020381E0020AC03002084010020CC12002052454144590D0A00424F4F540D0A0000CC0000204D414300F000002043464750000000003F170020F44BF5A2DB
:40E3C0001221F64839F038FCF4480A3888F1D1F8C6B23146F1480A38FFF7D2F918B90C20FFF718FC01E04FF00008A6E2402C07D10020FFF70FFCFFF78EFE4FF000080BE094
:40E40000E7A1284689F127FC30B10A20FFF702FCFFF781FE4FF000088FE2E34888F1A9F8C6B23146E048FFF7ABF918B90B20FFF7F1FB01E04FF000087FE2402C07D100205C
:40E44000FFF7E8FBFFF767FE4FF0000827E0AFF2A001284689F1FFFB0646FEB105F17F0086421BD296F82B000A2817D1B1462C224946CE4888F19CF82C22CD49CB4888F117
:40E4800033F818B10D20FFF7C5FB02E00F20FFF7C1FBFFF740FE4FF0000800BF00BF4CE2C44888F166F8C6B23146C248FFF768F918B90E20FFF7AEFB01E04FF000083CE284
:40E4C000402C07D10020FFF7A5FBFFF724FE4FF000080BE0B8A1284689F1BDFB30B10020FFF798FBFFF717FE4FF0000825E2B4480278B4A1B54887F117FFB4480078B44935
:40E500008872B2484078C872AD480088C0F30722ACA1AE4887F108FFAC480078AC490873AA4840784873084688F123F8C6B23146A748FFF725F918B91020FFF76BFB01E087
:40E540004FF00008F9E1402C07D10020FFF762FBFFF7E1FD4FF000080BE091A1284689F17AFB30B11120FFF755FBFFF7D4FD4FF00008E2E197A000680090FFF794FBC6B2D9
:40E58000324690A1684687F1CFFE9DF80000924988729DF80100C872FFF785FB060A324688A1684687F1C0FE9DF800008A4908739DF801004873084687F1DBFFC6B23146B7
:40E5C0008548FFF7DDF818B91220FFF723FB01E04FF00008B1E1402C07D10020FFF71AFBFFF799FD4FF000080BE06DA1284689F132FB30B11320FFF70DFBFFF78CFD4FF092
:40E6000000089AE173A000680090FFF761FB064632466CA1684687F187FE9DF800006F4988729DF80100C872084687F1A2FFC6B231466A48FFF7A4F818B91420FFF7EAFAEE
:40E6400001E04FF0000878E1402C05D10020FFF7E1FA4FF000081AE051A1284689F1FBFA30B10520FFF7D6FAFFF755FD4FF000085BA1284689F1EFFA48B10020FFF72BFB79
:40E680000520FFF7C7FAFFF746FD4FF0000854E10026B146B246FFF706FB1E280DDDFFF717FB012807D11E20FFF700FBFFF7FBFA00F01F0605E01F2603E0FFF7F4FA00F074
:40E6C0001F06FFF705FB00F0010046EA4016FFF70EFB00F0030046EA80163EA000680090324638A1684687F11FFE9DF800003E4988729DF80100C8724A4632A1684687F1F7
:40E7000013FE9DF80000384908739DF80100487352462CA1684687F107FE9DF80000324988739DF80100C873084687F122FF00F0FF0B59462C48FFF723F818B90620FFF788
:40E7400069FA01E04FF00008F7E0402C05D10020FFF760FA4FF000080BE011A1284689F17AFA30B11720FFF755FAFFF7D4FC4FF00008E2E01D4887F1FCFEC6B231461B48F0
:40E78000FEF7FEFF18B91620FFF744FA32E02FE02E17002025730D0A00000000DC0000204F4B0D0A00000000F00000206B1700203F1700204901002053415645440D0A002E
:40E7C0008801002025303278000000008C010020F9000020303000000A0100201B010020455252340D0A00002A0100203D0100204FF00008A1E0402C05D10020FFF70AFAE3
:40E800004FF0000819E0AFF26801284689F123FA38B11720FFF7FEF9FFF77DFC4FF000080BE048A1284689F116FA30B11720FFF7F1F9FFF770FC4FF000087EE0434887F1F8
:40E8400098FEC6B231464148FEF79AFF18B91820FFF7E0F901E04FF000086EE0402C05D10020FFF7D7F94FF000081FE038A1284689F1F1F928B11720FFF7CCF94FF0000883
:40E8800014E030A1284689F1E6F928B11520FFF7C1F94FF0000809E02FA1284689F1DBF920B11920FFF7B6F9FFF735FC45E0402C07D02BA1284689F1CEF910B11A20FFF7A8
:40E8C000A9F93AE0402C02D14FF0000813E026A1284689F1C0F970B11B20FFF79BF90321234833F149FDFFF716FC2248006880470646FFF701FA20E0402C0CD11E48007897
:40E90000012812D100201C490870194833F108FA4FF0000809E019A1284689F19CF920B1134833F1FDF94FF0000806E000BF0020FFF770F94FF0000800BF00BF4046BDE83F
:40E94000FC9F0000455252320D0A000043010020455252310D0A00004144560D0A00000052494E4720000000444154410D0A0000CC120020AC030020610100204449534350
:40E980000000000000210181418181814160704700B502467448754810601046FFF7F2FF104600BD10B5044620463FF10BFB0446204610BD70B504462046FFF7F3FF054632
:40E9C0003AF00CF870BD3EB505460020029000243220012301AA2A2100903820FDF7D2F99DF8040000F0010070B12A208DF808009DF8040020F001008DF809003223022262
:40EA000002A93820FDF798F96423022258493820FDF792F96423022256493820FDF78CF96423022254493820FDF786F96423022252493820FDF780F9FDF7D7F96420012386
:40EA400002AA0D2100903820FDF79CF99DF808001A281CD13220012301AA2A2100903820FDF790F99DF8040000F0010070B92A208DF808009DF8040040F001008DF80900CC
:40EA80003223022202A93820FDF756F9012420463EBD7FB504460025002001900290FDF7A4F90120034603AA002100903820FDF769F9B8BB9DF80C0000F0080090B3FDF7E1
:40EAC0009DF90120062301AA014600903820FDF759F938BB9DF805009DF8041040EA012000B220819DF807009DF8061040EA012000B260819DF809009DF8081040EA012087
:40EB000000B2A081B4F9080080102081B4F90A0080106081B4F90C008010A08135F15CFB60600125284604B070BD0146B1F9080070470146B1F90A0070470146B1F90C0079
:40EB40007047014648687047014601F108007047014601F10A007047014601F10C0070470146081D70470000C8CE1908E8D519088F010020910100209301002095010020BE
:40EB800010B5002807DA0A07140EFE4A00F00F031B1FD45403E00A07130EFB4A135410BD70B504460D460026082C0BDA0120A040C6B23146B32002F03BFE0021B42002F044
:40EBC00037FE27E0082C09D110260021B32002F02FFE3146B42002F02BFE1BE0092C09D120260021B32002F023FE3146B42002F01FFE0FE00F2C05DAA4F10A0084B201206C
:40EC0000A040C6B20021B32002F012FE3146B42002F00EFE2946B12002F00AFE70BD10B5044601EE102AF8EE411A01EE103AB8EE411A81EE812AB0EE420AB7EE001AB4EEBE
:40EC4000C10AF1EE10FA04DDB7EE001AB0EE410A08E0B5EEC00AF1EE10FA03D29FEDCB1AB0EE410AB7EE001A71EE401A01EE101AB8EE411A61EE811A01EE104AB8EE411A24
:40EC8000F0EE610A41EE000ABCEEE01A11EE100A10BD10B5044604F00F040121692001F0A8FB04F00101412001F0A3FBC4F34001392001F09EFBC4F38001602001F099FBF5
:40ECC000E108692001F095FB10BD7FB506460C4615460720029000200390019400956946304680F1C6FA7FBDF8B504460D46164600BF00200090A648006840F48000A449F3
:40ED000008600846006800F48000009000BF2560002060600021A160012121610021A16121626162E162A162E160E661216301216161984885421ED19748A06384639748EA
:40ED40009549086000204860002193488160C1602915016189004161890081610021C1614FF40031016200214162012181620021C162016346E08A48854220D18948A06342
:40ED8000846386483030874908604FF000704860002184488160C1602915016189004161890081610021C1614FF40031016200214162012181620021C162016322E07A483B
:40EDC00085421FD17948A063846374481830774908604FF080604860002174488160C1602915016189004161890081610021C1614FF40031016200214162012181620021A5
:40EE0000C162016320467FF110FEA06B81F1B6F9A06B00686149884207D100213820FFF7AFFE382000F09CFD1AE0A06B00685B493031884207D100213A20FFF7A1FE3A2001
:40EE400000F08EFD0CE0A06B006854491831884206D100213920FFF793FE392000F080FDF8BD8CB04FF00208002700250321504880F85D104F480021016041608160C16087
:40EE8000062244494C48FFF72FFF052244494B48FFF72AFF082244494948FFF725FF00210846FFF77DFE44480068406840F02000414909684860082201213F48FFF705FFE1
:40EEC000032202213C48FFF700FF0F2203213A48FFF7FBFE092204213748FFF7F6FE112205213548FFF7F1FE122206213248FFF7ECFE0A2201213148FFF7E7FE0B22022170
:40EF00002E48FFF7E2FE0C2203212C48FFF7DDFE0D2204212948FFF7D8FE0E2205212748FFF7D3FE002201212548FFF7CEFE012202212348FFF7C9FE022203212048FFF74A
:40EF4000C4FE062204211E48FFF7BFFE072205211B48FFF7BAFE092206211948FFF7B5FE0E2207211648FFF7B0FE0F2208211448FFF7ABFE1348006820F480000549C1F8A0
:40EF8000040321E018ED00E000E400E0000000003038024000200140701B00201064024000210140D01B002000220140301C0020F0080020601B0020901C0020D81C002065
:40EFC000201D00200423014000BF0021084689F1DDF809AB07C3099808280FD10A9800F4804058B10021F84880F85D100020F649886589F1EFF8044689F1F8F80026FDE394
:40F000003046FFF746FE062039F012FE01F0DDFA022807D1ED48008802F07EFB80F00100EB498855EB480068806840F00100E94909688860062201A9E64880F139F88146A5
:40F0400041F28831012089F1A1F809AB07C3099808287DD1B9F1000FFBD1DF48006880470446DE48C0F8F840C0F8FC40DC490598C1F8F8000698C1F8FC00DA490598C1F865
:40F08000F8000698C1F8FC00102E1ED2DFE806F0081E344A61778DA3B9F1F0EFEEEDECEBCE4804600464C0F88040CD4901980860029808640398C1F88000CA4901980860D4
:40F0C000029808640398C1F88000B0E2C34844604464C0F88440C24901984860029848640398C1F88400BF4901984860029848640398C1F884009AE2B84884608464C0F800
:40F100008840B74901988860029888640398C1F88800B44901988860029888640398C1F8880084E2AD48C460C464C0F88C40AC490198C8600298C8640398C1F88C00A949CB
:40F140000198C8600298C8640398C1F88C006EE26FE2A24804610465C0F89040A04901980861029808650398C1F890009D4901980861029808650398C1F8900057E2974886
:40F1800044614465C0F89440954901984861029848650398C1F89400924901984861029848650398C1F8940041E28C4884618465C0F898408A49019888610298886503980E
:40F1C000C1F89800874901988861029888650398C1F898002BE28148C461C465C0F89C407F490198C8610298C8650398C1F89C007C490198C8610298C8650398C1F89C00C2
:40F2000015E2764804620466C0F8A04044203EF1E2FB30B150203EF1DEFB40B10020019005E050203EF1D7FB08B9002001903A203EF1D1FB30B145203EF1CDFB40B10020DB
:40F24000029005E045203EF1C6FB08B90020029039203EF1C0FB68B138203EF1BCFB78B1002003900CE017E100E1E9E0D2E0BBE060E016E038203EF1AEFB08B90020039024
:40F28000574901980862029808660398C1F8A000544901980862029808660398C1F8A000C5E14E4844624466C0F8A44036203EF192FB30B137203EF18EFB40B10020019047
:40F2C00005E037203EF187FB08B90020019032203EF181FB30B133203EF17DFB40B10020029005E033203EF176FB08B9002002902E203EF170FB30B12F203EF16CFB40B14A
:40F300000020039005E02F203EF165FB08B900200390334901984862029848660398C1F8A400304901984862029848660398C1F8A4007CE1294884628466C0F8A840352055
:40F340003EF149FB30B134203EF145FB40B10020019005E034203EF13EFB08B90020019031203EF138FB30B130203EF134FB40B10020029005E030203EF12DFB08B900206F
:40F38000029017203EF127FB30B118203EF123FB40B10020039005E018203EF11CFB08B9002003900E4901988862029888660398C1F8A8000B4901988862029888660398FA
:40F3C000C1F8A80033E10000F0080020AC000010601B0020901C00205CCC19082C1A0020C4170020F8180020FD48C462C466C0F8AC40FC490198C8620298C8660398C1F826
:40F40000AC00F9490198C8620298C8660398C1F8AC000CE1F24804630467C0F8B040F14901980863029808670398C1F8B000EE4901980863029808670398C1F8B000F6E049
:40F44000E74844634467C0F8B440E64901984863029848670398C1F8B400E34901984863029848670398C1F8B400E0E0DC4884638467C0F8B840DB49019888630298886743
:40F480000398C1F8B800D84901988863029888670398C1F8B800CAE0D148C463C467C0F8BC40D0490198C8630298C8670398C1F8BC00CD490198C8630298C8670398C1F890
:40F4C000BC00B8F10E0F13D2DFE808F007131F2B37434F5B67737F8B97A3C148C0F8C040C0490498C1F8C000BF490498C1F8C0009BE0BB48C0F8C440BA490498C1F8C400EE
:40F50000B9490498C1F8C4008FE0B548C0F8C840B4490498C1F8C800B3490498C1F8C80083E0AF48C0F8CC40AE490498C1F8CC00AD490498C1F8CC0077E0A948C0F8D040F4
:40F54000A8490498C1F8D000A7490498C1F8D0006BE0A348C0F8D440A2490498C1F8D400A1490498C1F8D4005FE09D48C0F8D8409C490498C1F8D8009B490498C1F8D80020
:40F5800053E09748C0F8DC4096490498C1F8DC0095490498C1F8DC0047E09148C0F8E04090490498C1F8E0008F490498C1F8E0003BE08B48C0F8E4408A490498C1F8E4007D
:40F5C00089490498C1F8E4002FE08548C0F8E84084490498C1F8E80083490498C1F8E80023E07F48C0F8EC407E490498C1F8EC007D490498C1F8EC0017E07948C0F8F040D4
:40F6000078490498C1F8F00077490498C1F8F0000BE07348C0F8F44072490498C1F8F40071490498C1F8F40000BF00BF00BF00BF00BF6E487FF1E3FD6C487FF1C2FA6C48D1
:40F640000068806840F00100694909688860052201A967487FF12CFD814641F28831012088F194FD09AB07C30998082867D1B9F1000F64D138460DF04AFE04465D48006878
:40F68000804707465648C0F80071C0F80471C0F80871C0F80C71C0F8107152490198C1F800010298C1F804010398C1F808010498C1F80C010598C1F810014B4AD2F80011C7
:40F6C000484A0C23D2F800012246FFF7A8FA4649C1F800010A46D2F80411424A0C23D2F804012246FFF79BFA3F49C1F804010A46D2F808113B4A0C23D2F808012246FFF72B
:40F700008EFA3949C1F808010A46D2F80C11354A0C23D2F80C012246FFF781FA3249C1F80C010A46D2F810112E4A0C23D2F810012246FFF774FA2C49C1F8100100BF2C482C
:40F740007FF15DFD2A487FF13CFA2B480068806840F00100284909688860082201A926487FF1A6FC814641F28831012088F10EFD09AB07C3099808287ED1B9F1000F7BD19A
:40F7800028460DF0C4FD04461A480068804705461348C0F81451C0F81851C0F81C51C0F82051C0F82451C0F82851C0F82C51C0F830510C490198C1F814010298C1F818011C
:40F7C0000398C1F81C010498C1F820010598C1F824010698C1F828010798C1F82C010EE02C1A0020C4170020F8180020901C0020D81C00205CCC1908201D002074E00898A9
:40F80000C1F830015C4AD2F814115C4A0C23D2F814012246FFF703FA5749C1F814010A46D2F81811554A0C23D2F818012246FFF7F6F95149C1F818010A46D2F81C114F4A3F
:40F840000C23D2F81C012246FFF7E9F94A49C1F81C010A46D2F82011484A0C23D2F820012246FFF7DCF94449C1F820010A46D2F82411424A0C2300E02FE0D2F824012246E8
:40F88000FFF7CDF93C49C1F824010A46D2F828113A4A0C23D2F828012246FFF7C0F93649C1F828010A46D2F82C11344A0C23D2F82C012246FFF7B3F92F49C1F82C010A4605
:40F8C000D2F830112D4A0C23D2F830012246FFF7A6F92949C1F8300100BF29487FF18FFC27487FF16EF9761C102EFFF489AB08F101001FFA80F8B8F10D0F01DD4FF0020824
:40F9000000214046FFF74CF9FFF75FBB10B504461C4890F85D00032804D11A49886D012139F0FEF910BD10B51749886B80F17DFE10BD10B51549886B80F177FE10BD10B5B7
:40F940000F49886B80F171FE10BD10B50E487FF1A9FA0E487FF1A6FA09487FF1A3FA10BD00F01F02012191404209920002F1E022C2F8001170470000F8180020C41700204D
:40F98000201D0020F0080020901C0020D81C00202DE9F04106460C4615460027002E61D0B4F1D04F0ED36019401E8149884209D8A4F1D0412A46304634F120FB002851D125
:40F9C00001274FE07B4884420ED36019401E7A49884209D87748211A2A46304634F133F800283FD101273DE0744884420ED36019401E72493F31884208D87048211A2A46E2
:40FA0000304634F125F968BB01272BE0B4F1805F0BD36019401E6A49884206D82A462146304686F1C5FD01271CE0B4F1005F0BD36019401E6349884206D82A46214630461F
:40FA400086F1B6FD01270DE0B4F1006F0AD36019401EB0F1026F05D22A462146304686F1A7FD01273846BDE8F0812DE9F04106460C4615460027002E51D0B4F1D04F0ED317
:40FA80006019401E4A49884209D8A4F1D0412A46304634F111FA002841D101273FE0454884420DD36019401E4349884208D84148211A2A46304633F198FF08BB01272EE056
:40FAC0003E4884420ED36019401E3C493F31884208D83A48211A2A46304634F167F878B901271CE0B4F1805F0BD36019401E3449884206D82A463146204686F159FD012747
:40FB00000DE0B4F1005F0AD36019401E2D49884205D82A463146204686F14AFD01273846BDE8F08170B504460D460026002D3CD0B4F1D04F0CD36019401E1D49884207D892
:40FB4000A4F1D040294634F1B5FA00BB01262CE0184884420ED36019401E1749884209D8144AA21A5119134AA01A33F17DFE70B901261AE0B4F1805F0AD36019401E1049B1
:40FB8000884205D82946204686F15FFD01260CE0B4F1005F09D36019401E0A49884204D82946204686F151FD0126304670BD0000FF7F006800010168FF00016900000168AD
:40FBC000FFFF0010FFFF0220FD4800787047FC4908707047FB4800787047FA4908707047F94800787047F8490870704710B500221146DC2001F05EFE00221146DB2001F03F
:40FC000059FE00221146DE2001F054FE00221146DD2001F04FFE00221146E02001F04AFE00221146DF2001F045FE00221146E22001F040FE00221146E12001F03BFE002231
:40FC40001146E42001F036FE00221146E32001F031FE00221146E62001F02CFE00221146E52001F027FE00221146E82001F022FE00221146E72001F01DFE00221146EA2099
:40FC800001F018FE00221146E92001F013FE00221146EC2001F00EFE00221146EB2001F009FE00221146ED2001F004FE00221146EE2001F0FFFD00221146EF2001F0FAFD5E
:40FCC00000221146F02001F0F5FD00221146F12001F0F0FD00221146F22001F0EBFD00221146F32001F0E6FD00221146F42001F0E1FD00221146F52001F0DCFD002211463F
:40FD0000F62001F0D7FD00221146F72001F0D2FD00221146F82001F0CDFD00221146F92001F0C8FD00221146FA2001F0C3FD0022114640F2131001F0BDFD002211464FF48B
:40FD40008A7001F0B7FD0022114640F2151001F0B1FD002211464FF48B7001F0ABFD0022114640F2171001F0A5FD002211464FF48C7001F09FFD0022114640F2191001F0B6
:40FD800099FD002211464FF48D7001F093FD10BD10B5022200218D2001F08CFD022200218E2001F087FD022200218F2001F082FD02220021902001F07DFD02220021912053
:40FDC00001F078FD02220021922001F073FD02220021932001F06EFD02220021942001F069FD02220021952001F064FD02220021962001F05FFD02220021972001F05AFDC9
:40FE000002220021982001F055FD02220021992001F050FD022200219A2001F04BFD022200219B2001F046FD022200219C2001F041FD022200219D2001F03CFD0222002139
:40FE40009E2001F037FD022200219F2001F032FD02220021A02001F02DFD02220021A12001F028FD02220021A22001F023FD02220021A32001F01EFD02220021A42001F019
:40FE800019FD02220021A52001F014FD02220021A62001F00FFD02220021A72001F00AFD02220021A82001F005FD02220021A92001F000FD02220021AA2001F0FBFC0022FF
:40FEC0001146AC2001F0F6FC00221146AD2001F0F1FC00221146AE2001F0ECFC00221146AF2001F0E7FC00221146B02001F0E2FC00220121D72001F0DDFC00220121D82043
:40FF000001F0D8FC00220121D92001F0D3FC00221146DA2001F0CEFC00221146B12001F0C9FC00221146B22001F0C4FC01220021B32001F0BFFC00221146B42001F0BAFC1E
:40FF400000221146CC2001F0B5FC00221146D12001F0B0FC00221146CD2001F0ABFC00221146CE2001F0A6FC00221146CF2001F0A1FC00221146D02001F09CFC002211461A
:40FF8000D22001F097FC00221146D32001F092FC00221146D42001F08DFC00221146D52001F088FC00F011FB02280FD1FFF70CFE044622460021E62001F07CFC0EE00000E0
:40FFC000970100209801002099010020FFF7FCFD044622460021B52001F06CFCFFF7FAFD044622460021B62001F064FCFFF7F8FD044622460021B72001F05CFC00220121DD
:020000040801F1
:40000000D62001F057FC00221146B82001F052FC00221146B92001F04DFC00221146BA2001F048FC00221146BB2001F043FC00221146BC2001F03EFC00221146BD2001F097
:4000400039FC00221146BE2001F034FC00221146BF2001F02FFC00221146C02001F02AFC00221146C12001F025FC00221146C22001F020FC00221146C32001F01BFC002295
:400080001146C42001F016FC00221146C52001F011FC00221146C62001F00CFC00221146C72001F007FC932119203CF177F893211A203CF173F893211B203CF16FF89321B4
:4000C0001C203CF16BF8932146203CF167F8932147203CF163F8932148203CF15FF8932149203CF15BF8FD2119203CF1C5F8FD211A203CF1C1F8FD211B203CF1BDF8FD21D6
:400100001C203CF1B9F8FD2146203CF1B5F8FD2147203CF1B1F8FD2148203CF1ADF8FD2149203CF1A9F89FED610A19203BF1FAFE9FED5E0A1A203BF1F5FE9FED5C0A1B2071
:400140003BF1F0FE9FED590A1C203BF1EBFE9FED570A46203BF1E6FE9FED540A47203BF1E1FE9FED520A48203BF1DCFE9FED4F0A49203BF1D7FEFFF739FD10BD2DE9F04F73
:4001800089B04FF0200B4FF00A0A0321484880F8551001214748008800F02BF9022038F047FD00214348008800F023F9022038F03FFD01213F48008800F01BF90A2038F090
:4001C00037FD00F002FA10B93B4F3C4D01E03C4F3C4D20244FF0000915E009EB0400A84202D9A5EB0900C4B22246394601A87CF169FA00B909E02744214601A833F1ABFC79
:4002000000B102E0A144A945E7D32F48008801F083FA80462D48008801F07EFA0646B8F1000F17D0012E15D14FF00B0A022038F0FFFC01212648008800F0DBF8022038F047
:40024000F7FC00212248008800F0D3F8322038F0EFFC10E0B8F1010F03D116B94FF00D0A09E0B8F1000F04D1012E02D14FF00C0A01E04FF00E0ABAF10B0F09D1FFF788FD97
:400280003521C02001F0D4FA3521C42001F0D0FA074880F855A000200549086587F19AFF814687F1A3FF09B0BDE8F08F00000000F0080020A800001000010D6816E90400A5
:4002C0000001016830E40800A6000010AA000010A4000010F0B5FD4A0024204621460FE00A2600230446A4FB067C01FB06C500FB0351384612F8013B303B181841EBE371D5
:400300001378302B02DB1378392BE9DDF0BDF04800787047EE49087070470020EB4950310978412909DBE949503109785A2904DCE649503109784139C8B27047F0B5E34AE2
:4003400060320024204621460FE00A2600230446A4FB067C01FB06C500FB0351384612F8013B303B181841EBE3711378302B02DB1378392BE9DDF0BD0020D4492031097824
:40038000412909DBD149203109785A2904DCCF49203109784139C8B27047F0B5CB4A30320024204621460FE00A2600230446A4FB067C01FB06C500FB0351384612F8013B77
:4003C000303B181841EBE3711378302B02DB1378392BE9DDF0BD01464FF6FF70012905DB8C2903DCBB4A02EBC1029088704701207047F8B504460E460127B4F58D7F50DC74
:40040000B548005D082808D2DFE800F0040508090B0A240600BF00BF00BF41E000BF00BF00BF012E0AD1AB4A02EBC4029188A94A52F83400012280F12EFC09E0A54A02EBEE
:40044000C4029188A34A52F83400002280F123FC002725E0A4F18D0085B205EB45009F490844407806FA00F0C0B2009005EB45000844807850B105EB4500084481780120D3
:4004800088409DF800100843C0B2009005EB4500924A115C0122684633F188FB074600BF00BF3846F8BD2DE9F04786B004460D4616461F46DDE90E894FF0010A012C6EDB90
:4004C0008C2C7EDC834850F83400002879D04FF0000A804800EBC40080880190029503960497CDF814807E49681A8D422DD00DDC032D55D005DCDDB1012D32D0022D59D16A
:400500003EE0112D2ED0122D54D13AE0B0F5881F19D006DCB0F5803F14D0B0F5801F49D114E0B0F5001F12D0B0F5041F42D10BE0022069490855674951F8340001A980F14D
:4005400007FA3DE000BF00BF00BF00BF00BF0320614908555F4951F8340001A980F1F8F92EE000BF05205C4908555A4951F8340001A980F1EDF949462046FFF73AFF1FE00F
:4005800000BF042054490855524951F8340001A980F1DEF949462046FFF72BFF10E010E001204D4908554B4951F8340001A980F1CFF905E00020484908554FF0010A00BF5B
:4005C00000BF504606B0BDE8F08710B545480078032834D10A2244A13C48303037F089FC30B10A2243A13948303037F082FC18B900203C49087022E00A2241A133483030E9
:4006000037F077FCA0B10A2240A13048303037F070FC68B10A2240A12C48303037F069FC30B10A223FA12948303037F062FC18B902202C49087002E001202A49087029484F
:40064000007810BD1CB5FFF7C0FF02283DD13220374908803320374908803420364908803520364908808A20354908808B20354908808C20344908804D20344908804E2019
:40068000334908804F2033490880742032490880012000210B460246CDE9001001463220FFF701FF012000210B460246CDE9001001463320FFF7F7FE012000210B460246FB
:4006C000CDE900100146342048E0CEE0786F0008AE000010F8D204089C2600104CD1040800001110AF00001030363430313731333332000030363430313731343636000067
:400700003036343031373135303100003036343031373135303600003036343031373135323500003036343031373135323600007C0000107E000010800000108200001087
:4007400084000010860000108800001076000010780000107A000010AC000010FFF7A3FE012000210B460246CDE9001001463520FFF799FE0020052102230246CDE9001089
:4007800019464D20FFF78FFE0020052102230246CDE9001019464E20FFF785FE0020052102230246CDE9001019464F20FFF77BFE0020009003460222012101905220FFF73D
:4007C00072FE0020009003460222012101905320FFF769FE0020009003460222012101906120FFF760FE0020009003460222012101906220FFF757FE002000900346024666
:40080000014601907420FFF74EFE0020009003460246012101907F20FFF745FE0020009003460246012101908020FFF73CFE012000210B460246CDE9001001468A20FFF7F2
:4008400032FE012000210B460246CDE9001001468B20FFF728FE012000210B460246CDE9001001468C20FFF71EFE1CBD002003E00021FE4A1154401CB0F58D7FF8D97047B4
:400880001FB50520FA4908806420FA4908804220F94908800620F94908800720F84908800820F84908803120F74908808220F74908801F20F64908808420F64908801B20F9
:4008C000F54908801C20F54908801920F44908801A20F44908801620F34908801E20F34908802B20F24908802C20F24908803C20F14908803D20F14908805120F0490880AB
:400900006D20F04908805B20EF4908805F20EF4908806520EE4908806320EE4908804420ED490880FFF7A2FFFFF761FD002800F0F28683F1C9FF044684F142F9B4FBF0F007
:40094000012809D984F13CF94000E449B0FBF1F0401E80B2039007E084F132F9DF49B0FBF1F0401E80B2039083F1AEFF044684F133F9B4FBF0F0012809D984F12DF94000C7
:40098000D649B0FBF1F0401E80B2029007E084F123F9D249B0FBF1F0401E80B2029000BF00200190CE48006840F00100CC4908600846006800F00100019000BF00BF0020B7
:4009C00001900846006840F0020008600846006800F00200019000BF00BF002001900846006840F0040008600846006800F00400019000BF00BF002001900846006840F00C
:400A0000080008600846006800F00800019000BF00BF002001900846006840F0100008600846006800F01000019000BF00BF002001900846006840F02000086008460068E0
:400A400000F02000019000BF00BF002001900846006840F0400008600846006800F04000019000BF00BF002001900846006840F0800008600846006800F08000019000BF2E
:400A800000BF002001900846006840F4807008600846006800F48070019000BF00BF002001900846006840F4001008600846006800F40010019000BF00BF00200190084600
:400AC000006840F4800008600846006800F48000019000BF00BF0020019081481430006840F001007E49143108600846006800F00100019000BF00BF00200190081F006878
:400B000040F00200091F08600846006800F00200019000BF00BF002001900846006840F0040008600846006800F00400019000BF00BF002001900846006840F00800086079
:400B40000846006800F00800019000BF00BF002001900846006840F0100008600846006800F01000019000BF00BF00200190081D006840F00200091D08600846006800F040
:400B80000200019000BF00BF002001900846006840F4803008600846006800F48030019000BF00BF002001900846006840F4003008600846006800F40030019000BF00BFEC
:400BC000002001900846006840F4802008600846006800F48020019000BF00BF00200190081F006840F04000091F08600846006800F04000019000BF00BF002001900846C5
:400C0000006840F4802008600846006800F48020019000BF00BF002001900846006840F4804008600846006800F48040019000BF00BF002001900846006840F480000860F8
:400C40000846006800F48000019000BF00BF002001900846006840F0007008600846006800F00070019000BF00BF3BE09C26001062000010640000106600001068000010E6
:400C80006A0000106C0000106E0000107000001072000010740000108A0000108C0000108E00001090000010920000109400001096000010980000109A0000109C000010DC
:400CC0009E000010A0000010A2000010A4000010A6000010A8000010AA00001040420F0030380240002001900846006840F0806008600846006800F08060019000BF00BF59
:400D000000200190081D006840F40050091D08600846006800F40050019000BF00BF002001900846006840F4807008600846006800F48070019000BF00BF002001900846BF
:400D4000006840F4007008600846006800F40070019000BF00BF002001900846006840F4806008600846006800F48060019000BF00BF002001900846006840F0100008604B
:400D80000846006800F01000019000BF00BF002001900846006840F4805008600846006800F48050019000BFFE4902988862FE4903980860FD4903980860FD49039808602A
:400DC000FC4902980860FC4902988862FB4902980860FB4902980860FA49039808600020009003460246014601900120FFF75BFB0020009003460246014601900220FFF75A
:400E000052FB0020009003460246014601900320FFF749FB0020009003460246032101900420FFF740FB0020009003460246012101900520FFF737FB00200521034602468C
:400E4000CDE9001002210620FFF72DFB0020052103460246CDE9001002210720FFF723FB0020052103460246CDE9001002210820FFF719FB00200090034602460121019064
:400E80000920FFF710FB0020009003460246012101900A20FFF707FB0020009003460246012101900B20FFF7FEFA0020009003460246012101900C20FFF7F5FA0020009030
:400EC00003460246012101900D20FFF7ECFA0020009003460246032101901120FFF7E3FA002100910B460A46019103211220FFF7DAFA002100910B460A4601910121162069
:400F0000FFF7D1FA0020009003460246012101901720FFF7C8FA002100910B460A46019101211820FFF7BFFA002100910B460A46019101211920FFF7B6FA012100200346AE
:400F40000246CDE900011A20FFF7ADFA0021042002230A46CDE9000112211B20FFF7A3FA0021042002230A46CDE9000112211C20FFF799FA002100910B460A4601910121B9
:400F80001D20FFF790FA0121002003460246CDE900011E20FFF787FA0020052103460246CDE9001002211F20FFF77DFA002100910B460A46019101212020FFF774FA0020FE
:400FC000009003460246014601902120FFF76BFA002100910B460A4622200191FFF763FA002100910B460A4623200191FFF75BFA0020009003460246014601902420FFF71C
:4010000052FA002100910B460A4625200191FFF74AFA002100910B460A46019103212620FFF741FA0020009003460246012101902720FFF738FA002100910B460A46019138
:4010400001212820FFF72FFA0020009003460246012101902920FFF726FA002100910B460A46019101212A20FFF71DFA002107200B460A46CDE9000102212B20FFF713FA25
:40108000002107200B460A46CDE9000102212C20FFF709FA002100910B460A462D200191FFF701FA002100910B460A462E200191FFF7F9F9002000900346024601460190D1
:4010C0002F20FFF7F0F9002100910B460A4630200191FFF7E8F9012000210B460A46CDE9001001463120FFF7DEF9002100910B46022232200191FFF7D6F9002100910B46D5
:40110000022233200191FFF7CEF90020009003460222014601903420FFF7C5F9002100910B46022235200191FFF7BDF9002100910B46022236200191FFF7B5F900200090CF
:4011400003460222014601903720FFF7ACF9002100910B46022238200191FFF7A4F90020009003460246012101903920FFF79BF9002100910B460A463A200191FFF793F9FC
:40118000002100910B460A46019101213B20FFF78AF9002107200B460A46CDE9000102213C2011E0000001402804004028080040280C004028040140004001402844014018
:4011C0002848014028180040FFF76DF9002100910B460A46019102213D20FFF764F9002100910B460A463E200191FFF75CF90020009003460246012101903F20FFF753F987
:40120000002100910B460A46019101214020FFF74AF90020009003460246012101904120FFF741F90121002003460246CDE9000111214220FFF737F9002100910B460A46F2
:4012400043200191FFF72FF90020009003460246014601904420FFF726F90121002003460246CDE900014520FFF71DF9002100910B460A46019101214620FFF714F900203E
:40128000009003460246112101904720FFF70BF9002100910B460A4648200191FFF703F90020009003460246014601904920FFF7FAF8002100910B460A464A200191FFF7FB
:4012C000F2F8002100910B460A464B200191FFF7EAF8002100910B460A464C200191FFF7E2F8002100910B460A46019101214D20FFF7D9F8002100910B4602224E20019159
:40130000FFF7D1F80020009003460246012101904F20FFF7C8F8002100910B460A4650200191FFF7C0F80020009003460246012101905120FFF7B7F8002100910B460222A1
:4013400052200191FFF7AFF8002100910B46022253200191FFF7A7F80020009003460246014601905420FFF79EF80020009003460246014601905520FFF795F8002100912F
:401380000B460A4656200191FFF78DF80020009003460246012101905720FFF784F8002100910B460A46019101215820FFF77BF8002100910B460A4659200191FFF773F885
:4013C000002100910B460A465A200191FFF76BF80121002003460246CDE9000111215B20FFF761F8002100910B460A46019101215C20FFF758F8002100910B460A465D2016
:401400000191FFF750F8002100910B4602225E200191FFF748F80020009003460246012101905F20FFF73FF8002100910B460A46019101216020FFF736F80020009003462B
:401440000222014601906120FFF72DF8002100910B46022262200191FFF725F8002100910B460A46019111216320FFF71CF80020009003460246112101906420FFF713F859
:401480000020009003460246014601906520FFF70AF8002100910B46022266200191FFF702F80020009003460246014601906720FEF7F9FF002100910B460A46682001916D
:4014C000FEF7F1FF0020009003460246012101906920FEF7E8FF002100910B4602226A200191FEF7E0FF002100910B460A466B200191FEF7D8FF002100910B460A466C207C
:401500000191FEF7D0FF002100910B460A46019101216D20FEF7C7FF002100910B460A466E200191FEF7BFFF0020009003460246014601906F20FEF7B6FF002100910B468B
:401540000A4670200191FEF7AEFF0020009003460222014601907320FEF7A5FF002100910B46022274200191FEF79DFF002100910B46022275200191FEF795FF00200090D1
:4015800003460222014601907620FEF78CFF0020009003460246012101907720FEF783FF002100910B460A46019102217820FEF77AFF002000900346024602210190792032
:4015C000FEF771FF002100910B460A46019101217A20FEF768FF0020009003460246012101907B20FEF75FFF0020009003460246012101907C20FEF756FF002100910B46CA
:401600000A46019101217D20FEF74DFF002100910B4602227E200191FEF745FF002100910B4602227F200191FEF73DFF002100910B46022280200191FEF735FF002000907D
:4016400003460246012101908120FEF72CFF002105200B460A46CDE9000102218220FEF722FF0020009003460246012101908320FEF719FF002105200B460A46CDE90001AA
:4016800002218420FEF70FFF002100910B46022285200191FEF707FF0020009003460246012101908620FEF7FEFE0020009003460246012101908720FEF7F5FE0021009147
:4016C0000B460A46019101218820FEF7ECFE0020009003460246012101908920FEF7E3FE002100910B4602228A200191FEF7DBFE0020009003460222014601908B20FEF7D5
:40170000D2FE002100910B4602228C200191FEF7CAFEFEF797FF1FBDF8B50446002600200090B4F58D7F41DC9A48005D082807D2DFE800F0040507080A09191A00BF00BFD6
:4017400033E000BF00BF00BF934A02EBC4029188914A52F834007FF196FA012800D100E00020064621E000BFA4F18D0085B205EB45008A4A115C0122684632F169FA98B99A
:4017800005EB450085490844807868B105EB450008444178012088409DF80010084008B1012000E00020064600BF00BF3046F8BD01460020012913DB8C2911DC764A52F8BF
:4017C00031206AB1744A52F831205269724B03EBC1039B881A400AB1012200E00022104670471CB50120002102230A46CDE9001001466B480088FEF756FE00240AE0002148
:4018000067480088FEF7F5FD012165480088FEF7F0FD641C0A2CF2DB0020042102230246CDE9001012215E480088FEF73CFE1CBDF8B505460E460127B5F58D7F38DC554812
:40184000405D08280CD2DFE800F0040507080A090C0600BF00BF00BF00BF00BF00BF00BF25E0A5F18D0084B204EB44004B490844407806FA00F0C0B2009004EB44000844F6
:40188000807850B104EB440008448178012088409DF800100843C0B2009004EB44003F4A115C0122684632F181F9074600BF00BF3846F8BD2DE9F04104460D4616460127DF
:4018C0008D2C10DBB4F58D7F0DDC012D03D107203049085502E006202E49085531462046FFF7A6FF07463846BDE8F08110B52D480078022813D10A222B492C4836F0F9FA85
:4019000030B10A2228490C31284836F0F2FA18B901202449087002E00020224908702148007810BD10B522480078022813D10A221D491E4836F0DDFA30B10A221A490C31A9
:401940001A4836F0D6FA18B901201949087002E00020174908701648007810BD10B515480078022813D10A220F49104836F0C1FA30B10A220C490C310C4836F0BAFA18B9C3
:4019800001200C49087002E000200A4908700948007810BD9C260010F8D204084CD104088A000010B000001018070108A86F0008B1000010B200001010B5002807DA0A0702
:4019C000140EF94A00F00F031B1FD45403E00A07130EF64A135410BD01460620B1F5807F38D012DC102930D008DC012925D0022925D0042925D0082936D124E0202926D094
:401A0000402925D080292FD123E0B1F5805F26D009DCB1F5007F1ED0B1F5806F1DD0B1F5006F21D11AE0B1F5005F19D0B1F5804F17D0B1F5004F17D114E0062014E007204A
:401A400012E0082010E009200EE00A200CE000BF00BF00BF00BF172006E000BF00BF00BF00BF00BF282000BF00BF70470146FF20B1F5807F3BD012DC102930D008DC012993
:401A800025D0022925D0042925D008293FD124E0202926D0402926D0802938D125E0B1F5805F2CD009DCB1F5007F22D0B1F5806F21D0B1F5006F2AD11FE0B1F5005F20D04E
:401AC000B1F5804F1FD0B1F5004F20D11DE000201DE001201BE0022019E0032017E0042015E0052013E0062011E007200FE008200DE009200BE00A2009E00B2007E00C2059
:401B000005E00D2003E00E2001E00F2000BF00BF704710B5062034F086F80F210620FFF74BFF072034F07FF80F210720FFF744FF082034F078F80F210820FFF73DFF092059
:401B400034F071F80F210920FFF736FF0A2034F06AF80F210A20FFF72FFF172034F063F80F211720FFF728FF282034F05CF80F212820FFF721FF362034F055F8062136205A
:401B8000FFF71AFF002005E00021894A42F82010411CC8B21028F7DB8648006880B10020854908708348006836F018FF0020814908608248006836F011FF00207F4908608B
:401BC00010BD2DE9FC47FFF7A4FF002464E001A9204633F059FA00285CD001980068C16801988847002855D101980068816801988847092802D00A284AD100E000BF01982A
:401C00007CF11EFC00F0FF0840463AF166FE0746FEF7E1FB0646FFF729FF0546102D36DA01987CF10DFCC6B230463AF156FE644931F81510884215D101987CF101FC00F0D7
:401C4000FF0948463AF149FE8046FEF7C4FB0746FFF7C2FE064633F0D9FF5549019841F8250014E0DFF84C81534E019F307800904FF000090098FF2807D26A46414638465D
:401C800037F04AFF81460098307000BF00BF00E000BF00BF601C84B233F0F3F9A04296DC4548007800281DDD4348007836F09AFE4249086000240EE03E49096851F8240072
:401CC0007CF1BEFBC6B230463BF141FE3B4909680855601C84B2384800788442ECDB362033F094FFBDE8FC87014636480068084020B93448001D0068084008B10120704780
:401D00000020FCE77CB504462046FEF764FB06463046FFF7ABFE05463046FFF7E5FF48B10020009003460246014601902046FEF7BAFB0DE000200090034602462249019023
:401D40002046FEF7B0FB102D02DA1D4820F815407CBD10B5FFF7DDFE002405E00020184921F81400601CC4B2102CF7DB01201749C860592088623120C862052008600020B8
:401D800013490860002112480838C1600161416100200C49091D0860091F086009490C310860091F086010BD18ED00E000E400E0CC1D0020A0010020A8010020A401002097
:401DC0000C1E0020003C014000001110001000400838014070B505462846FFF747FE0446102C08DA3F4850F8240020B13D4951F824007CF1A6FA70BD10B501207EF16DFFF7
:401E000010BD10B502207EF168FF10BD10B504207EF163FF10BD10B508207EF15EFF10BD10B510207EF159FF10BD10B520207EF154FF40207EF151FF80207EF14EFF4FF430
:401E400080707EF14AFF4FF400707EF146FF10BD10B54FF480607EF140FF4FF400607EF13CFF4FF480507EF138FF4FF400507EF134FF4FF480407EF130FF4FF400407EF122
:401E80002CFF10BD70B500251748006900F0010038B300241BE01549096851F824007CF1CFFAC6B230463BF152FD054610480068005D38B9012D05D10C49096851F82400B2
:401EC0007CF13FFA0A4800680555601CC4B2094800788442DFDB0448006920F001000249086170BDCC1D002000100040A0010020A4010020A801002038B50446606800900F
:401F0000009D206880F3088800BFA84738BD10B572B66FF0040000F0FCF96FF0010000F0F8F94FF0FF3000F0F4F9042000F0F1F9052000F0EEF9062000F0EBF9072000F00A
:401F4000E8F9082000F0E5F9092000F0E2F90A2000F0DFF90B2000F0DCF90C2000F0D9F90D2000F0D6F90E2000F0D3F90F2000F0D0F9102000F0CDF9112000F0CAF912200C
:401F800000F0C7F9132000F0C4F9142000F0C1F9152000F0BEF9162000F0BBF9172000F0B8F9182000F0B5F9192000F0B2F91A2000F0AFF91B2000F0ACF91C2000F0A9F90B
:401FC0001D2000F0A6F91E2000F0A3F91F2000F0A0F9202000F09DF9212000F09AF9222000F097F9232000F094F9242000F091F9252000F08EF9262000F08BF9272000F00C
:4020000088F9282000F085F9292000F082F92A2000F07FF92B2000F07CF92C2000F079F92D2000F076F92E2000F073F92F2000F070F9302000F06DF9312000F06AF932200B
:4020400000F067F9332000F064F9342000F061F9352000F05EF9362000F05BF9372000F058F9382000F055F9392000F052F93A2000F04FF93B2000F04CF93C2000F049F92A
:402080003D2000F046F93E2000F043F9402000F040F9412000F03DF9422000F03AF9432000F037F9442000F034F9452000F031F9462000F02EF9472000F02BF9482000F0A2
:4020C00028F9492000F025F94A2000F022F94B2000F01FF94C2000F01CF94D2000F019F94E2000F016F9502000F013F9512000F010F96FF0040000F015F96FF0010000F08C
:4021000011F94FF0FF3000F00DF9042000F00AF9052000F007F9062000F004F9072000F001F9082000F0FEF8092000F0FBF80A2000F0F8F80B2000F0F5F80C2000F0F2F8AF
:402140000D2000F0EFF80E2000F0ECF80F2000F0E9F8102000F0E6F8112000F0E3F8122000F0E0F8132000F0DDF8142000F0DAF8152000F0D7F8162000F0D4F8172000F06A
:40218000D1F8182000F0CEF8192000F0CBF81A2000F0C8F81B2000F0C5F81C2000F0C2F81D2000F0BFF81E2000F0BCF81F2000F0B9F8202000F0B6F8212000F0B3F8222022
:4021C00000F0B0F8232000F0ADF8242000F0AAF8252000F0A7F8262000F0A4F8272000F0A1F8282000F09EF8292000F09BF82A2000F098F82B2000F095F82C2000F092F831
:402200002D2000F08FF82E2000F08CF82F2000F089F8302000F086F8312000F083F8322000F080F8332000F07DF8342000F07AF8352000F077F8362000F074F8382000F008
:4022400071F8392000F06EF83A2000F06BF83B2000F068F83C2000F065F83D2000F062F83E2000F05FF83F2000F05CF8402000F059F8412000F056F8422000F053F8432016
:4022800000F050F8442000F04DF8452000F04AF8462000F047F8472000F044F8482000F041F8492000F03EF84A2000F03BF84B2000F038F84C2000F035F84D2000F032F846
:4022C0004E2000F02FF8502000F02CF8512000F029F862B610BD00BF00BF00BF00BF00BFBFF34F8F00BF00BF00BF1348006800F4E06012490843001D0F49086000BF00BFEE
:4023000000BFBFF34F8F00BF00BF00BF00BF00BFFDE700F01F0201219140094A430942F82310704700F01F0201219140054A430942F82310704700000CED00E00000FA054D
:4023400080E100E080E200E02DE9F04104460025A01C02F052FF31287ED2DFE800F0193141537E8C9CBEC7FEFCFBFAF9F8F7F6F5F4F3F2F1F0EFEEEDECEBEAE9E8E7E6E532
:4023800065AEE4E3E2E1E0DFDEDDDCDBDAD9D800E01D02F032FF064604F1080002F02DFF074604F1090002F028FF804606EB460040000A30022111FB070011FB080553E2DE
:4023C000A01D02F01AFF0646E01D02F016FF074606EB460040000830022111FB070543E204F1080002F009FF064604F1090002F004FF074606EB460040000A30022111FB06
:40240000070531E204F1080002F0F7FE064604F1090002F0F2FE074606EB460040000A30022111FB07051FE204F10E0002F0E5FE064604F10F0002F0E0FE074604F11000E9
:4024400002F0DBFE804670001130062111FB0700022111FB080507E204E2201D02F0CDFE0646601D02F0C9FE07467000801D022111FB0705F8E1601D02F0BFFE0646A01DB6
:4024800002F0BBFE074606EB46004000C01D022111FB0705E8E104F10B0002F0AEFE064604F10C0002F0A9FE074606EB460040000D30022111FB0705D6E104F1080002F066
:4024C0009CFE064604F1090002F097FE074670000A30022111FB0705C6E104F10C0002F08CFE0646700000F10D05BDE104F1100002F083FE064604F11201881902F07DFEE4
:40250000074606F11300022111FB0705ACE1EAE065E1F1E056E1B2E070E16DE163E14FE142E133E153E0A8E09AE190E186E17CE172E165E155E11BE112E109E100E1F3E0C1
:40254000F0E0AEE090E086E07CE06BE061E057E04DE033E01AE009E0FFE704F1250002F04CFE0646700000F126057DE104F10A0002F043FE064604F10C0002F03EFE074679
:4025800070000D30022111FB07056DE104F10E0002F033FE804604F10F0002F02EFE08EB002086B204F11001881902F026FE074606F11100022111FB070555E104F11C00F8
:4025C00002F01BFE0646700000F11D054CE104F10A0002F012FE064604F10B0002F00DFE074670000C30022111FB07053CE104F10A0002F002FE0646700000F10B0533E177
:4026000004F10C0002F0F9FD0646700000F10D052AE104F10E0002F0F0FD0646700000F10F0521E104F10C0002F0E7FD064604F10D0002F0E2FD0746B0000E30022111FBE2
:40264000070511E104F1140002F0D7FD0646700000F1150508E104F1170002F0CEFD0646700000F11805FFE004F11A0002F0C5FD0646700000F11B05F6E02225F4E004F1F5
:402680000F0002F0BAFD064604F1100002F0B5FD074606EB460040001130022111FB0705E2E004F10C0002F0A8FD804604F10D0002F0A3FD08EB002804F10E0002F09DFDCF
:4026C00008EB004804F10F0002F097FD08EB006604F1100002F091FD074606F11100022111FB0705C0E004F10B0002F086FD0646700000F10C05B7E0201D02F07EFD074646
:40270000601D02F07AFD07EB0027A01D02F075FD07EB0047E01D02F070FD07EB006606F10805A1E007259FE0E01C02F066FD0746201D02F062FD07EB002086B2751D93E0E1
:40274000E01D02F05AFD0646700000F108058BE0E01D02F052FD0646700000F1080583E0E01D02F04AFD0646700000F108057BE0201D02F042FD0646611D881902F03DFD43
:402780000746B01D022111FB07056DE0201D02F034FD0646611D881902F02FFD0746B01D042111FB07055FE0E01C02F026FD0746201D02F022FD07EB002086B2751D53E03D
:4027C0000C2551E0201D02F018FD0746601D02F014FD07EB002086B2B000851D44E0092542E0052540E004F10C0002F006FD0646700000F10D0537E00C2535E0092533E0B9
:40280000E01C02F0FAFC0746201D02F0F6FC07EB002086B2751D27E0601D02F0EEFC064606EB46004000851D1EE0A01D02F0E5FC064606EB46004000C51D15E0601D02F00E
:40284000DCFC064606EB46004000851D0CE0601D02F0D3FC064606EB46004000851D03E0062501E0002500BF00BF2846BDE8F08170477047704770477047704770477047BE
:40288000704770477047704770477047704770477047704770B5044601260125ACB1072C09DC601E05FA00F0C5B202F030FC284058B9002609E0A4F1080005FA00F0C5B234
:4028C00002F028FC284000B90026304670BD70B50446254601E0681EC5B22846FFF7DAFF0028F8D0284670BD70B52DED028B044600259FEDF70AB0EE408A02F039FC10B140
:4029000001280AD104E002F0F1FBB0EE408A04E002F0F0FBB0EE408A00BF00BF9FEDED0AB4EEC08AF1EE10FA0BDB9FEDEB0AB4EEC08AF1EE10FA04D82046FFF7C8FF0546E4
:40294000F5E30F2C70D2DFE814F00F00BD003A01AB016802E502560304048604F704A405210692064A07C707B3EE080AB4EEC08AF1EE10FA04DB0E20FFF7A9FF0546A0E0C8
:402980009FEDD60AB4EEC08AF1EE10FA04DB0D20FFF79DFF054694E0B3EE000AB4EEC08AF1EE10FA04DB0C20FFF791FF054688E0B2EE080AB4EEC08AF1EE10FA04DB0B2024
:4029C000FFF785FF05467CE09FEDC50AB4EEC08AF1EE10FA04DB0A20FFF779FF054670E0B2EE000AB4EEC08AF1EE10FA04DB0920FFF76DFF054664E0B1EE080AB4EEC08A5F
:402A0000F1EE10FA04DB0820FFF761FF054658E09FEDB40AB4EEC08AF1EE10FA05DB0720FFF755FF05464CE0DBE3B1EE000AB4EEC08AF1EE10FA04DB0620FFF748FF05461D
:402A40003FE0B0EE080AB4EEC08AF1EE10FA04DB0520FFF73CFF054633E09FEDA30AB4EEC08AF1EE10FA04DB0420FFF730FF054627E0B0EE000AB4EEC08AF1EE10FA04DB3B
:402A80000320FFF724FF05461BE0B7EE080AB4EEC08AF1EE10FA04DB0220FFF718FF05460FE09FED920AB4EEC08AF1EE10FA04DB0120FFF70CFF054603E02046FFF707FF32
:402AC000054626E2B3EE080AB4EEC08AF1EE10FA04DB0E20FFF7FBFE05466FE0B3EE000AB4EEC08AF1EE10FA04DB0D20FFF7EFFE054663E0B2EE080AB4EEC08AF1EE10FAE1
:402B000004DB0B20FFF7E3FE054657E0B2EE000AB4EEC08AF1EE10FA04DB0A20FFF7D7FE05464BE0B1EE080AB4EEC08AF1EE10FA04DB0820FFF7CBFE05463FE0B1EE000A0A
:402B4000B4EEC08AF1EE10FA04DB0720FFF7BFFE054633E0B0EE080AB4EEC08AF1EE10FA04DB0520FFF7B3FE054627E0B0EE000AB4EEC08AF1EE10FA04DB0420FFF7A7FECC
:402B800005461BE0B7EE080AB4EEC08AF1EE10FA04DB0220FFF79BFE05460FE0B7EE000AB4EEC08AF1EE10FA04DB0120FFF78FFE054603E00020FFF78AFE054681E7B3EE52
:402BC000000AB4EEC08AF1EE10FA04DB0E20FFF77EFE054663E0B2EE080AB4EEC08AF1EE10FA04DB0C20FFF772FE054657E0B2EE000AB4EEC08AF1EE10FA04DB0B20FFF7F0
:402C000066FE05464BE0B1EE080AB4EEC08AF1EE10FA04DB0920FFF75AFE05463FE0B1EE000AB4EEC08AF1EE10FA04DB0820FFF74EFE054633E0B0EE080AB4EEC08AF1EED4
:402C400010FA04DB0620FFF742FE054627E0B0EE000AB4EEC08AF1EE10FA04DB0520FFF736FE05461BE0B7EE080AB4EEC08AF1EE10FA04DB0320FFF72AFE05460FE0B7EE41
:402C8000000AB4EEC08AF1EE10FA04DB0220FFF71EFE054603E00020FFF719FE054610E7B2EE080AB4EEC08AF1EE10FA04DB0E20FFF70DFE0546AFE09FED090AB4EEC08A8B
:402CC000F1EE10FA14DB0D20FFF701FE0546A3E000000000A4707D3FAE47813F52B8AA4152B82A4148E1AA4048E12A401F85AB3FB2EE000AB4EEC08AF1EE10FA04DB0C205F
:402D0000FFF7E5FD054687E0B1EE080AB4EEC08AF1EE10FA04DB0B20FFF7D9FD05467BE01FED100AB4EEC08AF1EE10FA04DB0A20FFF7CDFD05466FE0B1EE000AB4EEC08A14
:402D4000F1EE10FA04DB0920FFF7C1FD054663E0B0EE080AB4EEC08AF1EE10FA04DB0820FFF7B5FD054657E01FED210AB4EEC08AF1EE10FA04DB0720FFF7A9FD05464BE046
:402D8000B0EE000AB4EEC08AF1EE10FA04DB0620FFF79DFD05463FE0B7EE080AB4EEC08AF1EE10FA04DB0520FFF791FD054633E01FED320AB4EEC08AF1EE10FA04DB042005
:402DC000FFF785FD054627E0B7EE000AB4EEC08AF1EE10FA04DB0320FFF779FD05461BE0B6EE080AB4EEC08AF1EE10FA04DB0220FFF76DFD05460FE09FEDFA0AB4EEC08A2F
:402E0000F1EE10FA04DB0120FFF761FD054603E00020FFF75CFD054653E6B2EE080AB4EEC08AF1EE10FA04DB0E20FFF750FD05466FE0B2EE000AB4EEC08AF1EE10FA04DB65
:402E40000D20FFF744FD054663E0B1EE080AB4EEC08AF1EE10FA04DB0B20FFF738FD054657E0B1EE000AB4EEC08AF1EE10FA04DB0A20FFF72CFD05464BE0B0EE080AB4EEB5
:402E8000C08AF1EE10FA04DB0820FFF720FD05463FE0B0EE000AB4EEC08AF1EE10FA04DB0720FFF714FD054633E0B7EE080AB4EEC08AF1EE10FA04DB0520FFF708FD05469D
:402EC00027E0B7EE000AB4EEC08AF1EE10FA04DB0420FFF7FCFC05461BE0B6EE080AB4EEC08AF1EE10FA04DB0220FFF7F0FC05460FE0B6EE000AB4EEC08AF1EE10FA04DB06
:402F00000120FFF7E4FC054603E00020FFF7DFFC054610E2B2EE000AB4EEC08AF1EE10FA04DB0E20FFF7D3FC054663E0B1EE080AB4EEC08AF1EE10FA04DB0C20FFF7C7FC15
:402F4000054657E0B1EE000AB4EEC08AF1EE10FA04DB0B20FFF7BBFC05464BE0B0EE080AB4EEC08AF1EE10FA04DB0920FFF7AFFC05463FE0B0EE000AB4EEC08AF1EE10FA0F
:402F800004DB0820FFF7A3FC054633E0B7EE080AB4EEC08AF1EE10FA04DB0620FFF797FC054627E0B7EE000AB4EEC08AF1EE10FA04DB0520FFF78BFC05461BE0B6EE080AAA
:402FC000B4EEC08AF1EE10FA04DB0320FFF77FFC05460FE0B6EE000AB4EEC08AF1EE10FA04DB0220FFF773FC054603E00020FFF76EFC05469FE1B1EE080AB4EEC08AF1EE71
:4030000010FA04DB0E20FFF762FC0546A0E01FEDCB0AB4EEC08AF1EE10FA04DB0D20FFF756FC054694E0B1EE000AB4EEC08AF1EE10FA04DB0C20FFF74AFC054688E0B0EE7B
:40304000080AB4EEC08AF1EE10FA04DB0B20FFF73EFC05467CE01FEDDC0AB4EEC08AF1EE10FA04DB0A20FFF732FC054670E0B0EE000AB4EEC08AF1EE10FA04DB0920FFF77E
:4030800026FC054664E0B7EE080AB4EEC08AF1EE10FA04DB0820FFF71AFC054658E01FEDED0AB4EEC08AF1EE10FA04DB0720FFF70EFC05464CE0B7EE000AB4EEC08AF1EE6E
:4030C00010FA04DB0620FFF702FC054640E0B6EE080AB4EEC08AF1EE10FA04DB0520FFF7F6FB054634E09FED3F0AB4EEC08AF1EE10FA04DB0420FFF7EAFB054628E0B6EE0E
:40310000000AB4EEC08AF1EE10FA04DB0320FFF7DEFB05461CE0B5EE080AB4EEC08AF1EE10FA05DB0220FFF7D2FB054610E0F7E39FED2D0AB4EEC08AF1EE10FA04DB01209C
:40314000FFF7C5FB054603E00020FFF7C0FB0546F1E0B1EE080AB4EEC08AF1EE10FA04DB0E20FFF7B4FB054674E0B1EE000AB4EEC08AF1EE10FA04DB0D20FFF7A8FB054639
:4031800068E0B0EE080AB4EEC08AF1EE10FA04DB0B20FFF79CFB05465CE0B0EE000AB4EEC08AF1EE10FA04DB0A20FFF790FB054650E0B7EE080AB4EEC08AF1EE10FA04DB37
:4031C0000820FFF784FB054644E0B7EE000AB4EEC08AF1EE10FA09DB0720FFF778FB054638E0EBE31F852B3F7B14AE3EB6EE080AB4EEC08AF1EE10FA04DB0520FFF767FB2A
:40320000054627E0B6EE000AB4EEC08AF1EE10FA04DB0420FFF75BFB05461BE0B5EE080AB4EEC08AF1EE10FA04DB0220FFF74FFB05460FE0B5EE000AB4EEC08AF1EE10FA9D
:4032400004DB0120FFF743FB054603E00020FFF73EFB0546B3E3B1EE000AB4EEC08AF1EE10FA04DB0E20FFF732FB054663E0B0EE080AB4EEC08AF1EE10FA04DB0C20FFF7FA
:4032800026FB054657E0B0EE000AB4EEC08AF1EE10FA04DB0B20FFF71AFB05464BE0B7EE080AB4EEC08AF1EE10FA04DB0920FFF70EFB05463FE0B7EE000AB4EEC08AF1EEEC
:4032C00010FA04DB0820FFF702FB054633E0B6EE080AB4EEC08AF1EE10FA04DB0620FFF7F6FA054627E0B6EE000AB4EEC08AF1EE10FA04DB0520FFF7EAFA05461BE0B5EE5A
:40330000080AB4EEC08AF1EE10FA04DB0320FFF7DEFA05460FE0B5EE000AB4EEC08AF1EE10FA04DB0220FFF7D2FA054603E00020FFF7CDFA054642E3B0EE080AB4EEC08A40
:40334000F1EE10FA04DB0E20FFF7C1FA05469FE09FEDF70AB4EEC08AF1EE10FA04DB0D20FFF7B5FA054693E0B0EE000AB4EEC08AF1EE10FA04DB0C20FFF7A9FA054687E038
:40338000B7EE080AB4EEC08AF1EE10FA04DB0B20FFF79DFA05467BE09FEDE60AB4EEC08AF1EE10FA04DB0A20FFF791FA05466FE0B7EE000AB4EEC08AF1EE10FA04DB092043
:4033C000FFF785FA054663E0B6EE080AB4EEC08AF1EE10FA04DB0820FFF779FA054657E01FED800AB4EEC08AF1EE10FA04DB0720FFF76DFA05464BE0B6EE000AB4EEC08A6F
:40340000F1EE10FA04DB0620FFF761FA05463FE0B5EE080AB4EEC08AF1EE10FA04DB0520FFF755FA054633E01FED910AB4EEC08AF1EE10FA04DB0420FFF749FA054627E0A8
:40344000B5EE000AB4EEC08AF1EE10FA04DB0320FFF73DFA05461BE0B4EE080AB4EEC08AF1EE10FA04DB0220FFF731FA05460FE09FEDB10AB4EEC08AF1EE10FA04DB012054
:40348000FFF725FA054603E00020FFF720FA054695E2B0EE080AB4EEC08AF1EE10FA04DB0E20FFF714FA05466FE0B0EE000AB4EEC08AF1EE10FA04DB0D20FFF708FA0546DB
:4034C00063E0B7EE080AB4EEC08AF1EE10FA04DB0B20FFF7FCF9054657E0B7EE000AB4EEC08AF1EE10FA04DB0A20FFF7F0F905464BE0B6EE080AB4EEC08AF1EE10FA04DB3A
:403500000820FFF7E4F905463FE0B6EE000AB4EEC08AF1EE10FA04DB0720FFF7D8F9054633E0B5EE080AB4EEC08AF1EE10FA04DB0520FFF7CCF9054627E0B5EE000AB4EE8E
:40354000C08AF1EE10FA04DB0420FFF7C0F905461BE0B4EE080AB4EEC08AF1EE10FA04DB0220FFF7B4F905460FE0B4EE000AB4EEC08AF1EE10FA04DB0120FFF7A8F9054656
:4035800003E00020FFF7A3F9054618E2B0EE000AB4EEC08AF1EE10FA04DB0E20FFF797F9054663E0B7EE080AB4EEC08AF1EE10FA04DB0C20FFF78BF9054657E0B7EE000A51
:4035C000B4EEC08AF1EE10FA04DB0B20FFF77FF905464BE0B6EE080AB4EEC08AF1EE10FA04DB0920FFF773F905463FE0B6EE000AB4EEC08AF1EE10FA04DB0820FFF767F9C9
:40360000054633E0B5EE080AB4EEC08AF1EE10FA04DB0620FFF75BF9054627E0B5EE000AB4EEC08AF1EE10FA04DB0520FFF74FF905461BE0B4EE080AB4EEC08AF1EE10FA6E
:4036400004DB0320FFF743F905460FE0B4EE000AB4EEC08AF1EE10FA04DB0220FFF737F9054603E00020FFF732F90546A7E1B7EE080AB4EEC08AF1EE10FA04DB0E20FFF763
:4036800026F90546AAE09FED2B0AB4EEC08AF1EE10FA04DB0D20FFF71AF905469EE0B7EE000AB4EEC08AF1EE10FA04DB0C20FFF70EF9054692E0B6EE080AB4EEC08AF1EED8
:4036C00010FA04DB0B20FFF702F9054686E09FED1B0AB4EEC08AF1EE10FA04DB0A20FFF7F6F805467AE0B6EE000AB4EEC08AF1EE10FA04DB0920FFF7EAF805466EE0B5EE5D
:40370000080AB4EEC08AF1EE10FA04DB0820FFF7DEF8054662E09FED0A0AB4EEC08AF1EE10FA0FDB0720FFF7D2F8054656E0000048E12A401F85AB3F0C022B3E1F852B3FD5
:403740007B14AE3EB5EE000AB4EEC08AF1EE10FA04DB0620FFF7BBF805463FE0B4EE080AB4EEC08AF1EE10FA04DB0520FFF7AFF8054633E01FED100AB4EEC08AF1EE10FAB1
:4037800004DB0420FFF7A3F8054627E0B4EE000AB4EEC08AF1EE10FA04DB0320FFF797F805461BE09FEDFE0AB4EEC08AF1EE10FA04DB0220FFF78BF805460FE09FEDF90A29
:4037C000B4EEC08AF1EE10FA04DB0120FFF77FF8054603E00020FFF77AF80546EFE0B7EE080AB4EEC08AF1EE10FA04DB0E20FFF76EF805466FE0B7EE000AB4EEC08AF1EEAE
:4038000010FA04DB0D20FFF762F8054663E0B6EE080AB4EEC08AF1EE10FA04DB0B20FFF756F8054657E0B6EE000AB4EEC08AF1EE10FA04DB0A20FFF74AF805464BE0B5EE5C
:40384000080AB4EEC08AF1EE10FA04DB0820FFF73EF805463FE0B5EE000AB4EEC08AF1EE10FA04DB0720FFF732F8054633E0B4EE080AB4EEC08AF1EE10FA04DB0520FFF73B
:4038800026F8054627E0B4EE000AB4EEC08AF1EE10FA04DB0420FFF71AF805461BE09FEDC00AB4EEC08AF1EE10FA04DB0220FFF70EF805460FE09FEDBC0AB4EEC08AF1EE47
:4038C00010FA04DB0120FFF702F8054603E00020FEF7FDFF054672E0B7EE000AB4EEC08AF1EE10FA04DB0E20FEF7F1FF054664E0B6EE080AB4EEC08AF1EE10FA04DB0C2057
:40390000FEF7E5FF054658E0B6EE000AB4EEC08AF1EE10FA05DB0B20FEF7D9FF05464CE04EE0B5EE080AB4EEC08AF1EE10FA04DB0920FEF7CCFF05463FE0B5EE000AB4EE20
:40394000C08AF1EE10FA04DB0820FEF7C0FF054633E0B4EE080AB4EEC08AF1EE10FA04DB0620FEF7B4FF054627E0B4EE000AB4EEC08AF1EE10FA04DB0520FEF7A8FF054607
:403980001BE09FED870AB4EEC08AF1EE10FA04DB0320FEF79CFF05460FE09FED830AB4EEC08AF1EE10FA04DB0220FEF790FF054603E00020FEF78BFF054600E000BF00BF65
:4039C0002846BDEC028B70BD30B5039C994204D3CD1AA54201D2CD1A425530BD2DE9F84304460D4616461F46201D01F006FC8146FEF77AFF804633464246042128460097AF
:403A0000FFF7E2FFBDE8F88370477047704770B504460D46002615B1012D2FD111E001F065FBF0EE400A00EE104AB8EE401AB6EE000A01EE200ABCEEC00A10EE100A86B251
:403A40001CE001F057FBF7EE000AB4EEE00AF1EE10FA11D201F04EFBF0EE400A00EE104AB8EE401AB6EE000A01EE200ABCEEC00A10EE100A86B200E0264600BF00BF30464B
:403A800070BD2DE9F84304460F4690461D46E01C01F0B3FB8146201D01F0AFFB09EB002086B201F065FB814649463046FFF7AFFF0646F2B24346032138460095FFF784FF40
:403AC00032124346042138460095FFF77DFF601D01F093FB8146A01D01F08FFB09EB002086B201F045FB814649463046FFF78FFF0646F2B24346052138460095FFF764FF7C
:403B000032124346062138460095FFF75DFFBDE8F8832DE9F84304460F4690461D46E01C01F06BFB8146201D01F067FB09EB002086B201F01DFB814649463046FFF767FFBC
:403B40000646F2B24346032138460095FFF73CFF32124346042138460095FFF735FFBDE8F883704770472DE9F84304460F4690461D46E01C01F041FB8146201D01F03DFB28
:403B800009EB002086B201F0F3FA814649463046FFF73DFF0646F2B243460321384605E00000C03D9FCDAA3D0000803D0095FFF70BFF32124346042138460095FFF704FF3D
:403BC000601D01F01AFB8146A01D01F016FB09EB002086B201F0CCFA814649463046FFF716FF0646F2B24346052138460095FFF7EBFE32124346062138460095FFF7E4FE72
:403C000004F10C0001F0F9FA814604F10D0001F0F4FA09EB002086B201F0AAFA814649463046FFF7F4FE0646F2B243460C2138460095FFF7C9FE321243460D2138460095DE
:403C4000FFF7C2FEBDE8F8832DE9F84304460F4690461D46E01C01F0D0FA8146201D01F0CCFA09EB002086B201F082FA814649463046FFF7CCFE0646F2B243460321384673
:403C80000095FFF7A1FE32124346042138460095FFF79AFE601D01F0B0FA8146A01D01F0ACFA09EB002086B201F062FA814649463046FFF7ACFE0646F2B2434605213846F2
:403CC0000095FFF781FE32124346062138460095FFF77AFEBDE8F8832DE9F84304460F4690461D46E01C01F088FA8146201D01F084FA09EB002086B201F03AFA8146494653
:403D00003046FFF784FE0646F2B24346032138460095FFF759FE32124346042138460095FFF752FEBDE8F8832DE9F0412DED048B04460D461646002715B1052D5DD100E017
:403D400000BF01F0D7F9F7EE000AB4EEE00AF1EE10FA24D201F0E7F900EE100AF8EE408A01F0C8F9B0EE409A16F074FC00EE100AF8EE400AB0EE680A09EE600AF0EE000AAF
:403D8000C0EE208A01F0B6F9F0EE400A00EE104AB8EEC00AB0EE688A00EE208A17E001F0C2F900EE100AF8EE408A16F053FC00EE100AB8EE400A38EEC00AB0EE001AC0EE05
:403DC000010A00EE104AB8EEC00A30EE808A002C09DAB6EE000A38EE400ABDEEC00A10EE100A07B208E0B6EE000A38EE000ABDEEC00A10EE100A07B251E016B1012E4CD115
:403E000025E0002C11DA01F071F9F0EE400A00EE104AB8EEC01AB6EE000A11EE200ABDEEC00A10EE100A07B210E001F05FF9F0EE400A00EE104AB8EEC01AB6EE000A01EE38
:403E4000200ABDEEC00A10EE100A07B225E0002C11DA01F04FF9F0EE400A00EE104AB8EEC01AB6EE000A11EE200ABDEEC00A10EE100A07B210E001F03DF9F0EE400A00EE43
:403E8000104AB8EEC01AB6EE000A01EE200ABDEEC00A10EE100A07B200BF00BF00BF00BF3846BDEC048BBDE8F0812DE9F0412DED048B04460D461646002715B1052D5DD11D
:403EC00000E000BF01F016F9F7EE000AB4EEE00AF1EE10FA24D201F023F900EE100AF8EE408A01F007F9B0EE409A16F0B1FB00EE100AF8EE400AB0EE680A09EE600AF0EE62
:403F0000000AC0EE208A01F0F5F8F0EE400A00EE104AB8EEC00AB0EE688A00EE208A17E001F0FEF800EE100AF8EE408A16F090FB00EE100AB8EE400A38EEC00AB0EE001A72
:403F4000C0EE010A00EE104AB8EEC00A30EE808A002C09DAB6EE000A38EE400ABDEEC00A10EE100A07B208E0B6EE000A38EE000ABDEEC00A10EE100A07B251E016B1012E02
:403F80004CD125E0002C11DA01F0B0F8F0EE400A00EE104AB8EEC01AB6EE000A11EE200ABDEEC00A10EE100A07B210E001F09EF8F0EE400A00EE104AB8EEC01AB6EE000A0D
:403FC00001EE200ABDEEC00A10EE100A07B225E0002C11DA01F08EF8F0EE400A00EE104AB8EEC01AB6EE000A11EE200ABDEEC00A10EE100A07B210E001F07CF8F0EE400A45
:4040000000EE104AB8EEC01AB6EE000A01EE200ABDEEC00A10EE100A07B200BF00BF00BF00BF3846BDEC048BBDE8F0812DE9F84F0646884691461F4606F10C0001F0DDF867
:404040008246F01C01F0D9F88346301D01F0D5F80BEB002085B201F08BF8834659462846FFF7D5FC0546EAB24B46032140460097FFF7AAFC2A124B46042140460097FFF71E
:40408000A3FC701D01F0B9F88346B01D01F0B5F80BEB002085B201F06BF8834659462846FFF7B5FC0546EAB24B46052140460097FFF78AFC2A124B46062140460097FFF7A2
:4040C00083FC002457E00E2101EB8401881901F094F883460F2101EB8401881901F08DF80BEB002085B201F043F883465A46102128B2FFF7DAFE85B2EAB20E2000EB84017B
:404100004B4640460097FFF75FFC2A120F2000EB84014B4640460097FFF756FC102101EB8401881901F069F88346112101EB8401881901F062F80BEB002085B201F018F874
:4041400083465A46102128B2FFF7EEFD85B2EAB2102000EB84014B4640460097FFF734FC2A12112000EB84014B4640460097FFF72BFC601CC4B25445A5DBBDE8F88F2DE9AE
:40418000F84304460F4690461D46601D01F035F88146A01D01F031F809EB002086B200F0E7FF814649463046FFF731FC0646F2B24346052138460095FFF706FC321243462B
:4041C000062138460095FFF7FFFBE01D01F015F8814604F1080001F010F809EB002086B200F0C6FF814649463046FFF710FC0646F2B24346072138460095FFF7E5FB321240
:404200004346082138460095FFF7DEFBBDE8F8832DE9F84304460F4690461D46601D00F0ECFF8146A01D00F0E8FF09EB002086B200F09EFF814649463046FFF7E8FB064624
:40424000F2B24346052138460095FFF7BDFB32124346062138460095FFF7B6FBE01D00F0CCFF814604F1080000F0C7FF09EB002086B200F07DFF814649463046FFF7C7FB0E
:404280000646F2B24346072138460095FFF79CFB32124346082138460095FFF795FBBDE8F8832DE9F84304460F4690461D46601D00F0A3FF8146A01D00F09FFF09EB0020B0
:4042C00086B200F055FF814649463046FFF79FFB0646F2B24346052138460095FFF774FB32124346062138460095FFF76DFBE01D00F083FF814604F1080000F07EFF09EBD6
:40430000002086B200F034FF814649463046FFF77EFB0646F2B24346072138460095FFF753FB32124346082138460095FFF74CFBBDE8F8832DE9F84304460F4690461D4640
:40434000E01C00F05AFF8146201D00F056FF09EB002086B200F00CFF814649463046FFF756FB0646F2B24346032138460095FFF72BFB32124346042138460095FFF724FB6F
:40438000601D00F03AFF8146A01D00F036FF09EB002086B200F0ECFE814649463046FFF736FB0646F2B24346052138460095FFF70BFB32124346062138460095FFF704FBEB
:4043C000BDE8F8832DE9F84304460F4690461D46E01C00F012FF8146201D00F00EFF09EB002086B200F0C4FE814649463046FFF70EFB0646F2B24346032138460095FFF707
:40440000E3FA32124346042138460095FFF7DCFA601D00F0F2FE8146A01D00F0EEFE09EB002086B200F0A4FE814649463046FFF7EEFA0646F2B24346052138460095FFF7E1
:40444000C3FA32124346062138460095FFF7BCFABDE8F8832DE9F84304460F4690461D46E01C00F0CAFE8146201D00F0C6FE09EB002086B200F07CFE814649463046FFF79F
:40448000C6FA0646F2B24346032138460095FFF79BFA32124346042138460095FFF794FA601D00F0AAFE8146A01D00F0A6FE09EB002086B200F05CFE814649463046FFF7F3
:4044C000A6FA0646F2B24346052138460095FFF77BFA32124346062138460095FFF774FABDE8F8832DE9F84304460F4690461D46E01C00F082FE8146201D00F07EFE09EB7B
:40450000002086B200F034FE814649463046FFF77EFA0646F2B24346032138460095FFF753FA32124346042138460095FFF74CFA601D00F062FE8146A01D00F05EFE09EB02
:40454000002086B200F014FE814649463046FFF75EFA0646F2B24346052138460095FFF733FA32124346062138460095FFF72CFABDE8F8832DE9F84304460F4690461D4686
:40458000E01C00F03AFE8146201D00F036FE09EB002086B200F0ECFD814649463046FFF736FA0646F2B24346032138460095FFF70BFA32124346042138460095FFF704FAF4
:4045C000601D00F01AFE8146A01D00F016FE09EB002086B200F0CCFD814649463046FFF716FA0646F2B24346052138460095FFF7EBF932124346062138460095FFF7E4F971
:40460000BDE8F8832DE9F84304460F4690461D46E01C00F0F2FD8146201D00F0EEFD09EB002086B200F0A4FD814649463046FFF7EEF90646F2B24346032138460095FFF74B
:40464000C3F932124346042138460095FFF7BCF9601D00F0D2FD8146A01D00F0CEFD09EB002086B200F084FD814649463046FFF7CEF90646F2B24346052138460095FFF765
:40468000A3F932124346062138460095FFF79CF9BDE8F8832DE9F84304460F4690461D46201D00F0AAFD8146601D00F0A6FD09EB002086B200F05CFD814649463046FFF781
:4046C000A6F90646F2B24346042138460095FFF77BF932124346052138460095FFF774F9BDE8F88370472DE9FC5F0446894692461E4604F10B0000F080FD0190E01C00F010
:404700007CFD8346201D00F078FD0BEB002087B200F02EFD834659463846FFF778F90746FAB25346032148460096FFF74DF93A125346042148460096FFF746F9601D00F0F8
:404740005CFD8346A01D00F058FD0BEB002087B200F00EFD834659463846FFF758F90746FAB25346052148460096FFF72DF93A125346062148460096FFF726F900256DE0EF
:4047800005EB45010F2202EB4101081900F035FD834605EB4501102202EB4101081900F02CFD0BEB00200FFA80F800F0E1FC83465A4606214046FFF778FB804608F0FF02E4
:4047C00005EB45000F2303EB4001534648460096FFF7FAF805EB4500102202EB40015346C8F3072248460096FFF7EEF805EB4501112202EB4101081900F0FFFC834605EB0F
:404800004501122202EB4101081900F0F6FC0BEB00200FFA80F800F0ABFC83465A4606214046FFF781FA804608F0FF0205EB4500112303EB4001534648460096FFF7C4F851
:4048400005EB4500122202EB40015346C8F3072248460096FFF7B8F8681CC5B2019885428EDBBDE8FC9F2DE9F84F0546884691461E46681D00F0C1FC8246002469E004EB4F
:404880004401092202EB4101481900F0B6FC834604EB44010A2202EB4101481900F0ADFC0BEB002007B200F063FC83465A4605213846FFF7FAFA0746FAB204EB4400092397
:4048C00003EB40014B4640460096FFF77DF804EB44000A2202EB40014B46C7F3072240460096FFF771F804EB44010B2202EB4101481900F082FC834604EB44010C2202EB7E
:404900004101481900F079FC0BEB002007B200F02FFC83465A4605213846FFF705FA0746FAB204EB44000B2303EB40014B4640460096FFF749F804EB44000C2202EB400187
:404940004B46C7F3072240460096FFF73DF8601CC4B2544593DBBDE8F88F704770472DE9FC5F0446894692461E4604F1080000F044FC0190E01C00F040FC8346201D00F047
:404980003CFC0BEB002087B200F0F2FB834659463846FFF73CF80746FAB25346032148460096FFF711F83A125346042148460096FFF70AF8601D00F020FC8346A01D00F085
:4049C0001CFC0BEB002087B200F0D2FB834659463846FFF71CF80746FAB25346052148460096FEF7F1FF3A125346062148460096FEF7EAFF00256DE005EB45010C2202EB11
:404A00004101081900F0F9FB834605EB45010D2202EB4101081900F0F0FB0BEB00200FFA80F800F0A5FB83465A4603214046FFF73CFA804608F0FF0205EB45000C2303EB5F
:404A40004001534648460096FEF7BEFF05EB45000D2202EB40015346C8F3072248460096FEF7B2FF05EB45010E2202EB4101081900F0C3FB834605EB45010F2202EB4101EA
:404A8000081900F0BAFB0BEB00200FFA80F800F06FFB83465A4603214046FFF745F9804608F0FF0205EB45000E2303EB4001534648460096FEF788FF05EB45000F2202EB18
:404AC00040015346C8F3072248460096FEF77CFF681CC5B2019885428EDBBDE8FC9F2DE9F84F0546884691461E4605F1080000F084FB8246002469E004EB44010C2202EBBE
:404B00004101481900F079FB834604EB44010D2202EB4101481900F070FB0BEB002007B200F026FB83465A4602213846FFF7BDF90746FAB204EB44000C2303EB40014B46A6
:404B400040460096FEF740FF04EB44000D2202EB40014B46C7F3072240460096FEF734FF04EB44010E2202EB4101481900F045FB834604EB44010F2202EB4101481900F0CB
:404B80003CFB0BEB002007B200F0F2FA83465A4602213846FFF7C8F80746FAB204EB44000E2303EB40014B4640460096FEF70CFF04EB44000F2202EB40014B46C7F3072214
:404BC00040460096FEF700FF601CC4B2544593DBBDE8F88F2DE9F84F0546884691461E46A81D00F00AFB8246002469E004EB44010A2202EB4101481900F0FFFA834604EB4F
:404C000044010B2202EB4101481900F0F6FA0BEB002007B200F0ACFA83465A4601213846FFF743F90746FAB204EB44000A2303EB40014B4640460096FEF7C6FE04EB4400D1
:404C40000B2202EB40014B46C7F3072240460096FEF7BAFE04EB44010C2202EB4101481900F0CBFA834604EB44010D2202EB4101481900F0C2FA0BEB002007B200F078FA5C
:404C800083465A4601213846FFF74EF80746FAB204EB44000C2303EB40014B4640460096FEF792FE04EB44000D2202EB40014B46C7F3072240460096FEF786FE601CC4B268
:404CC000544593DBBDE8F88F2DE9F84F0546884691461E46E81D00F090FA8246002469E004EB44010C2202EB4101481900F085FA834604EB44010D2202EB4101481900F00F
:404D00007CFA0BEB002007B200F032FA83465A4600213846FFF7C9F80746FAB204EB44000C2303EB40014B4640460096FEF74CFE04EB44000D2202EB40014B46C7F30722D9
:404D400040460096FEF740FE04EB44010E2202EB4101481900F051FA834604EB44010F2202EB4101481900F048FA0BEB002007B200F0FEF983465A4600213846FEF7D4FF3F
:404D80000746FAB204EB44000E2303EB40014B4640460096FEF718FE04EB44000F2202EB40014B46C7F3072240460096FEF70CFE601CC4B2544593DBBDE8F88F2DE9F04122
:404DC00004460D4616461F46A01C00F016FA312875D2DFE800F01920272E3C434A585F666D757C8A91989FA6ADB4C9F3FAF0EFEEEDECEBEAE9E8E7E63551BB83E5E4E3E2F6
:404E0000E1E0C2DFD7DED0003B46324629462046FFF75AFF66E13B46324629462046FFF7D9FE5FE13B46324629462046FFF757FE58E13B46324629462046FFF790FD51E177
:404E40003B46324629462046FFF788FD4AE13B46324629462046FFF780FD43E13B46324629462046FFF7FFFC3CE13B46324629462046FFF738FC35E13B46324629462046A1
:404E8000FFF730FC2EE13B46324629462046FFF701FC27E13B46324629462046FFF7B2FB20E13B46324629462046FFF763FB19E13B46324629462046FFF714FB12E110E1B3
:404EC0003B46324629462046FFF7C4FA0AE13B46324629462046FFF775FA03E13B46324629462046FFF726FAFCE03B46324629462046FFF7D6F9F5E03B4632462946204638
:404F0000FFF786F9EEE03B46324629462046FFF736F9E7E03B46324629462046FFF786F8E0E03B46324629462046FEF7D5FED9E03B46324629462046FEF786FED2E03B46A9
:404F4000324629462046FEF70EFECBE03B46324629462046FEF706FEC4E03B46324629462046FEF7FEFDBDE03B46324629462046FEF7CFFDB6E03B46324629462046FEF78A
:404F800080FDAFE03B46324629462046FEF73EFDA8E059E051E073E06BE063E046E03EE036E097E08FE087E07FE077E06FE052E027E01FE017E00FE007E0FFE73B46324684
:404FC00029462046FEF721FD8CE03B46324629462046FEF719FD85E03B46324629462046FEF7FCFC7EE03B46324629462046FDF750FC77E03B46324629462046FDF748FC9B
:4050000070E03B46324629462046FDF740FC69E03B46324629462046FDF738FC62E03B46324629462046FDF730FC5BE03B46324629462046FDF728FC54E03B4632462946F6
:405040002046FDF720FC4DE03B46324629462046FDF718FC46E03B46324629462046FDF710FC3FE03B46324629462046FDF708FC38E03B46324629462046FDF700FC31E0F7
:405080003B46324629462046FDF7F8FB2AE03B46324629462046FDF7F0FB23E03B46324629462046FDF7E8FB1CE03B46324629462046FDF7E0FB15E03B4632462946204680
:4050C000FDF7D8FB0EE03B46324629462046FDF7D0FB07E03B46324629462046FDF7C8FB00E000BF00BFBDE8F0810000FE4890ED000A7047FC4890ED010A7047FA480089BC
:405100007047F948807A7047F748C07A7047F648007B7047F448407B7047F348807B7047F148C07B7047F048007C7047EE48807C7047ED48407C7047EB48C07C704700201E
:40514000E94991F8C310042906DAE74991F8C320283101EB0211087B704700B5FFF7EFFF00BDE148008C7047DF4890F824007047DD4890F890007047DB4981F89000704742
:40518000D94890F8C2007047D74890F8EA007047D54981F8EA007047D34890F8E8007047D14981F8E8007047CF4890F8E9007047CD4981F8E9007047CB4890F88E0070478B
:4051C00000B50021FFF7F8FF2D2800D10121084600BDC6484078C5490978884201D1012070470020FCE701460020BF4AD27C8A4202DB032900DC0120704770B504460025F2
:40520000B94890F88D00072846D2DFE800F046040C161E2B3800B44991F8B800214615F054F905463AE0B04AB2F8B41092F8B900224615F063F9054630E0AB4991F8BA000B
:40524000214615F09AF9054628E00420FFF7CBFF0646A54991F8BB002246314615F090F905461BE00520FFF7BEFF06469E4991F8BB002246314615F086F905460EE00620B6
:40528000FFF7B1FF0646984991F8BB002246314615F07CF9054601E000BF00BF00BF284670BD2DE9F05F8146884692469B460025BBF1010F04D100208D4908608D49086075
:4052C0008C480068A9EB0000504504D289480068A9EB000400E05446002607E0854909688819FFF78AFF08F80600761CA642F5D333E07F480068FDF727F807467C480068A6
:405300007C490968884217D2601B83B279480068DFF8DCC1DCF800C0A0EB0C0208EB050173480068FFF74AFD7248006870490968401A381A054409E0601B83B208EB0501DE
:4053400000226B480068FFF739FD3D44A54204D267480068384466490860A542C9D3654800682044634908602046BDE8F09F2DE9F04705460C4616460027B8465A4890F89D
:405380008D00072840D2DFE800F040040B141B273300554991F8B80015F0FBF8804635E0514AB2F8B41092F8B90015F008F980462CE04D4991F8BA0015F039F9804625E0DF
:4053C0000420FFF710FF8146474991F8BB00494615F030F9804619E00520FFF704FF8146414991F8BB00494615F027F980460DE00620FFF7F8FE81463B4991F8BB00494623
:4054000015F01EF9804601E000BF00BF00BF012D09D111202070721E0123611C4046FFF740FF471C06E00023324621464046FFF738FF07463846BDE8F0872DE9F041044641
:405440000D4616461F464FF00008052C15D2DFE804F0080903040A0000BF234880F88F400BE000BF00BF204880F88F403A4631462846FFF77CFF804600BF00BF4046BDE80E
:40548000F081002019490978491C184A527891427BD0164949783131144A127891427CD001204FF467421149097801EB81030F49091D21F823209222091F097801EB810341
:4054C0000A49091D01EB83018A72FF220749097801EB81030549091D01EB8301CA720349097801EB810307E0583C0010483D00108C02002090020020F94901EB83010A7359
:40550000F749091F097801EB8103F54901EB83014A73F349091F097801EB8103F04901EB83018A73EE49091F097801EB8103EC4901EB8301CA73EA49091F097801EB81032E
:40554000E74901EB83010A74E549091F097801EB8103E34901EB83014A740822E049091F097801EB8103DE4901EB83010A81DC49091F0978491C322908DBD949091F497862
:4055800019B10021D64A121F117006E0D449091F0978491CD24A121F1170704730B502460020CF4B1B1F1B785B1CCD4C241F6478A3427DD0CA4B1B1F5B783133C84C241FA6
:4055C0002478A34274D001204FF46744C44B1B1F1B7803EB8305C24B23F82540A0241B1F1B7803EB8305BE4B03EB85039C72BC4B1B1F1B7803EB8305B94B03EB8503DA7254
:405600001412B74B1B1F1B7803EB8305B44B03EB85031C73B24B1B1F1B7803EB8304B04B03EB84035973FF24AD4B1B1F1B7803EB8305AB4B03EB85039C73A94B1B1F1B78E6
:4056400003EB8305A64B03EB8503DC73A44B1B1F1B7803EB8305A24B03EB85031C74A04B1B1F1B7803EB83059D4B03EB85035C7408249B4B1B1F1B7803EB8305984B03EB57
:4056800085031C81964B1B1F1B785B1C322B08DB934B1B1F5B781BB10023914C241F237006E08F4B1B1F1B785B1C8D4C241F237030BD30B502460020894B1B1F1B785B1CCE
:4056C000874C241F6478A3427DD0854B1B1F5B783133834C241F2478A34274D001204FF467447F4B1B1F1B7803EB83057C4B23F82540A1241B1F1B7803EB8305784B03EB52
:4057000085039C72764B1B1F1B7803EB8305744B03EB8503DA721412714B1B1F1B7803EB83056F4B03EB85031C736D4B1B1F1B7803EB83046A4B03EB84035973FF24684BA4
:405740001B1F1B7803EB8305654B03EB85039C73634B1B1F1B7803EB8305614B03EB8503DC735F4B1B1F1B7803EB83055C4B03EB85031C745A4B1B1F1B7803EB8305584B2A
:4057800003EB85035C740824554B1B1F1B7803EB8305534B03EB85031C81514B1B1F1B785B1C322B08DB4E4B1B1F5B781BB100234B4C241F237006E0494B1B1F1B785B1C03
:4057C000474C241F237030BD30B502460020444B1B1F1B785B1C424C241F6478A3427DD03F4B1B1F5B7831333D4C241F2478A34274D001204FF46744394B1B1F1B7803EB7A
:405800008305374B23F82540A2241B1F1B7803EB8305334B03EB85039C72314B1B1F1B7803EB83052E4B03EB8503DA7214122C4B1B1F1B7803EB8305294B03EB85031C7380
:40584000274B1B1F1B7803EB8304254B03EB84035973FF24224B1B1F1B7803EB8305204B03EB85039C731E4B1B1F1B7803EB83051B4B03EB8503DC73194B1B1F1B7803EB0A
:405880008305174B03EB85031C74154B1B1F1B7803EB8305124B03EB85035C740824104B1B1F1B7803EB83050D4B03EB85031C810B4B1B1F1B785B1C322B08DB084B1B1F16
:4058C0005B781BB10023064C241F237006E0044B1B1F1B785B1C024C241F237030BD00004C3D0010F0B504460020FE4D2D786D1CFC4E7678B54278D0FA4D6D783135F94EC3
:405900003678B54271D001204FF46746F54D2D7805EB8507F34D2D1D25F82760A3262D1F2D7805EB8507EF4D2D1D05EB8705AE72EC4D2D7805EB8506EA4D2D1D05EB860532
:40594000EC72E84D2D7805EB8507E64D2D1D05EB870529730E12E34D2D7805EB8507E14D2D1D05EB87056E73DE4D2D7805EB8507DC4D2D1D05EB8705AA731612D94D2D784D
:4059800005EB8507D74D2D1D05EB8705EE73D54D2D7805EB8507D34D2D1D05EB87052B741E12D04D2D7805EB8507CE4D2D1D05EB87056E740826CB4D2D7805EB8507C94DAA
:4059C0002D1D05EB87052E81C64D2D786D1C322D06DBC44D6D7815B10025C24E357004E0C04D2D786D1CBF4E3570F0BD10B501460020BC4A1278521CBA4B5B789A4276D079
:405A0000B84A52783132B74B1B789A426FD001204FF46743B34A127802EB8204B14A121D22F82430A423121F127802EB8204AD4A121D02EB84029372AA4A127802EB820364
:405A4000A84A121D02EB8302D172FF23A54A127802EB8204A34A121D02EB84021373A14A127802EB82049F4A121D02EB840253739C4A127802EB82049A4A121D02EB84028B
:405A80009373984A127802EB8204964A121D02EB8402D373934A127802EB8204914A121D02EB840213748F4A127802EB82048D4A121D02EB8402537408238A4A127802EBCF
:405AC0008204884A121D02EB84021381854A1278521C322A06DB834A527812B10022814B1A7004E07F4A1278521C7E4B1A7010BD2DE9F04704460D4616461F46DDF820805D
:405B00004FF0000977480078401C7649497888427ED0744840783130724909788842F7D0B0B24146FDF773FF46B2B8B24146FDF76EFF47B24FF001094FF467416948007861
:405B400000EB80026748001D20F82210A521001F007800EB80026348001D00EB820081726048007800EB80025E48001D00EB8200C47221125B48007800EB80025948001D44
:405B800000EB820001735748007800EB80025548001D00EB8200457329125248007800EB80025048001D00EB8200817306F17F00C1B24C48007800EB80024A48001D00EBD5
:405BC0008200C17307F17F00C1B24648007800EB80024448001D00EB82000174FF214148007800EB80023F48001D00EB8200417408213C48007800EB80023A48001D00EB97
:405C00008200018137480078401C322808DB00E00BE03448407840B100203249087004E030480078401C2F4908704846BDE8F0872DE9F04706460F4614461D46DDE9088901
:405C40004FF0000A27480078401C2649497888427ED0244840783130224909788842F7D04A4641462046FEF720F904464A4641462846FEF759F805464FF0010A4FF467412E
:405C80001848007800EB80021648001D20F82210B421001F007800EB80021248001D00EB820081720F48007800EB80020D48001D00EB8200C67231120A48007800EB80025D
:405CC0000848001D00EB820001730648007800EB80020448001D00EB8200477339120148007801E0483D001000EB8002FE4800EB82008173FC48001F007800EB8002FA4873
:405D000000EB8200C473210AF748001F007800EB8002F54800EB82000174F348001F007800EB8002F04800EB82004574290AEE48001F007800EB8002EB4800EB8200817493
:405D40000921E948001F007800EB8002E64800E018E000EB82000181E348001F0078401C322808DBE048001F407858B10020DE49091F087006E0DC48001F0078401CDA4965
:405D8000091F08705046BDE8F0872DE9F04106460C4615461F464FF00008D348001F0078401CD149091F497888427DD0CE48001F40783130CC49091F0978884274D03946E4
:405DC0002046FDF724FE044639462846FDF71FFE05464FF001084FF46741C348001F007800EB8002C04820F82210A621001F007800EB8002BC4800EB82008172BA48001FB0
:405E0000007800EB8002B84800EB8200C6723112B548001F007800EB8002B34800EB82000173B148001F007800EB8002AE4800EB820044732112AC48001F007800EB800276
:405E4000A94800EB82008173A748001F007800EB8002A54800EB8200C5732912A248001F007800EB8002A04800EB82000174FF219D48001F007800EB80029B4800EB8200FF
:405E8000417408219848001F007800EB8002964800EB820001819448001F0078401C32280ADB9148001F00E00DE0407858B100208D49091F087006E08B48001F0078401C7D
:405EC0008949091F08704046BDE8F08130B502460020854B1B1F1B785B1C834C241F6478A3427DD0804B1B1F5B7831337E4C241F2478A34274D001204FF467447A4B1B1FF7
:405F00001B7803EB8305784B23F82540A7241B1F1B7803EB8305744B03EB85039C72724B1B1F1B7803EB83056F4B03EB8503DA7214126D4B1B1F1B7803EB83056A4B03EB84
:405F400085031C73684B1B1F1B7803EB8304664B03EB84035973FF24634B1B1F1B7803EB8305614B03EB85039C735F4B1B1F1B7803EB83055C4B03EB8503DC735A4B1B1FA6
:405F80001B7803EB8305584B03EB85031C74564B1B1F1B7803EB8305534B03EB85035C740824514B1B1F1B7803EB83054E4B03EB85031C814C4B1B1F1B785B1C322B08DB95
:405FC000494B1B1F5B781BB10023474C241F237006E0454B1B1F1B785B1C434C241F237030BD30B5024600203F4B1B1F1B785B1C3D4C241F6478A34278D03B4B1B1F5B7819
:406000003133394C241F2478A34278D001204FF46744354B1B1F1B7803EB8305324B23F82540A8241B1F1B7803EB83052E4B03EB85039C722C4B1B1F1B7803EB83052A4B61
:4060400003EB8503DA721412274B1B1F1B7803EB8305254B03EB85031C73FF24224B1B1F1B7803EB8305204B03EB85035C731E4B1B1F1B7803EB83051B4B03EB85039973F7
:406080000C0A194B1B1F1B7803EB8305164B03EB8503DC730C0C144B1B1F1B7803EB8305114B03EB85031C740C0E0F4B1B1F1B7803EB83050C4B03EB85035C7408240A4B0C
:4060C0001B1F1B7803EB8305074B03EB85031C81054B1B1F1B785B1C322B0BDB024B1B1F5B781BB1002302E04C3D001007E0FE4C237004E0FC4B1B785B1CFB4C237030BD9D
:406100002DE9F04706460C4615461F46DDF820804FF00009F4480078401CF349497888427DD0F14840783130EF49097888427CD041462046FDF76BFC044641462846FDF737
:4061400066FC05464FF001094FF46741E648007800EB8002E448001D20F82210A921001F007800EB8002E048001D00EB82008172DD48007800EB8002DB48001D00EB82006E
:40618000C6723112D848007800EB8002D648001D00EB82000173D448007800EB8002D248001D00EB820044732112CF48007800EB8002CD48001D00EB82008173CA4800789B
:4061C00000EB8002C848001D00EB8200C5732912C548007800EB8002C348001D00EB82000174C148007800EB8001BF48001D00EB810047740821BC48007800EB8002BA48DD
:40620000001D00EB82000181B7480078401C322806DBB548407810B10020B349087004E0B1480078401CB04908704846BDE8F087F0B50446059D0020AB4E3678761CAA4F8B
:406240007F78BE4277D0A84E76783136A64F3F78BE4270D001204FF46747A34E367806EB860CA14E361D26F82C70AA27361F367806EB860C9C4E361D06EB8C06B7729A4E51
:40628000367806EB860C984E361D06EB8C06F4722712954E367806EB860C934E361D06EB8C063773904E367806EB86078E4E361D06EB870671738C4E367806EB86078A4E64
:4062C000361D06EB8706B273874E367806EB8607854E361D06EB8706F373834E367806EB8607814E361D06EB87063574FF277E4E367806EB860C7C4E361D06EB8C067774A9
:406300000827794E367806EB860C774E361D06EB8C063781744E3678761C322E06DB724E767816B10026704F3E7004E06E4E3678761C6D4F3E70F0BDF0B5044600206A4DDB
:406340002D786D1C684E7678B54278D0664D6D783135654E3678B54271D001204FF46746614D2D7805EB85075F4D2D1D25F82760AB262D1F2D7805EB85075B4D2D1D05EBDB
:406380008705AE72584D2D7805EB8507564D2D1D05EB8705EC722612534D2D7805EB8507514D2D1D05EB87052E734F4D2D7805EB85064D4D2D1D05EB860569734A4D2D7873
:4063C00005EB8506484D2D1D05EB8605AA73464D2D7805EB8507444D2D1D05EB8705EB731E12414D2D7805EB85073F4D2D1D05EB87052E74FF263C4D2D7805EB85073A4D19
:406400002D1D05EB87056E740826374D2D7805EB8507354D2D1D05EB87052E81324D2D786D1C322D06DB304D6D7815B100252E4E357004E02C4D2D786D1C2B4E3570F0BD39
:40644000F0B504460020284D2D786D1C264E7678B5427BD0244D6D783135234E3678B54274D001204FF467461F4D2D7805EB85071D4D2D1D25F82760AC262D1F2D7805EB07
:406480008507194D2D1D05EB8705AE72164D2D7805EB8507144D2D1D05EB8705EC722612114D2D7805EB85070F4D2D1D05EB87052E730D4D2D7805EB85060B4D2D1D05EB75
:4064C00086056973084D2D7805EB8506064D2D1D05EB8605AA73044D2D7805EB8507024D2D1D05EB870501E0483D0010EB731E12FE4D2D7805EB8507FC4D2D1D05EB870585
:406500002E74FF26F94D2D7805EB8507F74D2D1D05EB87056E740826F44D2D7805EB8507F24D2D1D05EB87052E81F04D2D786D1C322D06DBED4D6D7815B10025EB4E35706A
:4065400004E0EA4D2D786D1CE84E3570F0BD70B504460025E5480078401CE449497888427DD0E24840783130E0490978884276D001254FF46741DD48007800EB8002DB4875
:40658000001D20F82210AD21001F007800EB8002D648001D00EB8200817214F05DF8C1B2D248007800EB8002D048001D00EB8200C17214F051F80112CC48007800EB80020E
:4065C000CA48001D00EB82000173C848007800EB8002C648001D00EB820044732112C348007800EB8002C148001D00EB82008173FF21BE48007800EB8002BC48001D00EB86
:406600008200C173B948007800EB8002B748001D00EB82000174B548007800EB8002B348001D00EB820041740821B048007800EB8002AE48001D00EB82000181AB48007831
:40664000401C322806DBA948407810B10020A749087004E0A5480078401CA4490870284670BD70B503460020A04C2478641C9F4D6D78AC4278D09D4C647831349B4D2D7898
:40668000AC4271D001204FF46745984C247804EB8406964C241D24F82650AE25241F247804EB8406914C241D04EB8604A5728F4C247804EB84058D4C241D04EB8504E3723E
:4066C0008A4C247804EB8406884C241D04EB860421730D12854C247804EB8406834C241D04EB86046573814C247804EB84067F4C241D04EB8604A27315127C4C247804EB31
:4067000084067A4C241D04EB8604E573FF25774C247804EB8406754C241D04EB86042574724C247804EB8406704C241D04EB8604657408256D4C247804EB84066B4C241DD2
:4067400004EB86042581694C2478641C322C06DB664C647814B10024644D2C7004E0634C2478641C614D2C7070BD70B5034600205E4C2478641C5D4D6D78AC4279D05B4C3F
:4067800064783134594D2D78AC4272D001204FF46745564C247804EB8406544C241D24F82650AF25241F247804EB84064F4C241D04EB8604A5724D4C247804EB84064B4C06
:4067C000241D04EB8604E3721D12484C247804EB8406464C241D04EB86042573434C247804EB8405414C241D04EB850461733F4C247804EB84063D4C241D04EB8604A27319
:40680000150A3A4C247804EB8406384C241D04EB8604E573150C354C247804EB8406334C241D04EB86042574150E304C247804EB84062E4C241D04EB8604657408252B4C1A
:40684000247804EB8406294C241D04EB86042581264C2478641C322C06DB244C647814B10024224D2C7004E0204C2478641C1F4D2C7070BD73B52DED020B02460B466946E9
:4068800000201A4C2478641C184D6D78AC427ED0164C64783134154D2D78AC4277D001204FF46745114C247804EB84060F4C241D24F82650AF25241F247804EB84060B4C9E
:4068C000241D04EB8604A572084C247804EB8406064C241D04EB8604E2721512034C247804EB8406014C241D02E00000483D001004EB86042573FE4C247804EB8405FC4CB7
:40690000241D04EB850463730D78F94C247804EB8406F74C241D04EB8604A5734D78F44C247804EB8406F24C241D04EB8604E5738D78EF4C247804EB8406ED4C241D04EBAC
:4069400086042574CD78EA4C247804EB8406E84C241D04EB860465740825E54C247804EB8406E34C241D04EB86042581E04C2478641C322C06DBDE4C647814B10024DC4DFC
:406980002C7004E0DA4C2478641CD94D2C7004B070BD30B502460020D54B1B785B1CD44C6478A34277D0D24B5B783133D04C2478A34270D001204FF46744CD4B1B7803EBFA
:4069C0008305CB4B1B1D23F82540B0241B1F1B7803EB8305C64B1B1D03EB85039C72C44B1B7803EB8305C24B1B1D03EB8503DA721412BF4B1B7803EB8305BD4B1B1D03EBD7
:406A000085031C73BA4B1B7803EB8304B84B1B1D03EB84035973FF24B54B1B7803EB8305B34B1B1D03EB85039C73B14B1B7803EB8305AF4B1B1D03EB8503DC73AC4B1B7849
:406A400003EB8305AA4B1B1D03EB85031C74A84B1B7803EB8305A64B1B1D03EB85035C740824A34B1B7803EB8305A14B1B1D03EB85031C819E4B1B785B1C322B06DB9C4B90
:406A80005B7813B100239A4C237004E0984B1B785B1C974C237030BD70B503460020944C2478641C924D6D78AC4278D0904C647831348F4D2D78AC4271D001204FF467450E
:406AC0008B4C247804EB8406894C241D24F82650B125241F247804EB8406854C241D04EB8604A572824C247804EB8406804C241D04EB8604E3721D127D4C247804EB840667
:406B00007B4C241D04EB86042573794C247804EB8405774C241D04EB85046173744C247804EB8406724C241D04EB8604A27315126F4C247804EB84066D4C241D04EB860447
:406B4000E573FF256A4C247804EB8406684C241D04EB86042574664C247804EB8406644C241D04EB860465740825614C247804EB84065F4C241D04EB860425815C4C24787F
:406B8000641C322C06DB5A4C647814B10024584D2C7004E0564C2478641C554D2C7070BD002053490978491C514A5278914276D04F49497831314E4A127891426FD001202D
:406BC0004FF467424A49097801EB81034849091D21F82320B222091F097801EB81034449091D01EB83018A72FF224149097801EB81033F49091D01EB8301CA723C4909780A
:406C000001EB81033A49091D01EB83010A733849097801EB81033649091D01EB83014A733349097801EB81033149091D01EB83018A732F49097801EB81032D49091D01EB9F
:406C40008301CA732A49097801EB81032849091D01EB83010A742649097801EB81032449091D01EB83014A7408222149097801EB81031F49091D01EB83010A811C49097855
:406C8000491C322906DB1A49497811B10021184A117004E016490978491C154A117070472DE9F04106460C461546002710480078401C0F49497888427ED00D484078313057
:406CC0000B4909788842F7D001274FF467410848007800EB80020648001D20F82210B321001F007800EB80020148001D02E00000483D001000EB82008172FE48007800EB73
:406D00008002FC48001D00EB8200C6723112F948007800EB8002F748001D00EB82000173F448007800EB8002F248001D00EB820044732112EF48007800EB8002ED48001DE8
:406D400000EB82008173FF21EA48007800EB8002E848001D00EB8200C173E648007800EB8002E448001D00EB82000174E148007800EB8002DF48001D00EB82004174DD48B6
:406D8000007800EB8002DB48001D00EB82008174601D81B2D748007800EB8002D548001D00EB82000181D348007800EB8001D148001D00EB810000E043E00089082809DA2F
:406DC0000821CC48007800EB8002CA48001D00EB82000181042C15DDC648007800EB8001C448001D00EB81002968C0F80F10281DC049097801EB8102BE49091D01EB820168
:406E000048600DE0BB49097801EB8102B949091D01EB820101F10F00224629467FF1C8FBB4480078401C322806DBB248407840B10020B049087004E0AE480078401CAD4944
:406E400008703846BDE8F081AB4890F8EB007047A94981F8EB007047A748B0F8B4007047302802DAA44981F88E00704700B50021A14880F8251080F826100020FFF7F0FFDC
:406E8000FF209D4981F8BD0000BD014600209A4AB2F8B6200A4002B101207047002318461946954A92F8C320042A06DA924A92F8C330283202EB031203CA7047012907D1C5
:406EC0008D4AB2F8B62002438B4BA3F8B62006E0894AB2F8B6208243874BA3F8B62070472DE9FC418548056828467FF1F0F90446804840787F49097888427CD07D484078BD
:406F000000EB80017B48001D30F82100B0F5674F71D1794890F8BD00FF2808D07649D1F8940040F2DC5112F006FE0028E5D000267048407800EB80016E48001D00EB81007B
:406F400000896E49096888420BD96C48008881B26848407800EB80026648001D00EB820001816448407800EB80016248001D00EB81000089092827DD5E48407800EB800129
:406F80005C48001D00EB810050F80A1F216041686160007A20725748407800EB80035548001D00EB83000089A0F109025148407800EB80034F48001D00EB8300416804F1AB
:406FC00009007FF1F5FA15E04A48407800EB80034848001D00EB830002894648407800EB80034448001D00EB830000F10A0120467FF1DEFA00E033E0FFF750FFCDE9000172
:407000003C48407800EB80013A48001D00EB810002894FF46741204613F0AEF90646F6B13448407800EB80023248001D00EB82000189204666F13AFD20782F4981F8BD00BB
:407040002DF1CAF82C49C1F894002A484078401CC0B228494870322801DB0020487000BF204630F03AFDBDE8FC8170B500260025002426E0FFF712FF1F4A283202EB041339
:407080000CCB801A99411AD2012D0ED11A48283000EB0410D0E900301749283101EB0611D1E900219A1A884100D345B91248283000EB0410407B012801D126460125601C90
:4070C000C4B2042CD6DB35BB002422E00A48283000EB0410D0E900300749283101EB0611D1E900219A1A884100D385B90248283006E00000483D0010583C001060CC19086E
:4071000000EB0410407B012801D126460125601CC4B2042CDADB012D07D1EF4800EB0610D0E900211046F3F712F8284670BD70B50024002513F0D9FA06463146002013F00A
:407140003EFA18B113F0D1FA044609E046F26E51002013F034FA10B146F26E5400E00024DD482838B0F8B400A04204D0DA482838A0F8B4400125284670BDD749283981F8A6
:40718000C1007047D448283890F8C10070477CB502260024D048283890F8C45013F053FA0168009140680190CB482838B0F8B40060B1C9482838B0F8B40000128DF805007E
:4071C000C548283890F8B4008DF80600052D00DD0525002D1ADD002415E0C4EBC402BE489D301118072268467FF17EF928B1BA48283880F8BE40012607E0601CA84200D1C0
:407200000026601CC4B2AC42E7DB00BF30467CBD2DE9FF4104460025FF22082102A87FF10CFAFF208DF80800012C03D101208DF8090002E000208DF8090003208DF80A004B
:40724000FFF72CFE0822CDE900014FF4674102A813F092F830B12CF1BFFF9F492839C1F898000125284604B0BDE8F08110B50446042C0BDC9848283890F8C200A04205D0D0
:407280009548283880F8C24025F06FFE10BD10B500240020FFF7E4FD00218F48283880F8251080F8261000208B492839A1F8B600FF2081F8C300084690F88B1080F88C10B1
:4072C00000BF13E00021844800EB04104173824800EB04108160804A02EB0412116051607D4800EB04100173601CC4B2042CE9DB0020FFF7BBFF0020FDF752FF2CF16CFFC8
:4073000075492839C1F89C000020A1F8B400012081F88D000020C1F8940081F8C00025F0FEFD6E4800786D49487010BD2DE9FF5F00BF0024A146FF22082102A87FF17DF90E
:4073400000BF1FE0644800EB0410407B01280DD1614901EB0411886840F61C4112F0EBFB20B100215C4800EB041041735A4800EB0410407B012803D109F1010000F0FF0937
:40738000601CC4B2042CDDDB4846FFF76FFF5248283890F8250068BBFDF7F2FE002829DD4D48283890F8C300042829DBF2F7CAFE05460E4600241AE0474800EB0410407BFE
:4073C000012812D10020014668407140084307D0414800EB041103C968407140084304D13D48283880F8C34003E0601CC4B2042CE2DB05E02CF1F0FE37492839C1F89C0089
:40740000F2F7B5FE074634492839D1F89C00394612F091FB50B100200146F2F798FEFFF725FDFF202C49283981F8C3002A48283890F82600012828D100212748283880F8D9
:407440002610007E00F00400042806D022482838007E00F01000102805D100201E49283981F8BF0008E01C48283890F8BF00401C1949283981F8BF00FDF79EFE022814D103
:4074800001210846FFF71AFD0FE01348283890F82500012809D110492839C86940F61C4112F049FB08B1FFF7E1FCFDF785FE06280BDB09492839D1F898004FF47A7112F0D6
:4074C0003AFB10B10020FFF7A3FEFDF775FE312880F0C18704E00000803C0010483D0010DFE810F031003B00460057007000780088008C00AC00C400DF00F3000E012201E2
:407500003D015101750189019601BC01D001EB014E025E02AF02CC02DD02F90319043E047804A704E20411054C057B05B305D8050B0634066D068D06B106FF0610071A0773
:4075400079079507B607FDF71FFE20B9FFF79FFE0120FFF785FC00F07EBF12F0ACFF30B100210120FFF7AAFC0220FFF779FCF2E70120FFF78AFC58B10121FE4880F8251063
:407580002CF12AFEFB49C1F894000320FFF768FCE1E7002012F0C0FE18B10420FFF760FC0FE0F449D1F894004FF4FA6112F0C3FA38B12CF111FEEF49C1F89400012012F0EE
:4075C000ABFEC8E70120FFF723FE10B10520FFF747FCC0E7E749D1F898004FF47A7112F0AAFA30B10020FFF713FE10B10620FFF737FCB0E70720FFF733FCACE70020FFF72C
:4076000027FC0F208DF80800FE208DF8090000208DF80A00FFF742FC0322CDE900014FF46A4102A812F0A8FE38B12CF1D5FDD149C1F894000820FFF713FC8CE7FFF704FCEB
:4076400040B1FFF774FD0020FFF702FC0920FFF707FC0AE0C749D1F894004FF4FA6112F06AFA10B10720FFF7FBFB74E700210220FFF724FCC7208DF80800FFF70FFC0822FA
:40768000CDE900014FF4674102A812F075FE38B12CF1A2FDB749C1F894000A20FFF7E0FB59E70220FFF7F1FB18B10B20FFF7D8FB0AE0B049D1F8940040F2DC5112F03BFA45
:4076C00010B10920FFF7CCFB45E700210420FFF7F5FBC3208DF80800FFF7E0FB0822CDE900014FF4674102A812F046FE38B12CF173FDA049C1F894000C20FFF7B1FB2AE704
:407700000420FFF7C2FB18B10D20FFF7A9FB0AE09849D1F8940040F2DC5112F00CFA10B10B20FFF79DFB16E700210820FFF7C6FBC2208DF80800FFF7B1FB0822CDE90001EA
:407740004FF4674102A812F017FE38B12CF144FD8849C1F894000E20FFF782FBFBE60820FFF793FB18B10F20FFF77AFB0AE08149D1F8940040F2DC5112F0DDF910B10D2031
:40778000FFF76EFBE7E600218020FFF797FBC0208DF8080000208DF80A008DF80B008DF80C008DF80D00FFF779FB0822CDE900014FF4674102A812F0DFFD38B12CF10CFDB8
:4077C0006C49C1F894001020FFF74AFBC3E68020FFF75BFB18B11120FFF742FB0AE06549D1F894004FF4FA6112F0A5F910B10F20FFF736FBAFE65F4890F88D00022803D1C1
:407800001A20FFF72DFB02E01220FFF729FBA2E600211020FFF752FB0020564981F8BE0081F8C40023215348C5307EF10EFFDF208DF80800FFF732FB0822CDE900014FF450
:40784000674102A812F098FD38B12CF1C5FC4949C1F894001320FFF703FB7CE61020FFF714FB18B11420FFF7FBFA0AE04149D1F8940040F2DC5112F05EF910B11220FFF761
:40788000EFFA68E6FFF783FC10B101280FD10AE0FDF78AFC18B11520FFF7E2FA02E01720FFF7DEFA07E01520FFF7DAFA03E01A20FFF7D6FA00BF00BF4DE60020FFF75DFC4E
:4078C00000212020FFF7FAFAD2208DF80800294890F8BE00C0EBC0012648C530405C8DF80900244890F8BE00C0EBC000401C2149C531085C8DF80A001E4890F8BE00C0EBEB
:40790000C000801C085C8DF80B001A4890F8BE00C0EBC000C01C085C8DF80C00154890F8BE00C0EBC000001D085C8DF80D00114890F8BE00C0EBC000401D085C8DF80E0094
:407940000C4890F8BE00C0EBC000801D085C8DF80F00FFF7A3FA0822CDE900014FF4674102A812F009FD50B12CF136FC0149C1F8940001E0583C00101620FFF771FAEAE58A
:407980002020FFF782FA38B9FE49D1F8940040F2DC5112F0D0F810B11220FFF761FADAE512F051FE82460020FFF7E7FB00214020FFF784FAD1208DF808009AF800008DF8B9
:4079C00009009AF801008DF80A009AF802008DF80B009AF803008DF80C009AF804008DF80D00E848B0F8B40058B1E648B0F8B40000128DF80E00E34890F8B4008DF80F002B
:407A000007E09AF805008DF80E009AF806008DF80F00FFF743FA0822CDE900014FF4674102A812F0A9FC58B10020D64981F8BF002CF1D2FBD349C1F894001820FFF710FAAE
:407A400089E54020FFF721FA78B1FFF79BFB18B92C20FFF705FA10E0FFF794FB00F0040058B91A20FFF7FCF907E0C64890F8BF00032802DB1720FFF7F3F96CE5C14890F882
:407A8000C00004280ADABF49D1F8940042F2107112F051F810B11A20FFF7E2F95BE50020B849087500218020FFF708FA0020B54981F8B800C1F8A40000240BE0204612F00B
:407AC00068FDB049D1F8A4100844AE49C1F8A400601CC4B2204612F05CFD08B1FF2CEDDB0020A84981F8B900C1F8A80000240EE0A448B0F8B410204612F061FDA149D1F825
:407B0000A81008449F49C1F8A800601CC4B29D48B0F8B410204612F052FD08B1FF2CE7DB0020984981F8BA00C1F8AC0000240BE0204612F07CFD9349D1F8AC100844914948
:407B4000C1F8AC00601CC4B2204612F070FD08B1FF2CEDDB00208B4981F8BB00C1F8B000002410E00420FDF73EFB07463946204612F060FD8349D1F8B01008448149C1F882
:407B8000B000601CC4B20420FDF72DFB07463946204612F04FFD08B1FF2CE3DB002410E00520FDF720FB07463946204612F045FD7449D1F8B01008447249C1F8B000601CD1
:407BC000C4B20520FDF70FFB07463946204612F034FD08B1FF2CE3DB002410E00620FDF702FB07463946204612F02AFD6549D1F8B01008446349C1F8B000601CC4B20620AF
:407C0000FDF7F1FA07463946204612F019FD08B1FF2CE3DB5B48D0F8A8005A49C1F8A000084690F88D00012827D10846D0F8A000D1F8A41008445349C1F8A0000846D0F85C
:407C4000A000D1F8B01008444E49C1F8A000FFF725F94FF478420020114080EA000280EA01031A4309D14748D0F8A0004549D1F8AC1008444349C1F8A000C0208DF8080064
:407C8000404890F8A0008DF80A003E48B0F8A000000A8DF80B003B48D0F8A000000C8DF80C003848D0F8A000000E8DF80D00FFF7F5F80822CDE900014FF4674102A812F0B2
:407CC0005BFB38B12CF188FA2E49C1F894001B20FFF7C6F8BFE38020FFF7D7F878B12948007DB8B9274890F88D00022803D12620FFF7B6F80EE01C20FFF7B2F80AE02149DA
:407D0000D1F894004FF4FA6111F015FF10B11A20FFF7A6F89FE31B4991F8B80012F039FCB0B10020174981F88F00FFF7B7F807468846144991F8B80012F02BFC00F1010ADA
:407D40003A46434651464FF4674012F083FB03E002200C4981F88F001D20FFF781F87AE3084890F88F0002281FD1064991F8B80012F00FFC70B1034890F8B800401C01491E
:407D800002E00000583C001081F8B8001C20FFF767F81EE00020F94981F8BB00042081F88D001E20FFF75CF813E0F44890F88F0003280ED1F14890F8C000401CEF4981F857
:407DC000C0002CF109FAED49C1F894001920FFF747F840E30420FDF706FA0746E74991F8BB00394612F026FCD8B10020E34981F88F00FFF753F8074688460420FDF7F3F9D6
:407E00008346DE4991F8BB00594612F013FC00F1010A3A46434651464FF4674012F01AFB03E00220D54981F88F001F20FFF718F811E3D24890F88F00022820D10420FDF7F9
:407E4000D2F90746CD4991F8BB00394612F0F2FB50B1CA4890F8BB00401CC84981F8BB001E20FEF7FDFF1EE00020C44981F8BB00052081F88D002020FEF7F2FF13E0BF4852
:407E800090F88F0003280ED1BC4890F8C000401CBA4981F8C0002CF19FF9B849C1F894001920FEF7DDFFD6E20520FDF79CF90746B24991F8BB00394612F0BFFBD8B10020DA
:407EC000AE4981F88F00FEF7E9FF074688460520FDF789F98346A94991F8BB00594612F0ACFB00F1010A3A46434651464FF4674012F0B0FA03E00220A04981F88F00212040
:407F0000FEF7AEFFA7E29D4890F88F00022820D10520FDF768F90746984991F8BB00394612F08BFB50B1954890F8BB00401C934981F8BB002020FEF793FF1EE000208F49C2
:407F400081F8BB00062081F88D002220FEF788FF13E08A4890F88F0003280ED1874890F8C000401C854981F8C0002CF135F98349C1F894001920FEF773FF6CE20620FDF717
:407F800032F907467D4991F8BB00394612F058FBD8B10020794981F88F00FEF77FFF074688460620FDF71FF98346744991F8BB00594612F045FB00F1010A3A4643465146F1
:407FC0004FF4674012F046FA03E002206B4981F88F002320FEF744FF3DE2684890F88F0002281DD10620FDF7FEF80746634991F8BB00394612F024FB50B1604890F8BB0042
:40800000401C5E4981F8BB002220FEF729FF1BE003205A4981F88D002420FEF721FF13E0564890F88F0003280ED1544890F8C000401C524981F8C0002CF1CEF84F49C1F890
:4080400094001920FEF70CFF05E24C4991F8BA0012F0EDFAB0B10020484981F88F00FEF71DFF07468846454991F8BA0012F0DFFA00F1010A3A46434651464FF4674012F011
:40808000E9F903E002203D4981F88F002520FEF7E7FEE0E1394890F88F00022818D1374991F8BA0012F0C3FA50B1344890F8BA00401C324981F8BA002420FEF7D1FE1BE072
:4080C00002202E4981F88D002620FEF7C9FE13E02A4890F88F0003280ED1284890F8C000401C264981F8C0002CF176F82349C1F894001920FEF7B4FEADE1204AB2F8B41013
:4081000092F8B90012F05BFAC0B100201B4981F88F00FEF7C3FE07468846184AB2F8B41092F8B90012F04BFA00F1010A3A46434651464FF4674012F08DF903E002200F4912
:4081400081F88F002720FEF78BFE84E10B4890F88F0002281ED1094AB2F8B41092F8B90012F02DFA60B1054890F8B900401C034981F8B9002620FEF773FE1FE0583C001055
:408180000020F94981F8BC002820FEF769FE24F0F1FE13E0F44890F88F0003280ED1F24890F8C000401CF04981F8C0002CF114F8ED49C1F894001920FEF752FE4BE100216A
:4081C0004FF48070FEF77AFE12208DF80800FEF765FE0822CDE900014FF4674102A812F0CBF858B10020E04981F8BF002BF1F4FFDD49C1F894002920FEF732FE2BE14FF4C4
:408200008070FEF742FE30B1FEF7BCFFD0B92A20FEF726FE16E0D44890F8BF00032811DBD14890F8BC0003280ADACF4890F8BC00401CCD4981F8BC002820FEF711FE01E091
:40824000FEF714FE07E112F0FEF982460020FEF794FF00214FF40070FEF730FED0208DF808009AF800008DF809009AF801008DF80A009AF802008DF80B009AF803008DF8B2
:408280000C009AF804008DF80D00B748B0F8B40058B1B548B0F8B40000128DF80E00B24890F8B4008DF80F0007E09AF805008DF80E009AF806008DF80F00FEF7EFFD082216
:4082C000CDE900014FF4674102A812F055F838B12BF182FFA449C1F894002B20FEF7C0FDB9E04FF40070FEF7D0FD38B99E49D1F8940047F2305111F01EFC10B12C20FEF70C
:40830000AFFDA8E00020984981F8C00081F88D002D20FEF7A5FD9EE0FEF796FD68B10020FEF796FDFEF703FFF0B302208E4981F88D001120FEF794FD4CE0FCF72DFF50B182
:40834000FEF793FE18B12E20FEF78AFD42E00020FCF726FF3EE0FCF717FF18B12E20FEF77FFD37E0804890F88C1090F88B0081422ED07D4890F88C00C0EBC0017A48683065
:408380000844016802918188ADF80C1080798DF80E00FEF783FD0822CDE900014FF4674102A811F0E9FF00E014E098B1072102A865F17CFB6C4890F88C00401CC1B26A4846
:4083C00080F88C10052905DB002180F88C1001E0FEF786FD3FE000214FF48060FEF76EFDB2208DF80800FEF759FD0822CDE900014FF4674102A811F0BFFF38B12BF1ECFE3C
:408400005949C1F894002F20FEF72AFD23E04FF48060FEF73AFDD0B1FEF728FDFCF7BCFEA8B1002410E0F1F78DFE4F4A283202EB04130CCB50405940084303D14A4880F848
:40844000C34003E0601CC4B2042CECDB00BF02E0FEF70CFD00BF00BFBDE8FF9F2DE9F04F044689469246DDE909676079A17940EA0120E17940EA014594F8008094F801B000
:40848000FCF75DFE98420CD1B8F1010F08D1B5F5674F04D1BBF1FF0F01D1FEF7E7FC00BF00BFBDE8F08F70B504460D462E4880F8C440052C00DD0524C4EBC40229462A48A9
:4084C000C5307EF175F870BD70B504460D46164625488472C572068112F0B7F800EE100AF8EE400A2048008900EE100AB8EE400A80EE201A1C4880ED001A70BD1A4B1873BD
:4085000059739A7370472DE9F0412DED028B06460F4614461D4612F09BF800EE100AF8EE400A00EE104AB8EE400A80EE201AB0EE418A12F08FF800EE100AF8EE400A00EE9A
:40854000105AB8EE400A80EE201AF0EE418A064886744774C4730574B4EEE88AF1EE10FA04D280ED018A04E0583C0010FE48C0ED018ABDEC028BBDE8F0812DE9F05F0446D1
:408580008A4693469846DDE90A6794F800900025B9F1FE0F33D100BF2EE0F348283000EB051103C97040794008430AD0EE48283000EB0510D0E90010002359405840014357
:4085C00018D12BF109FEE849283101EB051188600121E548283000EB05104173E248283000EB051080F80C80DF48283000EB0510C0C003E0681CC5B2042DCEDB00BFFCF7B1
:408600009EFD40457DD1B9F1AD0F7BD054DCB9F1250F78D027DCB9F1080F75D008DCB9F1080F72D2DFE809F0A6A7A8A9AAABACADB9F1200F6AD00CDCB9F1090F67D0B9F129
:408640000A0F65D0B9F1120F71D0B9F1130F5CD1E9E0B9F1210F6BD0B9F1220F69D0B9F1240FF4D1E3E0B9F1A40F74D01ADCB9F1A00F71D00CDCB9F1260F6ED0B9F1270F3A
:408680006CD0B9F1900F6AD0B9F1920FDFD1D3E0B9F1A10F77D0B9F1A20F75D0B9F1A30FD5D1CDE0A9F1A5000828BAD2DFE800F0CACBCCCDCECFD0D1B9F1C00F7ED00EDC8E
:4086C000A9F1AE001128ACD2DFE800F0C5C6C7C8CBD0D1D2D3D4D5D6D7D8D9DADB00B9F1D10F6CD026DCB9F1C50F69D015DCB9F1C10F66D0B9F1C20F7BD0B9F1C30F79D032
:4087000007E041E1A6E093E03CE032E18CE03CE07CE0B9F1C40F9AD1D4E0B9F1C60F6AD0B9F1C70F68D0B9F1D00F90D1DDE06EE07BE07BE0B9F1D60F71D011DCB9F1D20F24
:408740006ED0B9F1D30F6CD0B9F1D40F6AD0B9F1D50F86D1E3E074E06FE06AE06AE06AE0B9F1E00F7BD0B9F1FD0F79D0B9F1FE0F8CD1E0E000BF00BF00BF00BF00BF00BFD2
:4087800000BF00BFF5E059E059E0774890F88B00401C754991F88C10884236D0724890F88C00001D704991F88B1088422DD06E4890F88B00C0EBC0016B4803E062E09CE0FB
:4087C00081E069E06830084421680160A1888180A1798171644890F88B00401C05280CDB614890F88C0080B100215F4880F88B100BE052E05CE067E067E05B4890F88B0036
:40880000401CC1B2584880F88B10B2E0B1E06078FEF7B3FC01210802FEF750FBA9E07FE073E07AE07AE000BF00BF00BF00BF00BF00BF00BF00BF00BF00BF00BF00BF00BF09
:4088400000BF00BF00BF00BF00BF00BF00BF00BF00BF00BF00BF00BF00BF00BF89E060E068E001218802FEF729FB82E000BF00BF00BF00BF00BF00BF00BF00BF00BF00BFF8
:4088800000BF76E060783849C874A078087501218020FEF713FB6CE06BE063792279A179E079FFF730FE01210820FEF707FB60E0E279A1796079FFF721FE01210420FEF7F0
:4088C000FDFA56E000BF00BF53E0237994F805C043EA0C22E378C3F34001A078FFF7F4FD01210220FEF7EAFA43E06079FEF745FC01214802FEF7E2FA3BE06079FEF73DFC53
:4089000001214020FEF7DAFA33E06079FEF735FC01212020FEF7D2FA2BE000BF00BF00BF27E06078A11CFFF7BEFD01211020FEF7C5FA1EE01DE02BF14FFC0B49C86101211B
:40894000094880F82610617880F82410A078E17840EA0121044801842079617940EA012101484184A07901E0583C00101E49087600BF00BF1C4890F8BD002178884203D137
:40898000FF20194981F8BD00BDE8F09F2DE9FC4781460E4617469846DDE90A45B6F5664F14D111F08DFDFE2807DAFCF7C8FB404503D13946484665F1AFFD43463A46314693
:4089C0004846CDE90045FFF7D8FD0AE0B6F5684F07D143463A4631464846CDE90045FFF73DFDBDE8FC870000583C00102DE9F04104460D4616461F463A4631462046F0F711
:408A0000BBFA04462C482060E5602046BDE8F08110B504462046F0F7B4FA0446204610BD70B504462046FFF7F3FF05462FF0D6FF70BD01460120704770B504460D460026CB
:408A400000202860E06820B12946E0683EF180F90646304670BD2DE9F04104460D4616460027E06828B132462946E0683EF189F907463846BDE8F0812DE9F04104460D46BA
:408A800016461F464FF00008E06830B13B4632462946E0683EF193F980464046BDE8F08170B504464FF0FF35E06818B1E0683EF1A5F90546284670BDCCCF190870B504469F
:408AC0000025022614B9544D00BF00BF00BF25B13246294651483EF12EFF70BD70B504460D466FF00040206015B1012D06D100E008E0206840F00040206003E00020FFF7BA
:408B0000DDFF00BF00BF204670BD70B504460E46154626F00040206015B1012D06D100E008E0206840F00040206003E00020FFF7C5FF00BF00BF204670BD0A6802607047F0
:408B400070470A680260704770B50446062520467FF15CF828B1012805D12068C0F3826501E0002500BF00BF284670BD0146086800F0807008B1012070470020FCE7014664
:408B8000086800F0007008B1012070470020FCE770B504464FF0FF3520467FF137F801280DD1206800F47000B0F5700F04D21C49206801EA102502E02068C0F311252846AF
:408BC00070BD70B50446FF2520467FF11FF8012802D12068C0F30745284670BD70B50446FF2520467FF112F8012808D1206800F47000B0F5700F02D22088C0F3072528465C
:408C000070BD70B50446FF2520467EF1FFFF012800D12578284670BDC9DD0408BADD040800FF03000246104649B108B9084606E000E000680368002BFBD101601046704773
:408C40002DE9F04706460C4617469846DDF82090B24600250DE024B139465046A047012803D1A84500D107E06D1C50467EF1E2FE8246BAF1000FEED100BFB9F1000F01D0D4
:408C8000C9F800505046BDE8F0872DE9F8430446884615461E460027B8F1000F14D09DB1002000900023324641462068FFF7C8FF074647B93046A847074639462068FFF7A5
:408CC000B1FF206000E000273846BDE8F8832DE9F04706460C4617464FF0FF39B04600250EE024B139464046A047012800D16D1C40467EF19FFE8046B5F1FF3F00D102E0A4
:408D0000B8F1000FEDD100BF2846BDE8F087014621B10868884201D1012070470020FCE700B5024612B1106800B912601046FFF7EEFF00BD10B50346184600241470C0B196
:408D4000B9B1884204D100680C600124147010E00AE004688C4206D10C68046000240C600124147003E000680468002CF1D100BF184610BD38B504460D46002000906A46F8
:408D800029462046FFF7D6FF38BD0021016070470021016070470000002101604160491E8160090AC1604FF0FF3101610021416181617047A4480068401CA349086008468E
:408DC0000068704770B504460025022624B1012C05D0022C09D105E09C4D022605E09C4D022602E09B4D022600BF00BF25B13246294699483EF19FFD70BD2DE9F041044636
:408E00000E4617464FF00008B7F1FF3F56D0002552E0C5EBC50104F1100000EB81000069B0F1FF3F47D100BF7068C5EBC50204F1100141F8220000BFB068C5EBC50201EBE7
:408E40008201486000BF06F10C00FFF7A1FEC5EBC50204F1100101EB8201C860C5EBC50204F1100000EB8200E1688160C5EBC50204F1100000EB820000F114013068082298
:408E8000036930469847012814D1C5EBC50104F1100000EB8100076120680A2808D22068401C2060A1682068884201D92068A0604FF0010802E06D1C0A2DAAD3B8F1000FC0
:408EC00005D10020FFF77EFF6068401C6060E068401CE0604046BDE8F08170B504460D460026B5F1FF3F25D0711E00201FE0C0EBC00304F1100202EB83021269AA4215D102
:408F0000C0EBC00304F1100202EB830292688A420CD2C0EBC00304F1100202EB83029168C0EBC00304F1100202EB8306401C0A28DDD302E00120FFF745FF304670BD70B598
:408F400004460D46002665B12869B0F1FF3F08D0701E2861206810B12068401E2060012602E00220FFF72EFF304670BD90ED000AB8EE400ADFED390A60EE200AB2EE041A5D
:408F800080EE810A704701464868704790ED020AB8EE400ADFED310A60EE200AB2EE041A80EE810A70470146C868704710B50446002020606060A060E0600A231C22AFF204
:408FC000272104F110007EF180FEA0F11004204610BD704770B505460E46002425E0C4EBC40105F1100000EB81000069B0F1FF3F1AD086B1C4EBC40105F1100000EB810086
:409000004068B04207D0C4EBC40105F1100050F82100B04208D1C4EBC40205F1100000EB82012846FFF78BFF641C0A2CD7D370BD10B50B48FFF7BAFF04460A4AAFF26D0139
:409040002EF024FF10BD00005401001013DE040823DE040852DE040801DE04080000C8423C2200200080000870B504460025022614B9544D00BF00BF00BF25B13246294618
:4090800051483EF158FC70BD70B5054628463EF181FF05464D48286008202FF0A7FC0646002030603446706084B1256060604848006810B9464804600BE04549086800E04C
:4090C000406841680029FBD1446002E00020FFF7CBFF284670BD70B506463C4830603C48046800250FE02068B0420AD11DB938496068086001E06068686020462FF06EFC64
:4091000003E025466468002CEDD100BF3148046800250FE02068B0420AD11DB92D496068086001E06068686020462FF057FC03E025466468002CEDD100BF30463EF12DFFC5
:409140000646304670BD70B504462046FFF7C3FF05462FF043FC70BD30B503461D4804681B48056800220020086005E0934201D120680860521C646814B108680028F5D04C
:4091800005E0934201D128680860521C6D6815B108680028F5D0086808B1012030BD0020FCE70C4B19680A4B1A68002001E0401C49680029FBD101E0401C5268002AFBD1EC
:4091C00070470000C3BF1908B6BF1908A0CE19085C0100105801001070B5044600250226082C1DD2DFE804F004070A0D10131619A14D012614E0A14D012611E0A04D0226E8
:409200000EE0A04D02260BE09F4D022608E09F4D022605E09E4D022602E09E4D022600BF00BF25B1324629469B483EF184FB70BD2DE9F05F04460F4615461E46DDE90A892E
:409240003A464946204638F19FFD04469348206084F81D800020A07700BF00BFE06865F31E00E06000BF00BF0020C4F81500C4F81900002E71D0607F08286FDC607F00282F
:409280006CD0627F314604F115007DF191F9207D022877DA00BF00BFE06800F0004008B1012000E0002000BF002858D0012864D120467EF198FCB0F1005F4AD220467EF169
:4092C00092FC00F0FF0ABAF1FE0F19DBBAF1FE0F3BD120467EF187FC71490840B0F56A0F06D1607D20B9A07DEE2801D1E07D38B120467EF178FC6A490840B0F56E0F24D1CC
:40930000217D04F1080250462FF038FA20467EF16AFC00F47000B0F5700F13D220467EF162FCC0F3072BBBF1FE0F07D0217D221D58462FF023FA0120A07702E00020FFF772
:409340004BFF05E00120A07702E00120FFF744FF02E00220FFF740FF13E01BE016E020467EF141FCB0F5006F02D20120A07702E00320FFF731FF04E004E00420FFF72CFFC3
:4093800000BF0AE00520FFF727FF06E00620FFF723FF02E00720FFF71FFF2046BDE8F09F10B50446204638F122FD0446204610BD70B504462046FFF7F3FF05462FF00EFB7E
:4093C00070BD014601207047024602F115000860012070472DE9F04104460D4616460027607FB04207D835B1627F04F1150128467DF1DEF801273846BDE8F0812DE9F041F3
:4094000004460D4616461F464FF00008F019617F884209D845B104F1150081193A4628467DF1C6F84FF001084046BDE8F0810146487F70470146887F704770B504462046BC
:409440007EF1D1FBC5B2217D04F1080228462FF095F920467EF1C7FB00F47000B0F5700F09D220467EF1BFFBC0F30725217D221D28462FF083F970BD91DE0408ADDE0408F5
:40948000C4DE0408E5DE040806DF04081EDF040832DF040846DF04087DDE04089CD00A080000FF0370B504460D462946204638F187FC0446FC4844F8180B55F8180F2060DC
:4094C000287B2073687B6073A87BA073D5E90101183DC4E90101183C204670BD70B504460D462946204638F16BFC0446EE4820600020A06184F82400286881692846884700
:4095000084F82500002084F826002868082204F11C01036928469847204670BD10B5044601220021204638F12FFC0446DE4820600020A061152084F82400002084F82500FC
:4095400084F82600E0612062204610BD10B50446204638F14CFC0446204610BD70B504462046FFF7F3FF05462FF038FA70BD014602207047024602F11C00086001207047B3
:409580002DE9F04104460D461646002794F82500B04208D83DB194F8252004F11C0128467DF106F801273846BDE8F0812DE9F04104460D4616461F464FF00008F01994F8D9
:4095C0002510884209D845B104F11C0081193A4628467CF1EDFF4FF001084046BDE8F081014691F825007047014691F8240008B9012070470020FCE7704770B50446002538
:4096000002260C2C2BD2DFE804F006090C0F1215181B1E212427A54D022620E0A44D02261DE0A44D02261AE0A34D022617E0A34D002614E0A24D022611E0A24D00260EE09D
:40964000A14D02260BE0A14D022608E0A04D022605E0A04D022602E09F4D022600BF00BF25B1324629469D483EF165F970BD2DE9F84F04460D46174698460AAE96E8400E53
:409680005146484638F11EFD012201460090204638F17AFB0446844820600E98A061002084F8240084F825800F9884F82600C4F80890C4F804A00020E0612062A068002815
:4096C00075D0D4E90101884272D0002F71D094F82500082877DC94F82500002873D0072E6ADCB5F5802F5BD294F82520394604F11C007CF15DFF207D02284ADAA068026812
:40970000D168884701283DD105F47040B0F5704F31D2E8B240BB606890B9BBF1FE0F08D0B00640EA052040EA0B2120462EF0A1FF64E0022084F824000420FFF75EFF5DE06A
:4097400060680268D1688847012806D1B00640EA052120462EF08DFF50E0022084F824000420FFF74AFF49E0032084F824000520FFF743FF42E0B00640EA052120462EF04F
:4097800078FF3BE0042084F824000620FFF735FF34E0052084F824000020FFF72EFF2DE0062084F824000320FFF727FF26E01FE017E00FE007E0FFE7072084F82400012035
:4097C000FFF71BFF1AE0082084F824000720FFF714FF13E0092084F824000220FFF70DFF0CE00A2084F824000820FFF706FF05E00B2084F824000920FFF7FFFE2046BDE8D7
:40980000F88F2DE9F05F04460F4615461E46DDE90DABDDE90A983A4620460C9938F1B4FA044621482060C4F818A0002084F8240084F8259084F826B0E061206200BF00BF6B
:40984000E06800F0004008B1012000E0002000BF002872D001286FD1002E65D094F8250008285ADC94F82500D0B3207D02284DDAB8F1070F43DCB5F1806F39D205F4700081
:40988000B0F5700F03D2C5F30720FE2829D094F82520314604F11C007CF18AFE45EA886120462EF0E6FE45E074D31908FCBF190810C0190825C0190837C019085BC019082F
:4098C00077C01908ABC01908C2C01908D6C01908EEC019080DC119082EC11908E7BF19081BE0032084F824000520FFF786FE21E0062084F824000320FFF77FFE1AE00720BA
:4099000084F824000120FFF778FE13E0052084F824000020FFF771FE0CE0082084F824000720FFF76AFE05E0092084F824000220FFF763FE3EE000E035E06EB394F8250078
:40994000082822DC94F82500F8B1207D022815DAB5F5006F0BD294F82520314604F11C007CF126FE294620462EF083FE1AE00C2084F824000A20FFF740FE13E0052084F89D
:4099800024000020FFF739FE0CE0082084F824000720FFF732FE05E0092084F824000220FFF72BFE06E0012084F824000B20FFF724FE00BF00BF2046BDE8F09F70B50446D5
:4099C00000255CB1002007E0265C2C2E03D114601870012502E0401C8842F5D31DB900201060FF201870284670BD2DE9F04105460F4614461E464FF0000833462246394698
:409A00002846FFF7DBFFD8B12068401B18D42068401BB84214D23078401C2168084420602168481B0AE0295C2A2906D12178491B411A31704FF0010802E0401CB842F2D3B1
:409A4000B8F1000F03D100202060FF2030704046BDE8F0812DE9F04105460F4614461E464FF000083346224639462846FFF7BDFFD8B12068401B18D42068401BB84214D2D8
:409A80003078401C2168084420602168481B0AE0295C2A2906D12178491B411A31704FF0010802E0401CB842F2D3B8F1000F03D100202060FF2030704046BDE8F0812DE9ED
:409AC000F04105460F4614461E464FF000083346224639462846FFF7BDFFD8B12068401B18D42068401BB84214D23078401C2168084420602168481B0AE0295C2A2906D117
:409B00002178491B411A31704FF0010802E0401CB842F2D3B8F1000F03D100202060FF2030704046BDE8F0812DE9F04105460F4614461E464FF000083346224639462846A6
:409B4000FFF7BDFFD8B12068401B18D42068401BB84214D23078401C2168084420602168481B0AE0295C2A2906D12178491B411A31704FF0010802E0401CB842F2D3B8F153
:409B8000000F03D100202060FF2030704046BDE8F0812DE9F04105460F4614461E464FF000083346224639462846FFF7BDFF20B32068401B21D42068401BB8421DD230783C
:409BC000401C2168084420602168481B0AE0295C2A2906D12178491B411A31704FF0010802E0401CB842F2D3B8F1000F05D12078401B381A30704FF00108B8F1000F03D1AA
:409C000000202060FF2030704046BDE8F0812DE9F04705460F46164698464FF0000900241FE029190422F8A02EF063F9C0B9241D285D502803D1641C2819306001E028191F
:409C40003060204609E0295C2C2905D1011B88F800104FF0010902E0401CB842F3D302E0641CBC42DDD3B9F1000F04D100203060FF2088F800004846BDE8F0872DE9F0477E
:409C800005460E46174698464FF00009002426E029190422DCA02EF02CF9F8B9241D285D502800D1641C15E0285D2C2811D1641C28193860204609E0295C2A2905D1011BCF
:409CC00088F800104FF0010902E0401CB042F3D302E0641CB442E7D300BF02E0641CB442D6D3B9F1000F04D100203860FF2088F800004846BDE8F0872DE9F04705460F4647
:409D0000164698464FF0000900241FE029190422BFA02EF0EEF8C0B9241D285D502803D1641C2819306001E028193060204609E0295C2C2905D1011B88F800104FF0010931
:409D400002E0401CB842F3D302E0641CBC42DDD3B9F1000F04D100203060FF2088F800004846BDE8F0872DE9F04705460E46174698464FF00009002426E029190422A4A009
:409D80002EF0B7F8F8B9241D285D502800D1641C15E0285D2C2811D1641C28193860204609E0295C2A2905D1011B88F800104FF0010902E0401CB042F3D302E0641CB4424D
:409DC000E7D300BF02E0641CB442D6D3B9F1000F04D100203860FF2088F800004846BDE8F08701468C4870470146886D704710B504462046FFF748F904468848206000202F
:409E00006060A060E06020616061A061E06120626062A062E06220636063A063E06320646064A065204610BD10B504462046FFF752F90446204610BD70B504462046FFF70C
:409E4000F3FF05462EF0CAFD70BD70B5044600250226052C13D2DFE804F00306090C0F006F4D02260BE06F4D022608E06E4D022605E06E4D022602E06D4D022600BF00BF51
:409E800025B13246294664483DF155FD70BD2DE9FC4704460F4690461D460A9E4FF00009002088F800003070002D7BD028706870172F78D2DFE807F00C1A283644526478FF
:409EC0008694BED1E4FDFCFBFAF9F87777F7F600E06850B100200190414601A8E268904781469DF80400287000BF3CE1206950B100200190414601A82269904781469DF8D3
:409F00000400287000BF2EE1606950B100200190414601A86269904781469DF80400287000BF20E1A06950B100200190414601A8A269904781469DF80400287000BF12E13B
:409F4000E06950B100200190414601A8E269904781469DF80400287000BF04E1206A70B100200190414601A8226A90478146BDF804002870BDF804000012687000BFF2E0BD
:409F8000606A70B100200190414601A8626A90478146BDF804002870BDF804000012687000BFE0E0ECE0DDE0A06A50B100200190414601A8A26A904781469DF804002870A8
:409FC00000BFD0E0E06A50B100200190414601A8E26A904781469DF80400287000BFC2E0206B78B10020019000904246694601A8236B984781469DF8040028709DF800007B
:40A00000687000BFAFE00000424C442C000000004150502C0000000046C1190890D40A0862C1190898C11908C6C11908F3C1190818C21908606B78B100200190009042465E
:40A04000694601A8636B984781469DF8040028709DF80000687000BF85E0A06B78B10020019000904246694601A8A36B984781469DF8040028709DF80000687000BF72E09A
:40A08000E06BC0B10020019000904246694601A8E36B984781469DF8040028709DF80000687007E04EE03FE030E021E059E057E010E001E000BF56E0206C50B10020019078
:40A0C000414601A8226C904781469DF80400287000BF48E0606C50B100200190414601A8626C904781469DF80400287000BF3AE0A06C50B100200190414601A8A26C9047F5
:40A1000081469DF80400287000BF2CE0E06C50B100200190414601A8E26C904781469DF80400287000BF1EE0206D50B100200190414601A8226D904781469DF80400287087
:40A1400000BF10E0606D50B100200190414601A8626D904781469DF80400287000BF02E000BF00BF00BF00BF687810B10220307006E0287810B10120307001E0002030703A
:40A180004846BDE8FC87FEB50546286881682846884700285ED001285DD0022802D003285BD159E02E4630467DF142FD08BBFF208DF8040000208DF80500002411E00DF13E
:40A1C000070002AB421E21460090FE48FFF75FFE28B19DF80500401CC0B28DF80500601CC4B2162CEBDD022201A9304637F149FC2FE0002700241DE08DF804400DF106001F
:40A20000431C421E21460090EE48FFF740FE78B130467DF10DFD401EB84207D19DF80600C21C01A9304637F12CFC05E0781CC7B2601CC4B2162CDFDD00BF96F8290038B985
:40A24000FF208DF80400012201A9304637F119FC00BF02E000BF00BF00BF00BFFEBD7CB504462068816820468847002872D0012871D0022802D003286ED189E0254600200F
:40A2800001902A20009028467DF1D2FC0C2877D2DFE800F0061218242A363C484E5A637001A8C9490968884706469DF804203146284637F1E6FB67E001226946284637F105
:40A2C000E0FB61E001A8C1490968884706469DF804203146284637F1D4FB55E001226946284637F1CEFB4FE001A8B9490968884706469DF804203146284637F1C2FB43E0FC
:40A3000001226946284637F1BCFB3DE001A8B1490968884706469DF804203146284637F1B0FB31E001226946284637F1AAFB2BE001A8A9490968884706469DF804203146C1
:40A34000284637F19EFB1FE001226946284637F198FB19E01AE01AE01BE001A89F490968884706469DF804203146284637F189FB0AE005E001226946284637F182FB03E0CE
:40A380000020FFF762FD00BF00BF02E000BF00BF00BF00BF7CBD7CB504462068816820468847002851D0012850D0022802D003284ED14CE02546002001902A20009028460A
:40A3C0007DF136FC06283AD2DFE800F0030F1521273301A882490968884706469DF804203146284637F14DFB2DE001226946284637F147FB27E001A87A4909688847064666
:40A400009DF804203146284637F13BFB1BE001226946284637F135FB15E001A872490968884706469DF804203146284637F129FB09E001226946284637F123FB03E001204B
:40A44000FFF703FD00BF00BF02E000BF00BF00BF00BF7CBDFEB504462068816820468847002839D0012838D0022802D0032836D134E02546002002902A20019028467DF136
:40A48000D7FB48B9594800688047009001226946284637F1F6FA1EE028467DF1C9FB401E00F0010090B928467DF1C2FB401EC0F3470702A938464E4A1268904706469DF8F0
:40A4C00008203146284637F1DCFA04E0012201A9284637F1D6FA02E000BF00BF00BF00BFFEBD10B504463D48006870B13848006858B13948006840B13348006828B1334882
:40A50000006810B13348006810B90220FFF79DFC3448006828B13248006810B13248006810B90320FFF791FC3148006810B12F48006810B90420FFF788FC00224FF6C5517F
:40A5400020463AF19CFF00224FF68D4120463AF196FF00224FF6DA6120463AF190FF00224FF68E4120463AF18AFF00224FF6425120463AF184FF00224FF6325120463AF1B9
:40A580007EFF10BD70B504460125A06810B1A06880470546284670BD2DE9FF4F89B00646DDF87480DDE918741A9D01200890B06D401CB0650F4838600020206006202870EF
:40A5C000002119E064230020F4CA1908F8CA1908ECCA1908FCCA1908F0CA1908E8CA190804CB190800CB190808CB190810CB19080CCB1908980200201B9801701C980160B5
:40A600000020C8F800004FF642520C98811A90427ED00ADCA0F57C40A0F18D00002878D0012877D0A52876D1F3E0832903D0B1F5CC7FF8D152E00020079007A8B7490968A4
:40A6400088479DF81C102068084420602068401C206007A8B249096888479DF81C102068084420602068401C206007A8AD49096888479DF81C102068084420602068401C51
:40A68000206007A8A849096888479DF81C102068084420602068401C206007A8A349096888479DF81C102068084420602068401C206007A89E49096888479DF81C1020684E
:40A6C000084420602068401C20600020386006202870AFF27540C8F800000CE1002007902068401C20604FF0000910E007A94846904A126890479DF81C10206808442060E0
:40A700002068401C206009F1010000F0FF0903E010E0C5E08FE0EBE08748006880474845E4DC0020386006202870AFF2D720C8F80000E0E04FF6FF7007900720069003200C
:40A7400005904FF6FF700490012003904FF6FF7002907068002859D002A803A9CDE9001004AB05AA06A907A8D6F804C0E04701284CD1BDF81C00A0F5FA6000F03F006F495B
:40A780000870084600789DF8181001F0030140EA81106A4908709DF81800C0F380004870084640789DF8141001F0030140EA410062494870084640789DF8181001F01801DC
:40A7C00008435E49487008464078BDF8101001F0070140EA411059494870BDF81000C0F3C70088700020C87008719DF80C00C007000E4871BDF808008871BDF80800000A52
:40A80000C871082020600620287001E00020089071E03046FFF7B6FE48490870FF2048708870C870087148718871C87108202060062028705FE04FF0000A0020079083468D
:40A840000690814615E006A805AB07AA494600903046FFF71CFB40B10BF1010000F0FF0B9DF8180050441FFA80FA09F1010000F0FF09B9F1160FE6DD0AF10200032101FB77
:40A880000B0020602068082801D2082020600020386006202870AFF21170C8F800002AE0002007900320206007A82549096888479DF81C1020680844206007A82149096822
:40A8C00088479DF81C1020680844206007A81E49096888479DF81C102068084420600020386006202870AFF25150C8F8000002E00020089000BF00BF08980DB0BDE8F08FF8
:40A9000070477047704710B51048FFF770FA04460F4AAFF6EB212DF0B9FA10BDF4CA1908F8CA1908ECCA1908FCCA1908F0CA1908E8CA19080CCB190810CB190898020020A8
:40A9400000CB190804CB190808CB1908642300200080000870B5044600250226052C13D2DFE804F00306090C0F006C4D02260BE06B4D022608E06B4D022605E06A4D0226E6
:40A9800002E06A4D022600BF00BF25B13246294667483CF1D0FF70BD2DE9F04F89B004460F4690469946C4F800801298606027721398607284F80A900020E072206808B15C
:40A9C000A07A10B90020FFF7C5FF606810B90120FFF7C0FF607A10B90220FFF7BBFF207A022802DB0320FFF7B5FF524A5249204602F01AF818B90420FFF7ACFF63E0227A3A
:40AA0000A17A20683AF10AFA0790002657E0E07A617A884250DA08A80090237AA27A304621683AF161F9002846D04FF0000B002006900898006881680898884702280CD105
:40AA400004A808992DF059FF0120069004A93B4839F14EFE08B1012000E0002082460390069810B104A839F1B9FF00BFDA4522D04FF0000B1C202DF0B9FF824601A8089958
:40AA80002DF03BFF4FF0010B217A002301AA504605F09CF882465546BBF1000F02D001A839F19CFFE07A401CE072606810B128466168884700BF00E004E0701C86B2079891
:40AAC0008642A4DB00BF204609B0BDE8F08F10B50446184A1849204602F0C8FB204610BD02460020086013480088824204DA1248006850F822000860086808B10120704703
:40AB00000020FCE70B48008870470146087A70470146C87A70470146487A7047CCDF0408E0DF040811E0040845E0040859E00408A8DF0408A4020020A0020020A0DF040865
:40AB400070B504460025022614B1012C06D102E0AE4D022602E0AE4D022600BF00BF25B132462946AB483CF1E6FE70BD10B50446A948206000206060A84AA949204601F03F
:40AB800053FF10B90020FFF7DBFF204610BD2DE9F04706460F46904674684FF0000A17B9B8F1000F36D008E02068B84204D16068404501D1A24602E0A468002CF4D100BFFC
:40ABC000BAF1000F23D10C202DF010FF81460020C9F80000C9F804004D46C9F8080085B12F60C5F80480A860AA46706808B975600CE0746800E0A468A0680028FBD1A56065
:40AC000004E00120FFF79CFF4FF0000A05E04FF0000A02E00120FFF793FF5046BDE8F08770B505460E467C48286000206860746805E02846D4E90012FFF7A9FFA468002CFE
:40AC4000F7D1764A7649284601F0EEFE10B90020FFF776FF284670BD10B50446206818B9606808B9A46006E0002020606060A06020462DF0B3FE10BD2DE9F04105460F4630
:40AC80006C680026B0460FE0A7420BD116B9A068686001E0A068B0602046FFF7DDFF4FF0010803E02646A468002CEDD100BF4046BDE8F08110B5044657482060574A5849C8
:40ACC000204602F0D3FA03E020466168FFF7D4FF60680028F8D1204610BD70B504462046FFF7E8FF05462DF079FE70BD0246002008604A480088824204DA4948006850F8DD
:40AD000022000860086808B1012070470020FCE742480088704770B505460C4600262CB1002221462846FFF732FF0646304670BD2DE9F04106460C461546002735B12CB1C0
:40AD40002A4621463046FFF722FF07463846BDE8F08170B505460C4600262CB1224600212846FFF714FF0646304670BD2DE9F04106460F4674680025A846BFB114E06068D7
:40AD8000B8420FD115B9A068706001E0A068A8602046FFF761FF4FF001080DB9746803E0AC6801E02546A468002CE8D14046BDE8F0812DE9F041074688467C6820E02668D8
:40ADC00065680020206060603EB11DB129464046B04708E04046B04705E025B128684146826828469047A068A04203D026606560A46805E00020A06020462DF0EFFD01E0AE
:40AE0000002CDCD100BFBDE8F0810000E1E7040811E80408C7E7040868D619086C0100106801001070B5044600250226082C1DD2DFE804F004070A0D10131619FB4D0226FE
:40AE400014E0FB4D012611E0FA4D01260EE0FA4D02260BE0F94D012608E0F94D012605E0F84D022602E0F84D022600BF00BF25B132462946F5483CF15EFD70BD70B50446C9
:40AE80000D4628197BF100FB25F122F9C0B200EE100AB8EE400ADFEDEE0A20EE200ABCEEC00A10EE100AC0B270BD2DE9F04104460D4690464346FE222946204637F130F94C
:40AEC0000446E4480C3444F80C0C00206060A060E060206120756075FE20A07528462DF02AFD0646FFF7CAFFE075002020766076A076E07601202077002060770C3CD64AE9
:40AF0000D649204601F090FD10B90020FFF78AFF2046BDE8F08110B50446CE482060CE4ACE49204602F0A2F9204637F118F90446204610BD70B504462046FFF7ECFF054646
:40AF40002DF04CFD70BD024600200860C2480088824204DAC148006850F822000860086808B1012070470020FCE7BB480088704730B591B0044613253AF1B2F830B3002031
:40AF80008DF84000EE208DF8410000208DF84200012000210622CDE90124CDE90310032010ABAF4A0121009006A8FEF72AFC00BF9DF83C0005462DB906A8AA49096888470F
:40AFC00000B90D2506A8FEF7C1FA00BF284611B030BD024601207047704770470146002070470146487BFE2805DA91F82000082801D1012070470020FCE770B504460D462A
:40B0000094F82000A84205D0974800688047606184F8205070BD10B50446207B022807DA607BFE2804DA617B207B00222DF048FBFE20607300212046FFF7DFFF0020103480
:40B040006074FE20A07400202060A060E06020756075A075E0750120207600206076103C00BF20463AF1AAFB00BF10BD014691F822007047014691F82000704770B50446DD
:40B080000D462046FFF7F6FF48B9FE2D02DA84F8225002E0FE2084F82200012603E00120FFF7C0FE0026304670BD014691F826007047014691F827007047014691F828005D
:40B0C000704780F828107047014608697047014688697047002180F8261080F82710704770B504460E462046FFF7C4FF0D283FD2DFE800F0070809363738393A0A3B3C3DD2
:40B100000B0000BF00BF00BF00BF94F82200B04221D0FE2E17DA207B022814DA207B31467CF1D2FC38B9012584F8226004212046FFF763FF13E00025012084F82900022062
:40B14000FFF770FE0BE00025012084F829000320FFF768FE03E00025012084F829000CE000BF00BF00BF00BF00BF00BF00BF00BF00250420FFF756FE00BF00BF284670BDB8
:40B180002DE9FC4705460C462846FFF773FF0D2842D2DFE800F007080938393A3B3C0A3D3E3F400000BF00BF00BF4FF0010805F10409A24648462DF0BEFB06460F4650467A
:40B1C0002DF0B9FB46404F403E4301D0012000E00020B8B120462DF0AEFB0646FFF74EFE85F823002E1D20462DF0A5FBCDE90001009830600198706000BF00BF0021284670
:40B20000FFF7FBFE0EE000BF00BF00BF00BF00BF00BF00BF00BF00BF4FF000080520FFF701FE00BF00BF4046BDE8FC874AE804087AE804089BE80408D0E80408FEE80408FC
:40B2400038E904086FE90408A2E9040830E804089A99193F64D40A08AC020020A8020020FEFFEA0058CC19085CCC190810B5014600BF48680246002017E0F84B1B6853F8B5
:40B280002030DB6993420ED10123F44C246854F8204084F8243000BF0B7AF04C246854F8204084F82530431C98B2ED4B1B889842E3DB10BDF0B591B00446002739F110FFD8
:40B2C000002858D020462DF012FB05460E46E8B28DF83C00280A40EA0660C0B28DF83D00280C40EA0640C0B28DF83E00280E40EA0620C0B28DF83F00F0B28DF84000300A48
:40B300008DF84100300C8DF84200300E8DF843000121AFF2A702207B0623CDE90130CDE903210820009094F82200CE4940EA01020FAB012105A8FEF764FA00BF0998E06126
:40B3400005A8FEF751F990B1002084F8240084F8250005A8C44909688847012807D1C34800688047A061002084F82900012705A8FEF7ECF800BF384611B0F0BD10B50446DC
:40B380002046FFF777FE082805D12046FFF792FF08B1012010BD0020FCE770B590B00446002639F19DFE00284ED02046FFF762FE0D2816D2DFE800F0090A0B0C0D0E0F104B
:40B3C000071112131400657B0DE000BF00BF00BF00BF00BF00BF00BF00BF00BF00BF00BF00BFFE2500BF00BF00208DF83C00EE208DF83D0000208DF83E0001210022207B27
:40B400000623CDE90130CDE9032103200090984845EA00020FAB05A8FEF7F3F900BF0998E06105A8FEF7E0F850B105A88E4909688847012804D18D4800688047A06101260C
:40B4400005A8FEF783F800BF304610B070BD70B5044600252046FFF70DFE082807D12046FFF79BFF18B10125012084F82900284670BD2DE9F041044694F82800C8B9207BE3
:40B48000022807DA607BFE2804DA617B207B00222DF016F9FE20607300212046FFF7ADFD00201C34607120602072607260731C3CFEE12046FFF7DEFD0D281CD2DFE800F085
:40B4C000071C303946A0F8F7F6F5F4F3F2002068016A2046884794F82200FE2807D194F82110206842692046904784F8220001212046FFF782FDDAE194F82900012804D11D
:40B5000003212046FFF779FD09E094F82310606901F007FF18B102212046FFF76EFDC6E12046FFF73AFF18B103212046FFF765FDBDE194F8232002F1FA01606901F0F1FE0F
:40B5400018B104212046FFF758FDB0E1002532E094F82210207B7CF1B7FA30B194F82210207B7CF1B1FAA04208D12046FFF7A2FE18B106212046FFF740FD23E0201D2DF0FE
:40B58000CBF918B194F82100FE2801DB012519E094F82100401C84F8210094F82110206842692046904784F8220094F82200FE2801DB012506E094F82200FE2802DA207BB8
:40B5C0000228C5DB00BF012D0ED1002084F8210094F82110206842692046904784F8220005212046FFF709FD94F82200FE2802DA207B022803DB0B212046FFF7FEFC56E199
:40B6000064E094F82210207B7CF15EFA60B194F82210207B7CF158FAA04205D094F82210207B7CF151FAC0B120462DF060F905460E4694F82210207B7CF146FA07462DF05B
:40B6400056F9281A8E4115D22046FFF733FE18B106212046FFF7D1FC3FE00BE0A8020020AC02002000FFEE0058CC19085CCC190800FFEA00201D2DF04FF938B90B212046B2
:40B68000FFF7BBFC0620FFF7CDFB26E094F82100FE280EDB0B212046FFF7AFFC0720FFF7C1FB1AE0F1E0E1E0C0E089E06AE03DE020E094F82100401C84F8210094F82110CC
:40B6C000206842692046904784F8220094F82200FE2802DA207B022893DB00BF94F82200FE2802DA207B022803DB0B212046FFF784FCDCE094F8240001280DD194F825001B
:40B70000012804D107212046FFF777FC0DE004212046FFF772FC08E0FA21606901F001FE18B104212046FFF768FCC0E0607BFE2823DA207B022820DA617B207B7CF1C4F9D0
:40B74000A04204D009212046FFF757FC19E0FA21606901F0E6FD40B108212046FFF74DFC2068C169204688470BE094F82900012807D12046FFF79EFD03E009212046FFF7E2
:40B780003CFC94E0607BFE2815DA207B022812DA617B207B7CF198F9A04204D009212046FFF72BFC0BE094F82900012807D12046FFF780FD03E009212046FFF71EFC76E011
:40B7C00094F82200FE2830DA207B02282DDA94F82210207B7CF178F938B320462DF087F805460E4694F82210207B7CF16DF907462DF07DF8281A8E4108D22046FFF75AFD33
:40B8000098B10A212046FFF7F8FB0EE0002084F8210094F82110206842692046904784F8220002212046FFF7E8FB40E094F82400012811D194F82500012808D10821204650
:40B84000FFF7DBFB2068C169204688470DE009212046FFF7D2FB08E0FA21606901F061FD18B109212046FFF7C8FB20E0002084F82100FE2084F822002046FFF71BFD18B1F2
:40B880000C212046FFF7B9FB11E094F8290001280CD194F82200FE2804D10B212046FFF7ACFB03E004212046FFF7A7FB00BF00BFBDE8F08110B5002407E00649096851F854
:40B8C0002400FFF7D6FD601C84B2034800888442F3DB10BDA8020020AC0200200146FB48704710B50246052300200DE0141D04EB8014646A8C4205D1141D04EB801494F8F4
:40B900003B3003E0441CE0B20528EFDB184610BD0146D1F8440170470146D1F84C01704770B503460024002014E01D1D05EB80156D6A8D420CD101261D1D05EB801585F83A
:40B9400038601D1D05EB801585F83920012403E0451CE8B20528E8DB204670BD10B50446002120463BF1AFF904460020203444F8140C44F8100C44F80C0C44F8080C401E36
:40B9800044F8040C20606060A0600020E06020826082A082FF20A0750020E07520766076A076E07620776077203C204610BD10B504462046FDF768FB0446C54820600523AC
:40B9C0004022AFF26701201D7CF17FF9041F002004F5A2742060FDF7EDF960600020A06020736073A4F5A274204610BD10B50446B748206005234022B649201D7AF167FFC1
:40BA00002046FDF768FB0446204610BD70B504462046FFF7EBFF05462CF0E0FF70BD70B5044600250226132C44D2DFE804F00A0D101316191C1F2225282B2E3134373A3D59
:40BA40004000A54D022635E0A44D022632E0A44D02262FE0A34D02262CE0A34D022629E0A24D022626E0A24D022623E0A14D022620E0A14D02261DE0A04D02261AE0A04D63
:40BA8000022617E09F4D002614E09F4D022611E09E4D00260EE09E4D00260BE09D4D002608E09D4D022605E09C4D012602E09C4D012600BF00BF25B13246294683483BF13E
:40BAC0003AFF70BD70B5054600BF68680646002413E0944800EB8410C069B0420BD100BF287A10B90020FFF79AFF01218D4800EB841080F83A10601CC4B2052CE9DB70BD07
:40BB00002DE9FE43054600BF686880460024AAE0844800EB8410C069404578D12868816828468847002873D0012872D0022802D003286FD186E02F46FF22082101A87AF1F2
:40BB40007CFD00BFB869B0B9764800EB8410008E072807DC734800EB841090F830008DF8040002E0FF208DF80400012201A9384635F187FF63E06B4800EB8410008E0728F8
:40BB800025DC684800EB8410806960B1654800EB8410028E634800EB841000F1180101A82CF0F2F90DE05F4800EB8410008E00905C4800EB8410002301AA016A5A483BF160
:40BBC000ABF9072201A9384635F15BFF37E000BFD7F81C9038467CF128F8A9EB0006082E00D908264F4800EB8410806998B138467CF11BF8411E4B4800EB8410806901EB11
:40BC000000093246494601A87AF1D2FC12E028E016E016E023E038467CF107F8A0F10109404800EB841000964B4601AA016A3E483BF172F9324601A9384635F122FF0EE06E
:40BC400000BF00BF00BF287A10B90120FFF7E7FE0121344800EB841080F8371000BF00BF04E0601CC4B2052CFFF652AFBDE8FE8370B504460D46002C26D02B48216A3BF195
:40BC8000E6F920463AF1B4FF0020203444F8140C44F8100C44F80C0C44F8080C401E44F8040C20606060A0600020E06020826082A082FF20A0750020E07520766076A0767A
:40BCC000E07620776077203C70BD000033C319084CD50A08977B190852C319087FC31908A4C31908F4C3190812C419082CC4190848C4190863C419087FC419089EC419081D
:40BD0000B3C41908E1C4190814C5190843C5190877C51908AEC51908D1C51908DDC5190802C61908C4230020142500202DE9F04F89B006460F4614469846DDE9149BDDE92C
:40BD4000125AE0B28DF81C0011208DF81D009DF81D0008F0070140EA41008DF81D009DF81D0004F4E06140EAE1008DF81D00E8B28DF81E00280A8DF81F00280C8DF820000E
:40BD80008DF821A009F0FF008DF822004FEA29208DF8230000211698CDE9021BCDE9040106203346082207A9CDE900704FF458403AF13AFC18B9012009B0BDE8F08F00204D
:40BDC000FAE72DE9F84304460D46012620462CF09DFDA8B1002600BFE06888B120462CF095FD074620467BF120FF8146E068804600974B464246F648296A3BF1FDF906465C
:40BE00003046BDE8F88370B50446002515B10220FFF705FEEF48006810B90320FFF7FFFDED48006810B90420FFF7F9FDEB48006810B90520FFF7F3FDE948006810B906200D
:40BE4000FFF7EDFDE748006810B90720FFF7E7FDE548006810B90820FFF7E1FD21464FF4594039F15BFA21464FF4574039F156FA70BD30B50346002401B9DAB1002017E0CF
:40BE80001D1D05EB801595F83D507DB11D1D05EB80152D698D4209D11D1D05EB8015ED68954203D11D1D05EB801403E0451CE8B20528E5DB204630BD2DE9F04704460D46F8
:40BEC00000BF05F10C00FCF763FE0746B7F5574F15D0B7F5594F48D12946C448D4F84821FCF78BFF38B90920FFF799FDD4F84401401CC4F84401012084F8510139E000BF34
:40BF000068688046A8688146424649462046FFF7B0FF064606B3B64800688047F06230463AF16CFFB0F1FF3F0DD1294630463AF16BFEC8B90A20FFF772FDD4F84401401C2F
:40BF4000C4F8440110E00B20FFF769FDD4F84401401CC4F8440107E00C20FFF760FDD4F84401401CC4F8440103E01020FFF757FD00BF00BFD4F84C01401CC4F84C01BDE809
:40BF8000F08770B505460E46002419E0281D00EB841090F83D0090B15EB1281D00EB8410C068B04205D0281D00EB84100069B04205D1291D01EB84100121FFF759FE641CF3
:40BFC000052CE3D370BD2DE9F04F91B082460C4694F83D00082872D2DFE800F0F9F804F7F6F5F4F3E56894F83A00012868D1804800688047E06294F83B0008287ED2DFE80F
:40C0000000F00413B9CBCCCDBDCE94F83670A06A40EA0761628E2846704F636A3F68B847052084F83D00C0E00020109004F1140010AB04F13001021DCDE9031302920590B7
:40C04000618E606ACDE9001094F8363094F83C102846634FA26A3F68B8479DF8400000281AD1A069C8B1218E04F1200258483BF143F878B1208E009000235548A269216AB1
:40C080003BF1BAF830B95248216A3AF1E0FF4FF0FF3020620020A06168E06069002865D0218E04F120024A483BF126F800285DD04FF000080027B9464FF0010B50E002E248
:40C0C00074E0208EB84239D90122218E606A3B46CDE90018CDE902022246AFF2193105A835F198FC05A86169884708F1010800BF9DF83D0040B100BF089800E050E030B9B1
:40C1000005A82CF003FC10B14FF0000B12E005A82CF0FCFB60B100BF9DF83C0008B94FF0000B05A82CF0F2FB07444FF0000901E009F1010905A835F190FC06E0208EB842B3
:40C1400002D24FF0000B00E00EE0BBF1000F07D11F48216A3AF17BFF4FF0FF30206203E009F101000028ACD100BF00BF052084F83D001AE0042084F83D0016E094F836301B
:40C18000A06A40EA03612846174B626A1B689847052084F83D0008E000BF00BF00BF00BF01212046FFF764FD00BF09E041F28831E06A01F0B6F818B101212046FFF758FD2F
:40C1C00081E14BE121E185E03DE013E070E16EE11425002020F7040824F7040828F704082CF7040830F7040834F704083C2200205CCC19082669E5684FF4FA71E06A01F0A7
:40C2000090F8A8B100204FF6FF72FF23CDE9022001930490D01C0090628E052331462846FFF784FD70B101212046FFF721FD09E041F28831E06A01F074F818B101212046AB
:40C24000FFF716FD3FE1E56894F83B0008283AD2DFE800F0323304343536373820463AF1CDFDB0F1FF3F1CD0012321460DA8626AFCF7BCFB54F8240FA17CCDE90010227E39
:40C280000DA92846FD4F63683F68B847FC4800688047A06005206076243C0DA8FCF7B8FB09E047F23051E06A01F03BF818B101212046FFF7DDFC0BE000BF00BF00BF00BF5C
:40C2C00000BF00BF00BF01212046FFF7D1FC00BF00BFF8E02669E56894F83800012871D194F8390001286FD194F83B00082863D2DFE800F0440445464748494A208EB0F5FC
:40C30000DF6F25DCA06918B9206AB0F1FF3F1FD0208E471C082F00D208270021AFF61F0204F11C00CDE9021006202B46CDE90060CDE904213A464FF457403AF175F930B90F
:40C34000CF4800688047E062062084F83D0014E000204FF6FF72FF23CDE9022001930490581C0090628E052331462846FFF7DEFC18B101212046FFF77BFC22E000BF00BF5B
:40C3800000BF00BF00BF00BF00204FF6FF72FF23CDE902200490CDE90003628E042331462846FFF7C3FC30B1B54800688047E062072084F83D0004E001212046FFF758FCCE
:40C3C00000BF21E016E0FFE700204FF6FF72FF23CDE9022001930490581C0090628E052331462846FFF7A2FC70B101212046FFF73FFC09E047F23051E06A00F092FF18B103
:40C4000001212046FFF734FC5DE02669E56894F83700012817D100204FF6FF72FF23CDE902200490CDE90003628E042331462846FFF77CFC88B1924800688047E06207202F
:40C4400084F83D0009E041F28831E06A00F069FF18B101212046FFF70BFC34E02669E5684FF4FA71E06A00F05CFFA8B100204FF6FF72FF23CDE9022001930490D01C00903E
:40C48000628E052331462846FFF750FC70B101212046FFF7EDFB09E041F28831E06A00F040FF18B101212046FFF7E2FB0BE000BF4FF4FA61E06A00F034FF18B1012120463E
:40C4C000FFF7D6FB00BF00BF11B0BDE8F08F70B505460026002418E0281D00EB841090F83D0080B9664800688047291D01EB8411C8620121281D00EB841080F83D10281DE0
:40C5000000EB841603E0601CC4B2052CE4DB304670BD2DE9F04F89B006460D4600200890686800287ED0286800287CD0E868B0F5594F79D12868026891688847002874D1C9
:40C54000D5F804902F68A97DE87D41EA0021287E41EA004A297D687D00F0E00041EAC00BA97EE87E41EA00200790687E0690687DC0F34208687DC0F3001005903A46494667
:40C580003046FFF776FC0446002C7DD13046FFF79EFF0446002C78D020463AF129FBE760C4F8109000206061A061401EE061206235F1E2FB6062C4F828A0069884F836001E
:40C5C000059884F83C00A4F832B084F83B804FF6FF70A0862A4800688047E0620020208684F8370084F8380084F8390084F83A0004F13400009094F83B2049463846DFF858
:40C6000084C0079BDCF800C0E047012821D10021A08EFF23CDE90201481ECDE900030491628E03E087E180E178E176E10B4649463846FFF77BFB38B1032084F83D00012064
:40C6400086F85001089067E101212046FFF710FB62E1022084F83D00AFF6973104F11C004FF6FF72FF23CDE90132CDE903014FF0FF300090628E0023494607E030F70408B1
:40C680005CCC190820F7040823E00DE03846FFF74DFB20B1012086F8500108903CE101212046FFF7E5FA37E100204FF6FF72FF23CDE9022001930490022001230022494688
:40C6C00000903846FFF732FB0028BCD00120089022E194F83D00082878D2DFE800F0878889048A8B8C78A06A504558D1608E584555D194F836100698814250D194F83B0056
:40C7000040454CD194F83C100598814247D107980090A38E94F83B2049463846DFF8C8C2DCF800C0E047012821D1022084F83D00002084F83A00AD4800688047E062AFF6C0
:40C740007B4104F11C004FF6FF72FF23CDE90132CDE903014FF0FF300090628E002349463846FFF7E3FA88B3012008902EE000204FF6FF72FF23CDE902200193049041F253
:40C78000030001230022494600903846FFF7CEFAE0B10D20FFF743F90120089016E000204FF6FF72FF23CDE90220019304904FF4805001230022494600903846FFF7B6FAA2
:40C7C00020B10E20FFF72BF901200890A3E0B8F1040F04D100212046FFF74AFA03E001212046FFF745FA0120089094E000BF00BF00BF00BF00BF0F20FFF711F994F83B0014
:40C80000082874D2DFE800F00416283A71724C5E00204FF6FF72FF23CDE9022001930490102001230022494600903846FFF77EFA08906EE000204FF6FF72FF23CDE9022093
:40C8400001930490112001230022494600903846FFF76CFA08905CE000204FF6FF72FF23CDE9022001930490122001230022494600903846FFF75AFA08904AE000204FF6CE
:40C88000FF72FF23CDE9022001930490132001230022494600903846FFF748FA089038E000204FF6FF72FF23CDE9022001930490162001230022494600903846FFF736FAB0
:40C8C000089026E000204FF6FF72FF23CDE9022001930490172001230022494600903846FFF724FA089014E001E000BF00BF00204FF6FF72FF23CDE90220019304901F2052
:40C9000001230022494600903846FFF70FFA089000BF00BF00BF00BF00BF05E01020FFF77EF80120089000BF0AE01120FFF777F80120089004E01220FFF771F80120089062
:40C94000089809B0BDE8F08F2DE9F041044694F8510101281FD1002084F85101002517E02348D4F84811FCF7B8FA0646002766B1012084F8510131462046FFF7CAFD20B18F
:40C9800031461B48FCF7DBFA012707B902E06D1C0A2DE5D300BF94F85001012816D1002084F8500100250FE0201D00EB851090F83D0040B1012084F85001201D00EB8511C7
:40C9C0002046FFF700FB6D1C052DEDD3BDE8F08110B50848FEF7EBFF0446074AAFF6F3712BF054FA10BD000024F704085CCC19083C220020C02300200080000870B5044699
:40CA00000025022614B1012C06D102E0FE4D022602E0FE4D022600BF00BF25B132462946FB483AF188FF70BD2DE9F04107460D4614464FF00008002657B320884FF6FF71C4
:40CA4000884229DA2188491C0904880B2BF0CAFF0646F6B14FF0010800200AE0296851F8201046F8201000212A6842F82010411C88B221888142F1DC208846F820702868A7
:40CA800010B128682BF0A6FF2E602088401C208002E00020FFF7B2FF4046BDE8F0810246082909DCC1F1080302FA03F3DAB250B2C1F10803184100E050B270470246102923
:40CAC00009DCC1F1100302FA03F39AB210B2C1F11003184100E010B270470246202907DCC1F120039A401046C1F12003184100E0104670472DE9F74F9046B8F1400F16DC65
:40CB0000C8F14002DDE9009A4846514667F1DAF9CDE90001DDE90067C8F1400234463D462046294679F1DDFB06460F4601E0DDE900673046394603B0BDE8F08F2DE9FC4783
:40CB400007460D4616461C46DDF828804FF00009FF202070002F5ED0002E5CDD082E5ADCB8F1000F03D0B8F1010F53D131E04FF001090020207000BF1AE005F00702C2EBDD
:40CB8000C00251B200290ADA227800EBD503FB5CC1F1000C43FA0CF31A43227007E0227800EBD503FB5C8B40DBB21A432270401C711E05F007021144012202EBD101814241
:40CBC000DBD82078C6F10802FF2111410840207020E0701E05F007010844012101EBD00A002008E000EBD5017A5C411CAAEB010101AB5A54401C5045F4D300200090A8190A
:40CC0000404200F007012346324601A8FFF796FF814600BF00BF4846BDE8FC872DE9FC4707460D4616461C46DDF828804FF000094FF6FF702080002F5FD0002E5DDD102E96
:40CC40005BDCB8F1000F03D0B8F1010F54D132E04FF001090020208000BF1AE005F00702C2EBC00251B200290ADA228800EBD503FB5CC1F1000C43FA0CF31A43228007E01F
:40CC8000228800EBD503FB5C8B409BB21A432280401C711E05F007021144012202EBD1018142DBD82088C6F110024FF6FF7111410840208020E0701E05F0070108440121AA
:40CCC00001EBD00A002008E000EBD5017A5C411CAAEB010101AB5A54401C5045F4D300200090A819404200F007012346324601A8FFF794FF814600BF00BF4846BDE8FC87D0
:40CD00002DE9FE4707460D4616461C46DDF82C804FF000094FF0FF302060002F5ED0002E5CDD202E5ADCB8F1000F03D0B8F1010F53D131E04FF001090020206000BF19E021
:40CD400005F00702C2EBC00251B200290ADA00EBD503FB5CC1F1000C23FA0CF322681A43226006E000EBD503FB5C8B4022681A432260401C711E05F007021144012202EB57
:40CD8000D1018142DCD8C6F120024FF0FF31D14020680840206020E0701E05F007010844012101EBD00A002008E000EBD5017A5C411CAAEB010101AB5A54401C5045F4D31D
:40CDC00000200090A819404200F007012346324601A8FFF795FF814600BF00BF4846BDE8FE872DE9F04F8BB080460D4616461C4600200590411E21606160B8F1000F7DD075
:40CE0000002E7BDD402E05E03EC9190868C9190821C9190879DC149810B1012874D150E00120059000212160616000272FE005F00700C0EBC70040B204900498002812DA41
:40CE400007EBD50018F800000021049A5242D2B2CDE906102AF0C2FED4E9003218431143C4E9000112E007EBD50018F800900020D4E900AB049A08904846089967F122F85A
:40CE80004AEA000A4BEA010BC4E900AB7F1C701E05F007010844012101EBD000B842C6D8C6F14002891ED4E900A70A91084609912AF094FE0AEA000207EA0103C4E90023C5
:40CEC00022E0701E05F007010844012101EBD007002008E000EBD50118F80120411C791A02AB5A54401CB842F4D300200090A819404200F007012346324600E005E002A8D7
:40CF0000FFF76FFF059000BF00BF05980BB0BDE8F08F2DE9FE4705460C4616461F46DDF82C904FF0000A002D7ED0002E7CDD202E7ADCB9F1000F03D0B9F1010F55D155E024
:40CF4000C6F120024FF0FF3020FA02F10F404FF0010A00203FE0C20021FA02F204F007039A4000EBD403EB5C23EA020200EBD403EA54C20021FA02F204F00703C3F1080334
:40CF8000DA4000EBD4035B1CEB5C934300EBD402521CAB54C30027FA03F204F007039A40D2B200EBD403EB5C1A4300EBD403EA54C30027FA03F204F00703C3F10803DA4088
:40CFC000D2B200EBD4035B1CEB5C134300EBD402521CAB54401C721ED31702EB53734FF0010C0CEBE3038342B5D831E0701E04F007010844012101EBD008002008E000EBE5
:40D00000D4016A5C411CA8EB010101AB5A54401C4045F4D300200090A019404200F007013B46324601A800E013E0FFF772FF70B1002008E0411CA8EB010101AA515C00EB44
:40D04000D402A954401C4045F4D34FF0010A00BF00BF5046BDE8FE872DE9F04F99B082460C469346DDE9225600200690BAF1000F7DD0BBF1000F7ADDBBF1400F77DC249805
:40D0800010B1012874D189E0CBF140024FF0FF310891084607912AF0A1FD074688463D4006EA0806012006904FF000096BE04FEAC90238464146CDE917872AF08FFD04F05D
:40D0C0000702CDE9151066F1FDFE09EBD4011AF8011021EA000009EBD4010AF801004FEAC90238464146CDE913872AF077FD04F00702C2F10802CDE911102AF06FFD09EB45
:40D10000D401491C1AF80110814309EBD400401C0AF800104FEAC90228463146CDE90F652AF05CFD04F00702CDE90D1066F1CAFEC0B209EBD4011AF80110084309EBD401B1
:40D140000AF801004FEAC90228463146CDE90B652AF044FD04F00702C2F10802CDE909102AF03CFDC1B209EBD400401C01E049E047E01AF80000084309EBD401491C0AF811
:40D18000010009F10109ABF10100C11700EB5171012202EBE101494589D832E0ABF1010004F007010844012101EBD007002008E000EBD4011AF80120411C791A03AB5A5444
:40D1C000401CB842F4D30020CDE90056029004EB0B00404200F007015A4603A8FFF73CFF70B1002008E0411C791A03AA515C00EBD4020AF80210401CB842F4D30120069048
:40D2000000BF00BF069819B0BDE8F08F02468A4201D3501A03E0C1F1FF331344581C7047B0EE402AF0EE602A81EE210AF0EE400AB7EE000AF4EEC00AF1EE10FA04DDB7EE4E
:40D24000000AF0EE400A08E0F5EEC00AF1EE10FA03D29FED440AF0EE400AB7EE000A30EE600A20EE220A02EE200A70472DE9F04107460C4615464FF0000800262068002887
:40D2800042D0002010E0216851F82010B94209D14FF001080021226842F820102988491E298004E0411C88B229888142EBDC288828B920682BF08EFB0020206024E0B8F197
:40D2C000010F21D1298888002BF08CFB0646A6B1002100200CE0226852F8202032B1226852F8202046F821204A1C91B2421C90B22A88521C8242EEDC02E00120FFF77EFB8E
:40D3000020682BF067FB26604046BDE8F08170B5044615480068804705462146FFF776FF70BD2DE9F04104460D460F48006880470646A64207D3301BA84201D3012000E0FF
:40D340000020074609E0C4F1FF303044401CA84201D3012000E0002007463846BDE8F08170477047000000005CCC190870B50446002502260C2C2BD2DFE804F006090C0F56
:40D380001215181B1E212427F84D022620E0F84D02261DE0F74D02261AE0F74D022617E0F64D022614E0F64D002611E0F54D01260EE0F54D01260BE0F44D012608E0F44DF4
:40D3C000022605E0F34D012602E0F34D012600BF00BF25B132462946F0483AF1ACFA70BD70B504460D462046FBF7CFFC04466560204670BD2DE9F0410546E9480468002722
:40D4000008E06068A84201D1274605E020467AF111FB0446002CF4D100BFB7B908202BF0E5FA06462946FFF7DBFF0646344644B127462146DA480068FBF7F4FBD8490860B7
:40D4400002E00020FFF792FF03E00020FFF78EFF00273846BDE8F081F8B505462C46002000906A462146CE480068FBF763FCCC4908609DF80000012807D134B12646304608
:40D48000FBF786FC07462BF0A9FA9DF80000F8BD70B588B004460D461646E0B28DF81C00200A8DF81D00200C8DF81E000020029003900490059006202B46032207A9CDE9EF
:40D4C00000604FF46A4039F1AFF810B9012008B070BD0020FBE70146B04870470146D1F8F40070470146D1F8F80070470146D1F8FC0070470146D1F8000170470146D1F832
:40D50000040170470146D1F80C01704770B50546002600241EE004EB4401281D00EBC100007DA8B99F480068804704EB4402291D01EBC2010861012104EB4402281D00EB70
:40D54000C200017504EB4401281D00EBC10603E0601CC4B20A2CDEDB304670BD2DE9F043044607ADE0CD4FF0000CE1B3DAB3002050E000EB400904F1040808EBC90898F8A8
:40D580001480B8F1000F41D000EB400904F1040808EBC908D8F80C80984537D100EB400904F1040808EBC90898F81580A8452DD100EB400904F1040808EBC90898F81680AC
:40D5C000B04523D100EB400904F1040808EBC908D8F80480884519D100EB400904F1040808EBC90800E017E0D8F80880904506D0082F0BD803F47048B8F5704F06D100EB74
:40D60000400904F1040808EBC90C05E000F1010808F0FF000A28ACDB6046BDE8F08370B505465F480468002608E06068A84201D1012605E020467AF1FDF90446002CF4D168
:40D6400000BF304670BD2DE9F04F91B007460E4690461D46DDE91AA900201090002E72D02846FFF7DCFF00286ED1B8F1000F6DD1012010904FF0000BA3E00FA95846FDF7AB
:40D6800062FC002871D000BF317B0F98027B91426BD100200E900D900C900B9006200A90002009900DA80EA909AA0AABCDE90332CDE905100BA80CA953462A46CDE90091B8
:40D6C000029031460F9837F1F1FF00286ED0012802D002286CD16AE00B982B463246CDE900A9029038460F99FFF738FF044664BB00209DF82430DDE90D12CDE90232CDE989
:40D7000004109DF828000021CDE9001028460F9BDDE90B2138F188FF08B33846FFF7F6FE0446A4B1C4F800800F986060A660E56084F815A084F816901A4800688047206162
:40D740000220207510E04BE148E109E03FE00320FFF70CFED7F8FC00401CC7F8FC0003E0104800688047206126E026E0B7EB0408F5EB040845EC040859EC040883EC040806
:40D780009AEC0408BCEC0408D4EC0408FFEC040822ED04082EED040853ED04088FEB0408D40200205CCC190800E001E000BF03E00420FFF7DBFD00BF00BF0BF101001FFA24
:40D7C00080FBFDF7D2FB58453FF757AF02E100200E900D900C900B9006200A90002009900DA80EA909AA0AABCDE90332CDE905100BA80CA953462A46CDE9009102903146DB
:40D80000404637F153FF20B1012835D002287CD1AAE001208DF81C00FF208DF81D008DF81E008DF81F0030467AF1F9F98DF82000E8B28DF82100280A8DF82200280C8DF8D4
:40D8400023000020029003900490059006204346082207A9CDE900604FF4684038F1E4FE48B90520FFF782FDD7F80001401CC7F8000101201090ABE00B982B46324641469C
:40D88000CDE900A902903846FFF768FE0446002C63D19DF82430DDE90D12CDE90232CDE904109DF828004346CDE900602846DDE90B2138F1B9FE48B33846FFF727FE0446F7
:40D8C00094B101201090C4F80080C4F80480A660E56084F815A084F81690F848006880472061022020753EE003208DF81C00FF208DF81D008DF81E008DF81F0030467AF196
:40D900008EF98DF82000E8B201E05DE022E08DF82100280A8DF82200280C8DF823000020029003900490059006204346082207A9CDE900604FF4684038F176FE98B906209A
:40D94000FFF714FDD7F8F400401CC7F8F4000120109008E00120109005E0D8480068804720610120109033E000208DF81C00FF208DF81D008DF81E008DF81F0030467AF131
:40D980004EF98DF82000E8B28DF82100280A8DF82200280C8DF823000020029003900490059006204346082207A9CDE900604FF4684038F139FE30B9D7F80401401CC7F856
:40D9C00004010120109003E00420FFF7CFFC00BF00BF00BF012087F8110101E001201090109811B0BDE8F08F00210160416081606FF07F41C160002101610175FF21417568
:40DA00008175704710B504462046FBF73DFB0446AB4820600A231822AFF23301201D7AF154F9041F002044F8F40F6060A060E0602061FBF7BFF960610020A06120776077AF
:40DA4000F43C204610BD10B504462046FBF743FB0446204610BD70B504462046FFF7F3FF05462AF0BBFF70BD70B50446002515B10120FFF77BFC4FF46E40FFF7BBFC21462B
:40DA80004FF46A4037F14AFC70BD7CB504460D46286808226946036928469847012816D129468848D4F80821FBF7A7F938B90220FFF75CFCD4F8F800401CC4F8F8000120C2
:40DAC00084F81001D4F80C01401CC4F80C017CBD30B50246002036E000EB4004131D03EBC4031B7D73B3B1B100EB4004131D53F834308B420FD000EB4004131D03EBC403FD
:40DB00005B688B4207D000EB4004131D03EBC4039B688B4216D1002400EB4005131D03EBC5031C7500EB4005131D43F8354000EB400503EBC5035C6000EB4005131D03EBE8
:40DB4000C5039C60401C0A28C6D330BD2DE9F04F8FB006460F4690461D46DDE919A9189C4FF0000B00200E900D900C900B900A9006200990B8F1000F3DD10CA80DA90EAA06
:40DB800009ABCDE90332CDE905100AA80BA953462246CDE9009102902946384637F186FDF0B1012802D002281ED11AE000209DF83830DDE90C12CDE90232CDE904109DF82A
:40DBC000240000213B46CDE900102046DDE90A2138F12AFD08B9012000E00020834609E000BF4FF0010B05E00420FFF7BFFB4FF0010B00BFA5E00CA80DA90EAA09ABCDE980
:40DC00000332CDE905100AA80BA953462246CDE9009102902946384637F148FD20B1012835D002287ED152E001208DF81C00FF208DF81D008DF81E008DF81F00284679F1FE
:40DC4000EEFF8DF82000E0B28DF82100200A8DF82200200C8DF823000020029003900490059006203B46082207A9CDE900504FF4684038F1D9FC48B90520FFF777FBD6F8FB
:40DC80000001401CC6F800014FF0010B57E000209DF83830DDE90C12CDE90232CDE904109DF824003B46CDE900502046DDE90A2138F1BAFC40B9012007E000005CCC190851
:40DCC0001CD819083C2200200020834637E000208DF81C00FF208DF81D008DF81E008DF81F00284679F19BFF8DF82000E0B28DF82100200A8DF82200200C8DF823000020B4
:40DD0000029003900490059006203B46082207A9CDE900504FF4684038F186FC40B9D6F8040100E005E0401CC6F804014FF0010B05E00420FFF71AFB4FF0010B00BF00BFA0
:40DD400000BF58460FB0BDE8F08F30B589B005460C46207D02286BD1A07D617DE268CDE9002102902846D4E901132268FFF7EEFE10B1002020755DE040F2DC512069FFF7BB
:40DD8000D0FA50B10720FFF7F1FAD5F8FC00401CC5F8FC00002020754CE04FF47A712069FFF7BFFA002845D02068A8B303208DF81C00FF208DF81D008DF81E008DF81F007F
:40DDC000A06879F12CFF8DF82000207B8DF82100A089000A8DF82200E068000C8DF82300002002900390049006210590A068CDE90001082207A94FF46840636838F114FCAD
:40DE000048B90620FFF7B2FAD5F8F400401CC5F8F400002020750DE0FFE70820FFF7A6FAD5F8FC00401CC5F8FC000020207501E00020207509B030BD2DE9FC4105460C4646
:40DE40000026606830B3206820B12068026891688847D0B9E068B0F56A4F10D1FF2000900190277D607D47EA0027A07D47EA00432846D4E90021FFF7E6FB064604E0092088
:40DE8000FFF774FA012600BF08E00A20FFF76EFA012603E00B20FFF769FA01263046BDE8FC812DE9F041044694F8100101281FD1002084F81001002517E02348D4F80811FB
:40DEC000FBF70BF80646002766B1012084F8100131462046FFF7B0FF20B131461A48FBF72EF8012707B902E06D1C0A2DE5D300BF94F81101012819D1002084F8110100252C
:40DF000012E005EB4501201D00EBC100007D50B1012084F8110105EB4502201D00EBC2012046FFF712FF6D1C0A2DEAD3BDE8F08110B50648FFF766FD0446054AAFF2F941A1
:40DF400029F0A4FF10BD00003C220020783900200080000870B505460C460020FE490870FE48006830B1FD4800682AF033FD0020FA490860DCB1D5B1E0002AF033FDF749D2
:40DF8000086000200FE005EBC0010979F34A126802EBC002117155F83010F04A126842F83010411CC8B2A042EDDBEB48047070BD2DE9FF410646306881683046884700282F
:40DFC00062D0012861D0022802D003285FD15DE03746384679F12CFE58B941208DF8040026208DF80500022201A9384633F149FD49E0384679F11CFE401E1FFA80F8694628
:40E00000404637F137F8002834D000982AF06FFC04460D46009879F105FE8DF80400E0B28DF80500200A40EA0560C0B28DF80600200C40EA0540C0B28DF80700200E40EACC
:40E040000520C0B28DF80800E8B28DF80900C5F30720C0B28DF80A00C5F30740C0B28DF80B00280E8DF80C00092201A9384633F108FD07E0FF208DF80400012201A9384656
:40E0800033F1FFFC00BF02E000BF00BF00BF00BFBDE8FF812DE9F04188B00646306881683046884700287DD001287CD0022802D0032879D196E03746384679F1B9FD58B9F1
:40E0C00041208DF80C0025208DF80D00022203A9384633F1D6FC82E0384679F1A9FD401E1FFA80F802AA01A9404601F0F7FD00286CD002982AF0FBFB04460D46029879F1C4
:40E1000091FD8DF80C00029879F189FD8DF80D00E0B28DF80E00200A40EA0560C0B28DF80F00200C40EA0540C0B28DF81000200E40EA0520C0B28DF81100E8B28DF8120068
:40E14000C5F30720C0B28DF81300C5F30740C0B28DF81400280E8DF8150001982AF0C7FB04460D46019879F15AFD8DF81600E0B28DF81700200A40EA0560C0B28DF81800DF
:40E18000200C40EA0540C0B28DF81900200E40EA0520C0B28DF81A00E8B28DF81B00C5F3072002E01CE01CE01DE0C0B28DF81C00C5F30740C0B28DF81D00280E8DF81E0037
:40E1C000132203A9384633F15CFC07E0FF208DF80C00012203A9384633F153FC00BF02E000BF00BF00BF00BF08B0BDE8F0812DE9FF4106463068816830468847002867D0BB
:40E20000012866D0022802D0032864D162E03746384679F10DFD58B941208DF8040024208DF80500022201A9384633F12AFC4EE0384679F1FDFC401E1FFA80F869464046E0
:40E2400001F037FD002839D000982AF050FB04460D46009879F1E6FC8DF80400009879F1DEFC8DF80500E0B28DF80600200A40EA0560C0B28DF80700200C40EA0540C0B2FA
:40E280008DF80800200E40EA0520C0B28DF80900E8B28DF80A00C5F30720C0B28DF80B00C5F30740C0B28DF80C00280E8DF80D000A2201A9384633F1E4FB07E0FF208DF89E
:40E2C0000400012201A9384633F1DBFB00BF02E000BF00BF00BF00BFBDE8FF812DE9FF410646306881683046884700286CD001286BD0022802D0032869D167E03746384640
:40E3000079F196FC58B941208DF8040023208DF80500022201A9384633F1B3FB53E0384679F186FC401E1FFA80F869464046FCF70AFE00283ED000982AF0D9FA04460D46E7
:40E34000009879F16FFC8DF80400009879F167FC8DF80500E0B203E0E0020020DC0200208DF80600200A40EA0560C0B28DF80700200C40EA0540C0B28DF80800200E40EA0F
:40E380000520C0B28DF80900E8B28DF80A00C5F30720C0B28DF80B00C5F30740C0B28DF80C00280E8DF80D000A2201A9384633F168FB07E0FF208DF80400012201A93846AF
:40E3C00033F15FFB00BF02E000BF00BF00BF00BFBDE8FF812DE9FE4F0646306881683046884700287CD001287BD0022802D0032879D177E0B246504679F11AFC58B9412038
:40E400008DF8000022208DF8010002226946504633F137FB61E0504679F10AFC401EC7B2504679F105FC401EC0F30728384641464FF00009FE2808DA022906DAC1EBC11292
:40E44000F74B03EBC20252F82090B9F1000F01D0012200E00022012A33D148462AF047FA04460D468DF800808DF80170E0B28DF80200200A40EA0560C0B28DF80300200C57
